:100000000C94D0120C9452130C9479130C94A013EA
:100010000C94D8200C9406210C9434210C94622169
:100020000C94F5120C94F5120C94F5120C94F51234
:100030000C94F5120C9432180C94F5120C94F512E1
:100040000C9453220C94F5120C94F5120C94F512A6
:100050000C94A4190C941E190C94E4180C94F51229
:100060000C94F5120C94F5120C94F5120C94F512F4
:1000700010111213141516171B1D1F080B00010277
:1000800003040506074453313853323000445331DA
:10009000383232004453313842323000756E6B6F63
:1000A000776E2066616D696C7920636F6465001AF4
:1000B0001C1E253032783A253032783A2530327895
:1000C0003A253032783A253032783A253032780085
:1000D00025642E25642E25642E2564004448435053
:1000E000206D736720747970652035332076616CDC
:1000F00075652025750D0A0044484350206D7367CF
:1001000020747970652035332076616C7565202503
:10011000750D0A004950004D41534B00444E5300A9
:100120004741544500444843502D436F6E6669670C
:10013000206765686F6C740D0A00444843502D4376
:100140006F6E666967204665686C67657363686C87
:100150006167656E0D0A00207C2D3E205665727326
:100160007563686520444843502D436F6E66696728
:10017000207A7520686F6C656E2E20000D0A25733D
:1001800000206665686C67657363686C6167656E9F
:100190000D0A00206665686C67657363686C61674B
:1001A000656E0D0A00205A6569743A202530326464
:1001B0003A253032643A253032642E253032640DCF
:1001C0000A004E5450534552564552005554435A16
:1001D0004F4E4500207C2D3E204E54502D536572CD
:1001E000766572205A65697420616B7475616C69FB
:1001F00073696572656E3A006F6E004E5450002050
:100200007C202020444E53202020203A2025730DAE
:100210000A00207C202020476174657761793A20AC
:1002200025730D0A00207C2020204E65746D6173BB
:100230006B3A2025730D0A00207C20202049502095
:10024000202020203A2025730D0A006F6E004448BC
:100250004350004448435000207C2D3E20544350DE
:100260002028487572726963616E2D656E67696ECC
:10027000652920696E697469616C69736965727456
:100280000D0A00207C2D3E205544502028546F72CA
:100290006E61646F2D656E67696E652920696E6990
:1002A0007469616C6973696572740D0A002D2B2D78
:1002B0003E2041525020696E697469616C697369AE
:1002C0006572740D0A00204C696E6B207265616462
:1002D000790D0A002046756C6C6475706C65783A0F
:1002E00000454E4332386A363020285265762E3A21
:1002F0002025642920696E697469616C6973696578
:10030000727420282048572D4164643A20253032E9
:10031000783A253032783A253032783A25303278BA
:100320003A253032783A253032782029004D414341
:10033000004D4143004D4350636F6E666967000D89
:100340000A000A00256300436F6E666967206973BF
:10035000742025642062797465732067726F7373EB
:100360002C20256420627974652077657264656E3F
:100370002062656E75747A742E204F66667365749C
:100380002025640D0A0D0A004F4646005752495475
:10039000455F50524F544543540020496E6974697B
:1003A000616C6973696572740D0A00204572726F21
:1003B000720D0A00544852454144005348454C4C84
:1003C0000046696C6573797374656D004D4D432FFC
:1003D000534400444346373700312D5749524500B6
:1003E000414443004750494F004F70656E4D4350A4
:1003F000202E2E2E0D0A004C434400202825642078
:100400004465766963657329005457490050434930
:100410004E5400455854494E5400436F6E66696708
:10042000004C45445F636F726500434C4F434B0083
:100430005354444F55540055415254004F70656E0B
:100440004D4350202E2E2E0D0A0054454D5053453D
:100450004E534F525F25303264003C2F7461626C02
:10046000653E003C666F726D20616374696F6E3D1E
:100470002274656D70636F6E6669672E63676922AB
:100480003E3C74723E3C74643E53656E736F7220E2
:100490002564202825732043293C2F74643E3C7436
:1004A000643E3C696E707574206E616D653D2242DC
:1004B000555322747970653D227465787422766193
:1004C0006C75653D2225732273697A653D22382259
:1004D000206D61786C656E6774683D2238223E3C01
:1004E0002F74643E3C74643E3C696E707574206E7B
:1004F000616D653D224144445245535322747970E5
:10050000653D22746578742276616C75653D22259F
:10051000732273697A653D223233226D61786C658E
:100520006E6774683D223233223E3C2F74643E3C39
:1005300074643E3C696E707574206E616D653D2219
:100540004E414D4522747970653D22746578742260
:1005500076616C75653D2225732273697A653D224B
:100560003238226D61786C656E6774683D2232386E
:10057000223E3C2F74643E3C74643E3C696E707550
:100580007420747970653D227375626D697422768A
:10059000616C75653D222641756D6C3B6E646572BC
:1005A0006E226E616D653D2254454D5053454E534C
:1005B0004F525F25303264223E3C2F74643E3C74BF
:1005C000643E3C6120687265663D2274656D7063AF
:1005D0006F6E6669672E6367693F64656C3D25646D
:1005E00022207374796C653D22746578742D64657E
:1005F000636F726174696F6E3A6E6F6E65222074FC
:1006000069746C653D2244656C223E3C696E707570
:100610007420747970653D22627574746F6E222047
:1006200076616C75653D224C266F756D6C3B73630E
:1006300068656E2220636C6173733D226163746927
:100640006F6E42746E223E3C2F613E3C2F74643EBE
:100650003C2F74723E3C2F666F726D3E0025733BDB
:1006600025733B2573004255530041444452455382
:1006700053004E414D450064656C0064656C003C60
:100680007461626C6520626F726465723D22302213
:100690002063656C6C70616464696E673D2235220D
:1006A0002063656C6C73706163696E673D223022F4
:1006B0003E3C74723E3C74643E3C2F74643E3C7419
:1006C000643E4275733C2F74643E3C74643E4164E6
:1006D00072657373653C2F74643E3C74643E42657E
:1006E00073636872656962756E673C2F74643E3C23
:1006F00074643E3C2F74643E006E2F6100256325B8
:10070000642E2530326400554450004F4E45574901
:100710005245005457490074656D70636F6E666989
:10072000672E6367690054656D7073656E736F72D1
:1007300020746872656164003C68746D6C3E3C684E
:100740006561643E3C73637269707420747970658E
:100750003D22746578742F6A617661736372697083
:100760007422207372633D226A732F6A71756572F9
:10077000792E6D696E2E6A73223E3C2F7363726907
:1007800070743E3C73637269707420747970653D57
:1007900022746578742F6A6176617363726970740C
:1007A00022207372633D226A732F686967686368E9
:1007B000617274732E6A73223E3C2F736372697088
:1007C000743E3C73637269707420747970653D2265
:1007D000746578742F6A61766173637269707422CC
:1007E000207372633D226A732F657863616E766150
:1007F000732D636F6D707265737365642E6A7322F7
:100800003E3C2F7363726970743E3C73637269700F
:100810007420747970653D22746578742F6A6176EE
:1008200061736372697074223E2428646F63756D0E
:10083000656E74292E72656164792866756E6374BD
:10084000696F6E28297B7661722063686172743DDE
:100850006E657720486967686368617274732E43B8
:1008600068617274287B63686172743A7B72656E2A
:10087000646572546F3A27636F6E7461696E657256
:10088000272C64656661756C745365726965735471
:100890007970653A2773706C696E65272C6D61728B
:1008A00067696E3A5B35302C3138302C36302C3855
:1008B000305D7D2C7469746C653A7B746578743A2C
:1008C00020272573272C7374796C653A7B6D6172D0
:1008D00067696E3A27313070782031303070782077
:1008E000302030277D7D2C78417869733A7B74798C
:1008F00070653A276461746574696D65277D2C7035
:100900006C6F744F7074696F6E733A7B73706C693F
:100910006E653A7B6C696E6557696474683A322C0F
:100920006D61726B65723A7B656E61626C65643A8B
:1009300066616C73657D2C706F696E74496E746549
:100940007276616C3A3630303030302C706F696EB0
:100950007453746172743A446174652E555443281B
:1009600025642C25642C25642C302C302C30292C2B
:100970007374617465733A7B686F7665723A7B6DE8
:1009800061726B65723A7B656E61626C65643A7424
:100990007275652C73796D626F6C3A276369726347
:1009A0006C65272C7261646975733A332C6C696EBF
:1009B0006557696474683A317D7D7D7D7D2C794110
:1009C0007869733A7B7469746C653A7B7465787482
:1009D0003A272573277D7D2C746F6F6C7469703A8C
:1009E0007B666F726D61747465723A66756E63745E
:1009F000696F6E28297B72657475726E273C623E42
:100A0000272B20746869732E7365726965732E6E67
:100A1000616D65202B273C2F623E3C62723E272B86
:100A2000486967686368617274732E6461746546AF
:100A30006F726D617428272525652E20252562207B
:100A40002525592C202525483A25254D272C746825
:100A500069732E78292B273A20272B746869732E07
:100A6000792B272573273B327D7D2C6C6567656E5E
:100A7000643A7B6C61796F75743A27766572746934
:100A800063616C272C7374796C653A7B6C65667452
:100A90003A276175746F272C626F74746F6D3A27F3
:100AA0006175746F272C72696768743A27313070EA
:100AB00078272C746F703A20273130307078277D7A
:100AC0007D2C7365726965733A5B005D7D293B7DA2
:100AD000293B3C2F7363726970743E3C2F686561DB
:100AE000643E3C626F64793E3C6469762069643D93
:100AF00022636F6E7461696E657222207374796C03
:100B0000653D2277696474683A38303070783B68A4
:100B100065696768743A3430307078223E3C2F64DF
:100B200069763E3C2F626F64793E3C2F68746D6C31
:100B30003E0D0A0D0A000D0A00466F6C67656E6473
:100B4000652042656665686C652073696E64207611
:100B50006F7268616E64656E3A0D0A0D0A00686511
:100B60006C7000485454502F312E30203430330DE7
:100B70000A436F6E74656E742D547970653A2074F3
:100B80006578742F68746D6C0D0A4B6565702D4126
:100B90006C6976653A20636C6F73650D0A0D0A3CCB
:100BA00048544D4C3E3C424F44593E34303320462D
:100BB000696C65206E6F7420666F756E64213C2FC2
:100BC000424F44593E3C2F48544D4C3E0D0A0D0AAD
:100BD00000504F53540047455400687474706400CB
:100BE000485454502D53657276657220506F72745C
:100BF0002025642E0D0A00696E6465782E68746D78
:100C00006C003C2F424F44593E3C2F48544D4C3EC3
:100C10000D0A0D0A003C48544D4C3E3C48454144A9
:100C20003E3C2F484541443E3C424F44593E0048DB
:100C30005454502F312E302032303020446F6375A1
:100C40006D656E7420666F6C6C6F77730D0A436F01
:100C50006E74656E742D547970653A20746578747D
:100C60002F68746D6C0D0A436F6E6E656374696FE7
:100C70006E3A20636C6F73650D0A0D0A0048545478
:100C8000502F312E302032303020446F63756D6527
:100C90006E7420666F6C6C6F77730D0A436F6E74A1
:100CA000656E742D4C656E6774683A20256C640D12
:100CB0000A436F6E74656E742D547970653A202501
:100CC0007325730D0A43616368652D436F6E7472FB
:100CD0006F6C3A206D61782D6167653D3336303039
:100CE0000D0A436F6E6E656374696F6E3A20636CB4
:100CF0006F73650D0A0D0A00746578742F006874AF
:100D00006D0068746D6C003E200051756974696EE9
:100D1000670D0A007175697400556E642C206C6F44
:100D200073206765687427732E2E2E2121212028B9
:100D30002268656C70222068696C6674203A2D29DF
:100D4000290D0A3E200074656C6E65740054656C54
:100D50006E65742D53657276657220506F727420C3
:100D600025642E0D0A0043524F4E5F454E54525992
:100D70005F253032640025643A206E696368742010
:100D800062656C6567740D0A0025643A202564204D
:100D900025642025730D0A0063726F6E004B656930
:100DA0006E6520496E666F732E00446174653A204B
:100DB00025752E25752E25303275202000256C6472
:100DC0002C2530336C6420257300496D70756C736D
:100DD0007A6165686C65723A0025730055707469B4
:100DE0006D653A20256C64730054656D7020256430
:100DF0003A2025734300202020202020202020207E
:100E00002020202020200D005A6569743A202530CA
:100E100032643A25303264202020200D0A004C43F1
:100E2000442D496E666F00666F6F2E6367690025FB
:100E3000732F257325730049502F4D41432F545470
:100E40004C0D0A0061727000696E20256C642050A0
:100E500061636B6574656E203B2044752062697325
:100E600074206465722025642E2042657375636862
:100E700065722061756620536F636B65742025640D
:100E80002E3C2F424F44593E3C2F48544D4C3E0D72
:100E90000A0D0A0020256C642E2530336C6420472F
:100EA0004279746573200020256C642E2530336CE4
:100EB00064204D4279746573200020256C64206B9A
:100EC0004279746573200020256C64204279746532
:100ED0007320002C2045746865726E65743A002595
:100EE0006C642073656B00256C64206D696E200056
:100EF000256C64207374642000256C642074616721
:100F0000652000256C642074616720003C48544DC6
:100F10004C3E3C484541443E3C6D657461206874DC
:100F200074702D65717569763D22726566726573A0
:100F3000682220636F6E74656E743D223630303BDC
:100F400020223E3C5449544C453E53747265616DB9
:100F5000696E673C2F5449544C453E3C2F484541EF
:100F6000443E3C424F4459206267636F6C6F723D50
:100F700022233232384232322220746578743D2284
:100F800023464646464646223E5A6569743A20251F
:100F90003032643A253032643A253032642E2530BE
:100FA000326420282025752F25752F253034752093
:100FB000292C20557074696D653A200050485354AF
:100FC000415432207C203078253034580D0A0050AE
:100FD000485354415431207C203078253034580D0A
:100FE0000A005265762E494420207C20202030784B
:100FF000253032580D0A002D2D2D2D2D2D2D2D2B68
:101000002D2D2D2D2D2D2D2D0D0A005265672E20F5
:101010002020207C20576572740D0A00454E433213
:10102000384A36303A0D0A005443502D5458204562
:1010300072726F72733A202564205443502D5258B7
:10104000204572726F72733A2025642028756E7382
:101050006F727465642025642C206F6C64736571F5
:10106000202564290D0A0D0A0045746865726E65B5
:10107000743A20256C6420427974657320696E206F
:10108000256C64205061636B6574656E204C6F63E2
:101090006B4572726F727320256C640D0A00737455
:1010A0006174732E636769007374617473005265B1
:1010B000736574007265736574007265736574009E
:1010C0007265736574003C666F726D20616374694C
:1010D0006F6E3D2272657365742E63676922206DA1
:1010E0006574686F643D226765742220616363657F
:1010F00070742D636861727365743D2249534F2D7E
:10110000383835392D31223E3C703E3C696E707561
:101110007420747970653D227375626D6974222044
:101120006E616D653D227265736574222076616C17
:1011300075653D227265736574223E3C2F703E3C9E
:101140002F666F726D3E0072657365742E636769FA
:1011500000726573657400646E73203C686F73740D
:101160006E616D653E0D0A004950207A7520257329
:10117000203D2025730D0A00646E73003C2F7461BE
:10118000626C653E003C74723E3C746420616C6924
:10119000676E3D227269676874223E414443202590
:1011A00064203D3C2F74643E3C746420616C69672C
:1011B0006E3D227269676874223E2025642E2530B8
:1011C0003364563C2F74643E3C2F74723E0D003CD9
:1011D0007461626C6520626F726465723D223022B8
:1011E0002063656C6C70616464696E673D223522B2
:1011F0002063656C6C73706163696E673D22302299
:101200003E003C48544D4C3E3C484541443E3C6DBC
:1012100065746120687474702D65717569763D22FE
:10122000726566726573682220636F6E74656E7492
:101230003D2233303B20223E3C5449544C453E41F4
:1012400044433C2F5449544C453E3C2F484541446F
:101250003E3C424F44593E00616463203C676574E4
:101260003E203C302E2E373E0D0A004572726F72C2
:101270002C20256420697374206B65696E2067C318
:10128000BC6C746572204144432D45696E67616E84
:10129000670D0A004144432028256429203D20256C
:1012A000640D0A006765740061696F2E63676900E9
:1012B000616463003C74723E3C74643E3C2F746411
:1012C0003E3C74643E3C696E707574207479706540
:1012D0003D227375626D697422206E616D653D22D9
:1012E000535542223E3C2F74643E3C2F74723E3C68
:1012F0002F7461626C653E3C2F666F726D3E003EDE
:101300003C2F74643E3C2F74723E00636865636BCF
:101310006564003C74643E3C696E70757420747939
:1013200070653D22636865636B626F7822206E6131
:101330006D653D224750494F25642220003C747260
:101340003E3C746420616C69676E3D227269676817
:1013500074223E506F727425632564203D3C2F74C7
:10136000643E003C666F726D20616374696F6E3D10
:101370002264696F5F6F75742E636769223E3C74E7
:1013800061626C6520626F726465723D223022205A
:1013900063656C6C70616464696E673D2235222000
:1013A00063656C6C73706163696E673D2230223EC9
:1013B000004750494F2564003C2F7461626C653EC4
:1013C0003C2F666F726D3E003C2F74643E3C2F7460
:1013D000723E003C74643E4F66663C2F74643E006F
:1013E0003C74643E4F6E3C2F74643E003C74723E0D
:1013F0003C746420616C69676E3D22726967687431
:10140000223E506F727425632564203D3C2F746426
:101410003E003C666F726D20616374696F6E3D22A1
:1014200064696F5F6F75742E636769223E3C7461F7
:10143000626C6520626F726465723D2230222063A7
:10144000656C6C70616464696E673D22352220634F
:10145000656C6C73706163696E673D2230223E007B
:101460004750494F2028256429203D2025640D0A36
:10147000006770696F5F6F7574203C6765747C737B
:1014800065747C746F67676C657C636C6561723EC4
:10149000203C302E2E25643E0D0A00636C6561727F
:1014A00000746F67676C650073657400676574002E
:1014B0004572726F722C202564206E6F74207661E5
:1014C0006C69642E0D0A0064696F5F6F75742E631A
:1014D00067690064696F5F696E2E63676900677092
:1014E000696F5F6F75740044484350004950004D68
:1014F00041534B004741544500444E53004D414336
:101500000045696E7374656C6C756E67656E2075E9
:10151000656265726E6F6D6D656E210D0A003C74BB
:10152000723E3C746420616C69676E3D227269672B
:101530006874223E48617264776172652D4D414343
:101540003C2F74643E3C74643E3C696E707574203C
:101550006E616D653D224D41432220747970653D79
:101560002274657874222073697A653D22313722AE
:101570002076616C75653D22257322206D61786C43
:10158000656E6774683D223137223E3C2F74643E9D
:101590003C2F74723E3C74723E3C74643E3C2F742B
:1015A000643E3C74643E3C696E707574207479705E
:1015B000653D227375626D6974222076616C756574
:1015C0003D222045696E7374656C6C756E672026CC
:1015D00055756D6C3B6265726E65686D656E202237
:1015E0003E3C2F74643E3C2F74723E3C2F7461620B
:1015F0006C653E3C2F666F726D3E004D4143003C72
:1016000074723E3C746420616C69676E3D2272693D
:10161000676874223E444E532D5365727665723C62
:101620002F74643E3C74643E3C696E707574206E29
:10163000616D653D22444E532220747970653D22D0
:1016400074657874222073697A653D2231352220D1
:1016500076616C75653D22257322206D61786C651D
:101660006E6774683D223135223E3C2F74643E3CE7
:101670002F74723E00444E53003C74723E3C7464BE
:1016800020616C69676E3D227269676874223E470B
:101690006174657761793C2F74643E3C74643E3CB0
:1016A000696E707574206E616D653D2247415445C9
:1016B0002220747970653D227465787422207369E4
:1016C0007A653D223135222076616C75653D222593
:1016D0007322206D61786C656E6774683D223135C8
:1016E000223E3C2F74643E3C2F74723E00474154AE
:1016F00045003C74723E3C746420616C69676E3DC9
:10170000227269676874223E4E65747A7765726BDF
:101710006D61736B653C2F74643E3C74643E3C6940
:101720006E707574206E616D653D224D41534B2284
:1017300020747970653D2274657874222073697A0B
:10174000653D223135222076616C75653D22257319
:1017500022206D61786C656E6774683D2231352298
:101760003E3C2F74643E3C2F74723E004D41534BFF
:10177000003C74723E3C746420616C69676E3D226B
:101780007269676874223E49502D416472657373B3
:10179000653C2F74643E3C74643E3C696E707574A5
:1017A000206E616D653D2249502220747970653D3F
:1017B0002274657874222073697A653D223135225E
:1017C0002076616C75653D22257322206D61786CF1
:1017D000656E6774683D223135223E3C2F74643E4D
:1017E0003C2F74723E004950003E3C2F74643E3CD6
:1017F0002F74723E00636865636B6564006F6E00F2
:101800003C74723E3C746420616C69676E3D227268
:1018100069676874223E4448435020616B7469765E
:10182000696572656E3C2F74643E3C74643E3C692D
:101830006E70757420747970653D22636865636BA2
:10184000626F7822206E616D653D224448435022CC
:101850002076616C75653D226F6E222000444843FE
:1018600050003C666F726D20616374696F6E3D223B
:101870006E6574776F726B2E636769223E3C74618C
:10188000626C6520626F726465723D223022206353
:10189000656C6C70616464696E673D2235222063FB
:1018A000656C6C73706163696E673D2230223E0027
:1018B000636F6E666967003C2F7072653E0D0A00AB
:1018C0007374617473006966636F6E666967003C68
:1018D0007072653E0D0A000D0A48572D4164723A38
:1018E00020253032783A253032783A253032783A2D
:1018F000253032783A253032783A253032780D0A60
:101900000D0A00444E533A25730D0A004761746571
:101910007761793A25730D0A004E65746D61736BBA
:101920003A25730D0A0049503A25730D0A006E6579
:1019300074776F726B2E636769006966636F6E669A
:101940006967004E5450004E54505345525645520C
:10195000005554435A4F4E450045696E7374656C8B
:101960006C756E67656E2075656265726E6F6D6D04
:10197000656E210D0A003C74723E3C746420616CFB
:1019800069676E3D227269676874223E534E5450F7
:101990002D5365727665723C2F74643E3C74643ED0
:1019A0003C696E707574206E616D653D224E5450B9
:1019B0005345525645522220747970653D22746514
:1019C0007874222073697A653D223235222076614F
:1019D0006C75653D22257322206D61786C656E679C
:1019E00074683D223235223E3C2F74643E3C2F7495
:1019F000723E3C74723E3C746420616C69676E3D5B
:101A0000227269676874223E5A6569747A6F6E65DE
:101A10003C2F74643E3C74643E3C696E7075742067
:101A20006E616D653D225554435A4F4E45222074D8
:101A30007970653D2274657874222073697A653DFA
:101A40002233222076616C75653D22257322206D3C
:101A500061786C656E6774683D2233223E3C2F745A
:101A6000643E3C2F74723E3C74723E3C74643E3C57
:101A70002F74643E3C74643E3C696E7075742074CF
:101A80007970653D227375626D6974222076616C90
:101A900075653D222045696E7374656C6C756E6763
:101AA000202655756D6C3B6265726E65686D656E5E
:101AB00020223E3C2F74643E3C2F74723E3C2F74B7
:101AC00061626C653E3C2F666F726D3E0030007443
:101AD000696D652E66752D6265726C696E2E646522
:101AE000003E3C2F74643E3C2F74723E0063686578
:101AF000636B6564006F6E003C666F726D2061639E
:101B000074696F6E3D226E74702E636769223E0D9C
:101B10003C7461626C6520626F726465723D223054
:101B2000222063656C6C70616464696E673D223568
:101B3000222063656C6C73706163696E673D22304F
:101B4000223E3C74723E3C746420616C69676E3D59
:101B5000227269676874223E534E545020616B7440
:101B60006976696572656E3C2F74643E3C74643EB0
:101B70003C696E70757420747970653D2263686588
:101B8000636B626F7822206E616D653D224E54500A
:101B9000222076616C75653D226F6E2220006E7486
:101BA00070203C6E74707365727665723E0D0A002B
:101BB0004665686C65720D0A004E657565205A654C
:101BC00069743A20253032643A253032643A25303F
:101BD00032640D0A00486F6C65205A65697420767E
:101BE0006F6E2025730D0A004665686C65720D0ADC
:101BF000006E74702E636769006E74700025730048
:101C000074656D700064656C0064656C0045696E98
:101C10007374656C6C756E67656E20756562657250
:101C20006E6F6D6D656E210D0A00256420256420A0
:101C30002225732200434D44004D4D004848004387
:101C40004D44003C666F726D20616374696F6E3D38
:101C50002263726F6E2E636769223E3C7461626C10
:101C60006520626F726465723D2230222063656C6C
:101C70006C70616464696E673D2235222063656C17
:101C80006C73706163696E673D2230223E3C7472F2
:101C90003E3C746420616C69676E3D2272696768BE
:101CA00074223E5374756E64653C2F74643E3C74BC
:101CB000643E3C696E707574206E616D653D2248AE
:101CC000482220747970653D2274657874222073EF
:101CD000697A653D2233222076616C75653D22303C
:101CE000226D61786C656E6774683D2233223E3CDC
:101CF0002F74643E3C2F74723E3C74723E3C74649C
:101D000020616C69676E3D227269676874223E4D7E
:101D1000696E7574653C2F74643E3C74643E3C6926
:101D20006E707574206E616D653D224D4D2220747C
:101D30007970653D2274657874222073697A653DF7
:101D40002233222076616C75653D223022206D6140
:101D5000786C656E6774683D2233223E3C2F746454
:101D60003E3C2F74723E3C74723E3C746420616C45
:101D700069676E3D227269676874223E436F6D6DBC
:101D8000616E643C2F74643E3C74643E3C696E70CA
:101D90007574206E616D653D22434D442220747937
:101DA00070653D2274657874222073697A653D22DE
:101DB000333022206D61786C656E6774683D223324
:101DC00030223E3C2F74643E3C2F74723E3C747251
:101DD0003E3C74643E3C2F74643E3C74643E3C69FB
:101DE0006E70757420747970653D227375626D69CB
:101DF00074222076616C75653D222045696E74728F
:101E00006167207369636865726E20223E3C2F749F
:101E1000643E3C2F74723E3C2F7461626C653E3CA4
:101E20002F666F726D3E0D006164646E6577003CD5
:101E300074723E3C746420616C69676E3D226C650F
:101E40006674223E3C6120687265663D2263726F53
:101E50006E2E6367693F6164646E657722207374D8
:101E6000796C653D22746578742D6465636F726169
:101E700074696F6E3A6E6F6E6522207469746C655A
:101E80003D22416464223E3C696E70757420747911
:101E900070653D22627574746F6E222076616C7578
:101EA000653D22616464206E65772063726F6E22E7
:101EB00020636C6173733D22616374696F6E427459
:101EC0006E223E3C2F613E3C2F74643E3C2F747268
:101ED0003E3C2F7461626C653E0D003C74723E3C6A
:101EE000746420616C69676E3D226C656674223E85
:101EF00025733C2F74643E3C746420616C69676E8A
:101F00003D226C656674223E3C6120687265663DC8
:101F10002263726F6E2E6367693F64656C3D256452
:101F200022207374796C653D22746578742D646524
:101F3000636F726174696F6E3A6E6F6E65222074A2
:101F400069746C653D2244656C223E3C696E707517
:101F50007420747970653D22627574746F6E2220EE
:101F600076616C75653D2264656C2220636C6173DB
:101F7000733D22616374696F6E42746E223E3C2F22
:101F8000613E3C2F74643E3C2F74723E003C746191
:101F9000626C6520626F726465723D22302220633C
:101FA000656C6C70616464696E673D2235222063E4
:101FB000656C6C73706163696E673D2230223E0010
:101FC00063726F6E2E636769003C2F7072653E000E
:101FD0003C7072653E0065656D656D203C70726F8A
:101FE000746563743E7C3C756E70726F7465637467
:101FF0003E203C616464205B6E616D652076616C9F
:102000005D3E203C64656C205B6E616D655D3E20CD
:102010003C7072696E743E203C636C65616E3E0D6F
:102020000A00636C65616E007072696E74006465AD
:102030006C0061646400756E70726F7465637465C2
:10204000740D0A0057524954455F50524F5445434E
:1020500054004F464600756E70726F74656374006D
:1020600057524954455F50524F54454354004F4EC8
:102070000070726F746563740065656D656D2E63C5
:1020800067690065656D656D003C2F7072653E0087
:102090004C4D37352053656E736F722067656675DA
:1020A0006E64656E20617566204164726573736548
:1020B0003A203078253032782C2054656D70657266
:1020C0006174757220257320430D0A000D0A536355
:1020D000616E6E65206E616368204C4D373520540B
:1020E000656D7065726174757273656E736F72651C
:1020F0006E3A0D0A0020307825303278002C003CF2
:102100007072653E5363616E6E65206E6163682018
:1021100054574920536C617665733A0D0A536C61CC
:1021200076657320676566756E64656E20616E20E6
:10213000416472657373653A007477692E636769E9
:10214000003A2025732043290D0A002530325820FB
:102150002800253032583A0049443A20004275732D
:10216000204572726F720D0A004E6F2053656E73B8
:102170006F7220666F756E640D0A003C7072653E6A
:10218000466F6C67656E646520476572616574654E
:102190002077757264656E20676566756E64656E1E
:1021A0003A0D0A006F6E65776972652E6367690084
:1021B000494D50554C535F5052455343414C455245
:1021C00000494D50554C535F434F554E54455200B6
:1021D000494D50554C535F4155544F53415645005E
:1021E000494D50554C535F554E4954004155544F3D
:1021F0005341564500554E495400505245534341B2
:102200004C455200696D70756C732E6C6F6700568B
:1022100065726C617566005665726272617563689D
:102220002028257329005D7D2C00256C642E253027
:10223000336C6420006E756C6C20002C007B206E6B
:10224000616D653A20227465737422202C64617478
:10225000613A205B0045696E7374656C6C756E67DE
:10226000656E2075656265726E6F6D6D656E2100BD
:102270003C666F726D20616374696F6E3D22696D9B
:1022800070756C732E636769223E3C7461626C6585
:1022900020626F726465723D2230222063656C6C2F
:1022A00070616464696E673D2235222063656C6CE1
:1022B00073706163696E673D2230223E3C74723EEA
:1022C0003C746420616C69676E3D22726967687452
:1022D000223E4175746F5361766520616B74697637
:1022E000696572656E3C2F74643E3C74643E3C6963
:1022F0006E70757420747970653D22636865636BD8
:10230000626F7822206E616D653D224155544F53B6
:10231000415645222076616C75653D226F6E222004
:102320002573203E3C2F74643E3C74723E3C7464C2
:1023300020616C69676E3D227269676874223E5045
:1023400072655363616C65723C2F74643E3C7464C7
:102350003E3C696E707574206E616D653D22505211
:10236000455343414C45522220747970653D227497
:10237000657874222073697A653D22313022207697
:10238000616C75653D22256C6422206D61786C65F9
:102390006E6774683D223130223E3C2F74643E3CAF
:1023A0002F74723E3C74723E3C746420616C6967A9
:1023B0006E3D227269676874223E45696E68656980
:1023C000743C2F74643E3C74643E3C696E7075745A
:1023D000206E616D653D22554E49542220747970FE
:1023E000653D2274657874222073697A653D2238D0
:1023F000222076616C75653D22257322206D6178FF
:102400006C656E6774683D2238223E3C2F74643ED2
:102410003C2F74723E3C74723E3C74643E3C2F749C
:10242000643E3C74643E3C696E70757420747970CF
:10243000653D227375626D6974222076616C7565E5
:102440003D222045696E7374656C6C756E6720263D
:1024500055756D6C3B6265726E65686D656E2022A8
:102460003E3C2F74643E3C2F74723E3C2F7461627C
:102470006C653E3C2F666F726D3E00636865636BF2
:102480006564006F6E00636F6E666967005A616510
:10249000686C65723A20256C642C2530336C64209E
:1024A00025732028256C6420496D70756C7365292F
:1024B0003C42523E3C42523E3C6120687265663D61
:1024C00022696D70756C732E6367693F636F6E660A
:1024D0006967223E45696E67657374656C6C756EDD
:1024E00067656E3C2F613E006F6E00496D70756CC4
:1024F0007365204C6F6767657200696D70756C73EA
:102500006C6F676765722E63676900696D70756CC3
:10251000732E6367690073656E736F720074656D07
:10252000706C6F675F253032642E6E646200546594
:102530006D706572617475727665726C6175660036
:1025400054656D7065726174757220282573290059
:10255000266465673B43005D7D2C00257320006E7B
:10256000756C6C20002C007B6E616D653A272573BD
:10257000272C646174613A205B0074656D706C6F28
:10258000676765722E6367690074656D702E6A7384
:102590006F6E0054656D70204C6F67676572000048
:1025A00014BE88E10FB6F89480936000109260002A
:1025B0000FBE11241FBECFEFD0E1DEBFCDBF11E0B3
:1025C000A0E0B1E0E0E9F6EF02C005900D92AE3870
:1025D000B107D9F718E0AEE8B1E001C01D92AB3BFE
:1025E000B107E1F704D00C94477B0C9400000E94E3
:1025F000EF460E9479620E9480620E947F48FDCF70
:10260000109269000895AC01039754F42DB381E052
:1026100090E002C0880F991F4A95E2F7282B2DBB46
:102620000895DC01833091051CF08EEF90E0089551
:10263000643071051CF08FEF90E0089520916900DF
:10264000FC01EE0FFF1F83E090E00E2E02C0880F0A
:10265000991F0A94E2F78095822380936900809104
:1026600069000E2E02C0660F771F0A94E2F7862BD0
:1026700080936900E25FFA4F51834083CD01C3DF4D
:1026800080E090E00895AC0103975CF42DB381E005
:1026900090E002C0880F991F4A95E2F78095822347
:1026A0008DBB08951F920F920FB60F9211242F9396
:1026B0003F934F935F936F937F938F939F93AF93CA
:1026C000BF93EF93FF93E0910E05F0910F050995ED
:1026D000FF91EF91BF91AF919F918F917F916F91FA
:1026E0005F914F913F912F910F900FBE0F901F90D0
:1026F00018951F920F920FB60F9211242F933F93AC
:102700004F935F936F937F938F939F93AF93BF93F9
:10271000EF93FF93E0911005F09111050995FF915A
:10272000EF91BF91AF919F918F917F916F915F9149
:102730004F913F912F910F900FBE0F901F901895C2
:102740001F920F920FB60F9211242F933F934F9326
:102750005F936F937F938F939F93AF93BF93EF9309
:10276000FF93E0911205F09113050995FF91EF9108
:10277000BF91AF919F918F917F916F915F914F9199
:102780003F912F910F900FBE0F901F901895FC0155
:10279000EE0FFF1FEE0FFF1FE80FF91FEC5EFA4F61
:1027A00086E084830895613019F4845E90E0089592
:1027B000673008F0615060FF03C08EE190E008953B
:1027C0008FE190E00895A0E0B0E0E9EEF3E10C9431
:1027D000ED75EC018E849F84A888B988EE84FF840F
:1027E00008891989698570E080E090E020E13EE089
:1027F00040E050E00E945875E60EF71E081F191FB2
:10280000EE86FF86088B198B8CE697E098878F837E
:102810006E857F858889998920E831E541E050E01F
:102820000E94AA757B018C016E857F8588899989B4
:1028300020E831E541E050E00E94AA756901C80135
:10284000B7012CE330E040E050E00E94AA756983B4
:10285000C801B70120E13EE040E050E00E94AA75C7
:102860002CE330E040E050E00E94AA752A83C801C2
:10287000B70120E13EE040E050E00E94AA752B83C2
:10288000C601049667E070E00E9483758C8322C0C5
:102890008F81988583709070892B99F48F819885AA
:1028A00064E670E00E948375892B41F48F819885DE
:1028B00060E971E00E948375892B19F48EE691E03E
:1028C00002C08DE691E0C81AD90A8F8198850196D9
:1028D00098878F838F81988583709070892B99F466
:1028E0008F81988564E670E00E948375892B41F49E
:1028F0008F81988560E971E00E948375892B19F4B6
:102900008EE691E002C08DE691E0C816D90608F087
:10291000BFCF1E8229C04E818F81988583709070B1
:10292000892B19F080E090E018C08F81988564E6CB
:1029300070E00E948375892B19F081E090E00DC052
:102940008F81988520E030E060E971E00E94837516
:10295000892B11F421E030E0C901642F24DFC81A6B
:10296000D1088E818F5F8E834E818F819885837091
:102970009070892B19F080E090E018C08F819885C5
:1029800064E670E00E948375892B19F081E090E085
:102990000DC08F81988520E030E060E971E00E94F1
:1029A0008375892B11F421E030E0C901642FFBDE2F
:1029B00090E0C816D90608F0AECF8E818F5F8E8367
:1029C0008C2D8F5F8D838E81833010F430E007C0B3
:1029D0008E8130E08B3008F031E081E038278D8146
:1029E0002C8190E0821B910949975CF08C818823AF
:1029F00019F48B81823028F08E818A3009F443C02B
:102A000004C08E81833009F43EC03323E1F18B8111
:102A10008F5F8B838B818831B1F51B828C818F5FB7
:102A20008C838C81873009F41C82ED804E818F81EC
:102A3000988583709070892B19F080E090E018C021
:102A40008F81988564E670E00E948375892B19F068
:102A500081E090E00DC08F81988520E030E060E952
:102A600071E00E948375892B11F421E030E0C901E7
:102A7000642F99DEE81621F41D828E818F5F8E838C
:102A80008D818F5F8D838E869F86A88AB98AECE0C0
:102A9000CDB7DEB70C9409761F93CF93DF93809167
:102AA0005C058F5F80935C0580915C05843611F036
:102AB00011E053C010925C0580915D058F5F80939B
:102AC0005D058091660590916705A0916805B091BC
:102AD00069050196A11DB11D809366059093670558
:102AE000A0936805B093690580916A0590916B0584
:102AF000A0916C05B0916D050196A11DB11D80934B
:102B00006A0590936B05A0936C05B0936D05809159
:102B10005D058C3311F012E020C010925D058091AC
:102B20005E058F5F80935E0580915E058C3311F0AA
:102B300013E013C010925E0580915F058F5F809354
:102B40005F058CE595E03FDE80915F05883111F0EF
:102B500014E003C010925F0515E0C0E0D0E0FE0174
:102B6000EE0FFF1FEE0FFF1FE45CFA4F8281181774
:102B700050F0123018F081E0838305C01382019079
:102B8000F081E02D09952196C830D10541F720E06C
:102B900030E0F901EE0FFF1FEE0FFF1FE45CFA4F6C
:102BA0008381813041F413820190F081E02D0995F9
:102BB00020E030E006C02F5F3F4F2830310549F755
:102BC000F7CFF901EE0FFF1FEE0FFF1FE20FF31F0C
:102BD000EC5EFA4F8481181798F080819181A28170
:102BE000B3810097A105B10559F080819181A2813F
:102BF000B3810197A109B10980839183A283B38333
:102C00002F5F3F4F28303105E1F6DF91CF911F91C3
:102C10000895A0E0B0E0EFE0F6E10C94EF75EC0170
:102C20001E861F86188A198A2CE637E02AC0EE8491
:102C3000FF8408891989C90183709070892B99F4E0
:102C4000C90164E670E00E948375892B39F4C901DB
:102C500060E971E00E948375892B29F480E095E892
:102C6000A2EEB1E004C080E893E3A1EEB1E08E0DE6
:102C70009F1DA01FB11F8E879F87A88BB98B2F5FC9
:102C80003F4F8F8198852817390788F2AA24A3948B
:102C90003BC0EE84FF84088919898F8198858370F1
:102CA0009070892B19F080E090E018C08F81988592
:102CB00064E670E00E948375892B19F081E090E052
:102CC0000DC08F81988520E030E060E971E00E94BE
:102CD0008375892B11F421E030E0C9016A2D63DD91
:102CE00090E0A0E0B0E0BC01CD0120E831E541E09A
:102CF00050E00E945875E60EF71E081F191FEE8659
:102D0000FF86088B198BA3948E81A81610F2EE848F
:102D1000FF84088919896D8170E0615070408827AF
:102D200077FD8095982F20E831E541E050E00E9442
:102D30005875E60EF71E081F191FEE86FF86088BD2
:102D4000198BEE84FF840889198929816B81AA80F7
:102D5000E20EF11C011D111D70E080E090E020E109
:102D60003EE040E050E00E945875E60EF71E081F56
:102D7000191FBB24CC24DD24C601B5012CE330E0AF
:102D800040E050E00E945875E60EF71E081F191F1C
:102D9000EE86FF86088B198BEE84FF8408891989DB
:102DA000698570E080E090E020E13EE040E050E0A6
:102DB0000E945875E61AF70A080B190BEE86FF8673
:102DC000088B198BEAE0CDB7DEB70C940B760F9326
:102DD0001F938C013BD142E150E0B8018CE595E0B6
:102DE0000E949D7739D180E090E01F910F91089566
:102DF0000F931F938C012AD142E150E06CE575E0FE
:102E0000C8010E949D7728D180E090E01F910F912A
:102E10000895EF92FF920F931F938C0117D1F80141
:102E2000EE0FFF1FEE0FFF1FE00FF11FEC5EFA4FDA
:102E3000E080F180028113810FD1C7011F910F91B2
:102E4000FF90EF900895BF92CF92DF92EF92FF92A2
:102E50000F931F936C017B01B42EF8D000E010E0BB
:102E6000F601EE0FFF1FEE0FFF1FEC0DFD1DEC5ED8
:102E7000FA4FE082F18202831383B482EDD01F9176
:102E80000F91FF90EF90DF90CF90BF900895CF9378
:102E9000DF93DCD0C0E0D0E0FE01EE0FFF1FEE0FAD
:102EA000FF1FEC0FFD1FEC5EFA4F8481863031F47A
:102EB0001082118212821382CFD007C02196C830AF
:102EC000D10551F7C9D0CFEFDFEFCE01DF91CF9120
:102ED00008950F931F93CF93DF938C01D8DFC82FF2
:102EE000D0E0C8016AE070E00E94837541E0CE0145
:102EF000AADFCE018EDF892BE1F7CE0148DCDF911E
:102F0000CF911F910F9108951F93CF93DF93EC0101
:102F1000162F9CD020E030E0F901EE0FFF1FEE0FDE
:102F2000FF1FE45CFA4F808191818C179D07A9F007
:102F30002F5F3F4F2830310579F720E030E0F9016D
:102F4000EE0FFF1FEE0FFF1FE45CFA4F80819181AF
:102F5000892B39F4D183C08312837ED080E090E046
:102F600008C02F5F3F4F2830310549F775D08FEFEC
:102F700090E0DF91CF911F91089520E030E0F901BA
:102F8000EE0FFF1FEE0FFF1FE45CFA4F118210825D
:102F900086E082832F5F3F4F2830310581F720E0A4
:102FA00030E0F901EE0FFF1FEE0FFF1FE20FF31FDE
:102FB000EC5EFA4F108211821282138286E08483C3
:102FC0002F5F3F4F2830310561F710926605109250
:102FD0006705109268051092690510926A051092B3
:102FE0006B0510926C0510926D05109265058CE5CD
:102FF00095E0E9DB60E070E084E690E003D08CE4EB
:1030000095E159C00F931F938B0110926F05109299
:103010006E052AE0209381009C0183E0220F331F7C
:103020008A95E1F740E050E060E074E284EF90E0E0
:103030000E94AA75201B310B3093890020938800D1
:1030400082E080936F001F910F910895EFE6F0E00A
:1030500080818D7F80830895EFE6F0E0808182603B
:10306000808308951F920F920FB60F9211242F9311
:103070003F934F935F936F937F938F939F93AF9300
:10308000BF93EF93FF93E0916E05F0916F0530973A
:1030900009F00995FF91EF91BF91AF919F918F91A9
:1030A0007F916F915F914F913F912F910F900FBE44
:1030B0000F901F90189520916E0530916F0528177D
:1030C000390719F481E090E00895232B19F080E08E
:1030D00090E0089590936F0580936E0581E090E0F5
:1030E0000895FC0183E0EE0FFF1F8A95E1F7E65A91
:1030F000FE4F0190F081E02D09950895FC0193E0C9
:10310000EE0FFF1F9A95E1F7E65AFE4F0280F3811A
:10311000E02D862F099590E008959B01FC0173E056
:10312000EE0FFF1F7A95E1F7E65AFE4F0680F78112
:10313000E02DBA01C90109950895FC0133E0880F1B
:10314000991F3A95E1F7EE0FFF1FE80FF91FE659B7
:10315000FE4F0190F081E02D09950895FC01862F26
:103160009F0153E0220F331F5A95E1F7EE0FFF1F27
:10317000E20FF31FE659FE4F0280F381E02D09951F
:103180000895FC0173E0880F991F7A95E1F7EE0F1F
:10319000FF1FE80FF91FE659FE4F0480F581E02D6F
:1031A000099590E00895FC01B3E0880F991FBA9546
:1031B000E1F7EE0FFF1FE80FF91FE659FE4F0680FB
:1031C000F781E02D099508951F920F920FB60F9287
:1031D00011248F93EF93FF93E1ECF0E080818F7BDC
:1031E000808310928E01FF91EF918F910F900FBE0F
:1031F0000F901F9018951F931FB7F8948091720538
:10320000909173050E94AC451FBF1F9108951F93B5
:103210001FB7F89480917205909173050E94AC4598
:10322000892B11F480E006C080917205909173059E
:103230000E9400461FBF90E01F9108951F920F92B9
:103240000FB60F9211242F933F934F935F936F9379
:103250007F938F939F93AF93BF93EF93FF9380914F
:103260007005909171050E94AC45892B49F08091C1
:103270007005909171050E9400468093C6000AC0B7
:103280008091C10080648093C1008091C1008F7DD6
:103290008093C100FF91EF91BF91AF919F918F916A
:1032A0007F916F915F914F913F912F910F900FBE42
:1032B0000F901F9018950F931F93182F0FB7F89426
:1032C00080917005909171050E94AC45892B31F574
:1032D00080918E01813091F4612F809170059091E1
:1032E00071050E94C3458091C1008F7B8093C1000E
:1032F0008091C10080628093C10022C01093C600FB
:103300008091C10080648093C1008091C1008F7D55
:103310008093C10081E080938E0112C0F894809167
:103320007005909171050E94AC45409714F00FBF55
:10333000F5CF612F80917005909171050E94C34572
:103340000FBF1F910F9108951F920F920FB60F920A
:1033500011241F932F933F934F935F936F937F930A
:103360008F939F93AF93BF93EF93FF931091C600FA
:1033700080917205909173050E94AC4540973CF492
:10338000612F80917205909173050E94C345FF9152
:10339000EF91BF91AF919F918F917F916F915F91CD
:1033A0004F913F912F911F910F900FBE0F901F9043
:1033B000189560E170E084E795E00E948145909364
:1033C00073058093720560E170E084E895E00E94E7
:1033D0008145909371058093700510928E01109233
:1033E000C50087E68093C40088E98093C10086E029
:1033F0008093C200089584E880937A0080E48093EB
:103400007C0080917A00806480937A0080917A00B9
:1034100086FDFCCF089590917C00987F90937C006E
:1034200090917C008770892B80937C0080917A003A
:10343000806480937A0080917A0086FDFCCF809131
:103440007800909179000895AF92BF92CF92DF9269
:10345000EF92FF920F931F937B010027F7FC0095DB
:10346000102F9C01442737FD4095542FC801B70108
:103470000E94587528EE33E040E050E00E94CC7581
:1034800079018A01CA01B90120E430E040E050E04E
:103490000E94CC7557016801A21AB30AC40AD50A62
:1034A000C801B70120E830E040E050E00E94CC7550
:1034B000A21AB30AC40AD50AC5011F910F91FF9041
:1034C000EF90DF90CF90BF90AF900895362F377078
:1034D000669566956695613029F1613038F0623005
:1034E00009F43CC0633009F454C06DC0813059F414
:1034F00021B181E090E002C0880F991F3A95E2F770
:10350000282B21B960C0823009F05DC021B181E073
:1035100090E002C0880F991F3A95E2F780958223C8
:1035200081B951C0813059F424B181E090E002C0EA
:10353000880F991F3A95E2F7282B24B944C08230AE
:1035400009F041C024B181E090E002C0880F991FCA
:103550003A95E2F78095822384B935C0813059F4D9
:1035600027B181E090E002C0880F991F3A95E2F7F9
:10357000282B27B928C0823031F527B181E090E0AF
:1035800002C0880F991F3A95E2F78095822387B988
:103590001AC0813059F42AB181E090E002C0880F4E
:1035A000991F3A95E2F7282B2AB90DC0823059F4B9
:1035B0002AB181E090E002C0880F991F3A95E2F7A6
:1035C000809582238AB98FEF90E00895382F377065
:1035D000869586958695813091F0813028F08230ED
:1035E000C9F0833011F12BC022B181E090E002C01C
:1035F000880F991F3A95E2F7282B22B920C025B1F0
:1036000081E090E002C0880F991F3A95E2F7282BDD
:1036100025B915C028B181E090E002C0880F991F3C
:103620003A95E2F7282B28B90AC02BB181E090E047
:1036300002C0880F991F3A95E2F7282B2BB98FEF1C
:1036400090E00895382F377086958695869581305D
:1036500099F0813028F08230D9F0833029F12FC0E1
:1036600022B181E090E002C0880F991F3A95E2F7FD
:103670008095822382B923C025B181E090E002C009
:10368000880F991F3A95E2F78095822385B917C074
:1036900028B181E090E002C0880F991F3A95E2F7C7
:1036A0008095822388B90BC02BB181E090E002C0E5
:1036B000880F991F3A95E2F7809582238BB98FEF97
:1036C00090E00895382F37708695869586958130DD
:1036D00051F0813030F0823041F0833041F02FEFF3
:1036E0000FC020B105C023B103C026B101C029B16C
:1036F00081E090E002C0880F991F3A95E2F72823F5
:10370000822F90E0089588E090E00895883018F0C6
:1037100080E090E00895E82FF0E0E059FF4FE49159
:103720008E2F90E00895883018F080E090E00895A2
:10373000E82FF0E0E059FF4FE4918E2FC3DF20E047
:10374000892B09F021E0822F90E00895883038F429
:10375000E82FF0E0E059FF4FE4918E2F73CF0895EA
:10376000883038F4E82FF0E0E059FF4FE4918E2FD5
:103770002DCF0895CF93DF93C0E7D0E005C0FE01C1
:10378000649181E0A3DE2196F0E0C837DF07B9F746
:10379000DF91CF9108958DE090E008958D3018F07D
:1037A00080E090E00895E82FF0E0E858FF4FE491C2
:1037B0008E2F90E00895FC010D9718F020E030E086
:1037C00006C0E858FF4F84917DDF282F30E0C90103
:1037D0000895CF93DF93C8E7D0E005C0FE01649160
:1037E00082E074DE2196F0E0C538DF07B9F7DF919B
:1037F000CF9108950F931F93CF93DF93EC018B012B
:103800002C986AE703C0F80161918F0180E090E095
:1038100075DC2197FFEFCF3FDF07A9F783E08A959B
:1038200001F0E9F7C8952C9ADF91CF911F910F9184
:1038300008951F93142F2C986F71682B80E090E0EF
:103840005DDC612F80E090E059DC83E08A9501F037
:10385000E9F7C8952C9A1F9108951F93CF93DF9392
:10386000182FC82FD0E0C076D0708091960590E0D8
:10387000C817D90781F043E06FE180EADADF85E01D
:10388000D595C7958A95E1F74C2F6FE180E8D1DF98
:10389000107610939605DF91CF911F9108950F93A5
:1038A0001F93082F162FD9DF412F602F80E4C1DF2F
:1038B0001F910F9108950F931F938C01FC0160815C
:1038C00084EEEDDFF801618185EEE9DFF8016281C8
:1038D00082EEE5DFF801638183EEE1DFF8016481C8
:1038E00080EEDDDFF801658181EED9DF1F910F9158
:1038F00008951F93162F2C986F71682B80E090E02D
:10390000FDDB60E080E090E0F9DB17FF04C060E0E1
:1039100080E090E0F3DB982F83E08A9501F0E9F7EF
:10392000C8952C9A892F90E01F9108951F93182F06
:1039300094DF612F80E0DDDF90E01F9108950F9309
:103940001F93CF93DF93EC018B018FE1EFDF83FDBA
:10395000FCCF60E082E0A3DF68E183E0A0DF6C2FB2
:1039600086E09DDFC050D84E6D2F772767FD7A9592
:10397000C050D84187E093DF40E060E08AE759DF3C
:10398000B801CE0137DF40E86FE180E852DF40E860
:103990006FE180EA4EDF48E06FE180E84ADF8FE1C7
:1039A000C5DF83FDFCCF48E06FE180EA42DFDF91B5
:1039B000CF911F910F91089582E7B8DF90E00895AD
:1039C0000F931F938B01682F84ED69DF602F86EDC5
:1039D00066DF012F110F110B602F87ED60DF8AEE7C
:1039E000A5DF80FDFCCF1F910F91089580E090E04E
:1039F00078DB249A2C9A4FEF60E08FEF1ADF8DE18D
:103A000095DF80FFFCCF109295051092940560E041
:103A100088E045DF60E089E042DF60E08CE03FDF86
:103A200060E08DE03CDF6EEF8AE039DF67E18BE03C
:103A300036DF60E084E033DF68E185E030DF61EAB3
:103A400088E32DDF6DE080EC2ADF60E081EC27DF8A
:103A500063E088EC24DF42E362EC80E8EADE62E1C6
:103A600086EC1DDF6CE087EC1ADF62E184EC17DF87
:103A700068E58AEC14DF62E08BEC11DF60E071E056
:103A800080E19EDF8FE1E9DE40EC6BE180E8D1DE92
:103A900044E06FE180E8CDDE66E774E084E190CF3A
:103AA0000F931F93682F84EDFADE61E082EDF7DE5D
:103AB0008AEE3CDF80FDFCCF60E082EDF0DE88ED39
:103AC00035DF082F10E089ED31DF90E0982F88274F
:103AD000802B912B1F910F9108954CE06FE180EAAC
:103AE000A8DE80E0DDDF9E7FBC0180E069DF82EC44
:103AF0001DDF90E08E7F682F82ECD1DE65E184ECE3
:103B0000CEDE62E186ECCBDE6CE087ECC8DE44E022
:103B10006FE180E88ECE81E0C3DF9695879596951C
:103B200087958095817090E00895EF92FF920F93B2
:103B30001F938C017B012C986AE380E090E0DEDA31
:103B4000A801B70180E090E0E8DA83E08A9501F00F
:103B5000E9F7C8952C9A1F910F91FF90EF90089567
:103B6000A0E0B0E0E6EBFDE10C94F175EC017B0127
:103B70008CE1DCDE86FD05C089E3D8DE882309F40C
:103B800047C06091940580E08ADE60919405709151
:103B90009505672F772781E082DE60E08AE3A9DE62
:103BA000082F10E0109395050093940560E08AE3D8
:103BB000A0DE90E0982F8827802B912B909395057D
:103BC0008093940560E08AE394DE082F10E060E0C3
:103BD0008AE38FDE90E0D82ECC24C02AD12A60E080
:103BE0008AE387DE60E08AE384DECC15DD059CF4A1
:103BF000609194058CE053DE609194057091950579
:103C0000672F77278DE04BDE40E46EE180E811DE20
:103C1000CC24DD243EC0B701C60187DF89E086DE03
:103C2000082F10E0102F002788E080DEE82E8BE0C0
:103C30007DDE90E0D82FCC278AE078DE90E0C82B9C
:103C4000D92B6091940570919505CB010197FF24C4
:103C50000E291F298017910718F0C817D90740F4BB
:103C60006C2F8CE01CDE6D2F772767FD7A950BC0DB
:103C700061508CE014DE609194057091950561505F
:103C80007040672F77278DE00ADE40E46EE180E820
:103C9000D0DDC601E8E0CDB7DEB70C940D763FB7B6
:103CA000F8942998219A80E897E00197F1F72198F4
:103CB00088E691E00197F1F723B180EF95E0019755
:103CC000F1F7199902C081E002C0822F82703FBFD4
:103CD00090E00895982F3FB7F894219A25E0822F1D
:103CE0008A95F1F7911121988AE48A95F1F7199B49
:103CF00090E080EF8A95F1F721982A95F1F73FBF80
:103D0000892F90E008950F931F93182F08E0812FBB
:103D10008170E0DF1695811110680150C1F7812F85
:103D200090E01F910F9108958FEFEDCF299A219A7E
:103D30000895A0E0B0E0EFE9FEE10C94F175D82E13
:103D4000EB01ADDF882319F08FEF90E037C080EFF3
:103D5000DADFCC2480E4E82EF12C08E081E0BADF41
:103D6000182F81E0B7DF882329F0112391F08EEF1F
:103D700090E024C0112369F42D2D30E0E216F30603
:103D800034F0888180FF05C02E153F0511F0CE2C40
:103D900011E0812F9FDF888186958883112311F0A0
:103DA000806888830894E108F1080150B9F6E114AD
:103DB000F10411F02196D1CF8C2D90E0E8E0CDB741
:103DC000DEB70C940D760F931F93CF93DF93082FDC
:103DD000EB0165DF209741F085E595DF18E08991DB
:103DE00092DF1150E1F702C08CEC8DDF802F8BDF6A
:103DF000DF91CF911F910F910895E4E7F1E020E06A
:103E000030E005C03396981729F02F5F3F4F90811F
:103E10009923C1F7F901EE0FFF1FE20FF31FEC58D2
:103E2000FE4F8181928108950F931F93CF93DF936B
:103E3000EC018881883239F0823229F0803119F022
:103E400080E090E81FC0BE0184E4BDDF6FDF88EE34
:103E500093E03FD8BE018EEBB6DF66DF8C0164DFF6
:103E6000382F2227202B312B8881803129F443E001
:103E7000220F331F4A95E1F7C90124E0880F991FEB
:103E80002A95E1F7DF91CF911F910F9108959B0142
:103E9000AC011092B90060E074E284EF90E00E94FF
:103EA000AA7520513040404050405695479537956F
:103EB00027952093B8008091B8008C30B8F084EA40
:103EC0008093BC0020E030E08091BC0087FF06C0FA
:103ED00081E080938F011092BC0008C085E38A9531
:103EE000F1F72F5F3F4F2436310571F780918F0135
:103EF00090E0089580918F01813039F484E98093B6
:103F0000BC008091BC0084FDFCCF08951F93282F36
:103F1000162F80918F01813009F04EC08091B90039
:103F2000887F883059F08091B900887F803131F0E6
:103F30008091B900887F883F09F03EC084EA809371
:103F4000BC008091BC0087FFFCCF8091B90090E05D
:103F5000887F90708830910511F0409749F4220FC6
:103F6000210F2093BB0084E88093BC0091E002C045
:103F7000C1DF90E08091BC0087FFFCCF9130E9F475
:103F8000112369F48091B900282F30E0287F307028
:103F90002831310591F02032310571F40CC0809147
:103FA000B900282F30E0287F30702034310529F007
:103FB0002834310509F49EDF90E0892F90E01F91AD
:103FC0000895982F80918F018130D9F48091B900A4
:103FD000887F883129F08091B900887F883289F400
:103FE0009093BB0084E88093BC008091BC0087FF65
:103FF000FCCF8091B900887F883211F481E002C043
:1040000079DF80E090E0089580918F01813039F46C
:1040100084EC8093BC008091BC0087FFFCCF809132
:10402000BB0090E0089580918F01813039F484E8DD
:104030008093BC008091BC0087FFFCCF8091BB00C7
:1040400090E008951F93CF93DF9380918F0181308B
:1040500019F0C0E0D0E00DC010E1C0E0D0E060E0B9
:10406000812F54DF813011F4219644DF1F5F103817
:10407000B1F7CE01DF91CF911F910895CF93DF93D8
:10408000EC019881892F88548830A8F460E0892F4A
:104090003DDF813081F480E094DF2CDF61E08881B6
:1040A00035DFB2DF90E0D82FCC27BDDF90E0C82B02
:1040B000D92B20DF02C0C0E0D0E8CE01DF91CF9144
:1040C00008958FB7F8941092980510929705109262
:1040D0009A051092990510929C0510929B051092DA
:1040E0009E0510929D058FBF0895E82F8FB7F89415
:1040F000F0E0EE0FFF1FE956FA4F718360838FBF28
:1041000080E090E00895E8E6F0E0908121E030E082
:1041100002C0220F331F8A95E2F7922B908380E032
:1041200090E00895382F2091680041E050E0CA01E6
:10413000062E02C0880F991F0A94E2F7282B2093BD
:104140006800613091F0613028F06230C9F063306E
:1041500011F12BC080916B0002C0440F551F3A959E
:10416000E2F7842B80936B0020C080916C0002C02A
:10417000440F551F3A95E2F7842B80936C0015C0CD
:1041800080916D0002C0440F551F3A95E2F7842BD1
:1041900080936D000AC08091730002C0440F551FC8
:1041A0003A95E2F7842B8093730080E090E00895C5
:1041B0001F920F920FB60F9211242F933F934F939C
:1041C0005F936F937F938F939F93AF93BF93EF937F
:1041D000FF93D89A8091970590919805892B29F0A3
:1041E000E0919705F09198050995FF91EF91BF91A6
:1041F000AF919F918F917F916F915F914F913F917F
:104200002F910F900FBE0F901F9018951F920F9235
:104210000FB60F9211242F933F934F935F936F9399
:104220007F938F939F93AF93BF93EF93FF93D99A0D
:104230008091990590919A05892B29F0E091990533
:10424000F0919A050995FF91EF91BF91AF919F91E0
:104250008F917F916F915F914F913F912F910F902F
:104260000FBE0F901F9018951F920F920FB60F92CE
:1042700011242F933F934F935F936F937F938F936B
:104280009F93AF93BF93EF93FF93DA9A80919B052F
:1042900090919C05892B29F0E0919B05F0919C055C
:1042A0000995FF91EF91BF91AF919F918F917F9170
:1042B0006F915F914F913F912F910F900FBE0F9093
:1042C0001F9018951F920F920FB60F9211242F93E3
:1042D0003F934F935F936F937F938F939F93AF938E
:1042E000BF93EF93FF93DB9A80919D0590919E057C
:1042F000892B29F0E0919D05F0919E050995FF918C
:10430000EF91BF91AF919F918F917F916F915F914D
:104310004F913F912F910F900FBE0F901F901895C6
:10432000833038F4E82FF0E0E155FF4FE4918E2F11
:1043300089C90895833038F4E82FF0E0E155FF4F44
:10434000E4918E2F43C908951F93182F833070F482
:10435000E82FF0E0E155FF4FE4918E2FB3D9892B80
:1043600019F0812FDDDF02C0812FE4DF1F91089556
:10437000CF93DF93C0E0D0E0FE01E155FF4FE49121
:104380006E2F81E0A3D88C2FCBDF2196C330D105CF
:1043900099F7DF91CF9108952F9A84B1806A84B9FB
:1043A000269880E58CBD81E08DBD08958EBD0DB44D
:1043B00007FEFDCF8EB590E00895DC018C918EBD97
:1043C00081E090E009C0FD01E80FF91FE0810DB424
:1043D00007FEFDCFEEBD019686179707A0F30DB43B
:1043E00007FEFDCF0895AC011EBC20E030E00BC0FD
:1043F0000DB407FEFDCF1EBC8EB5FA01E20FF31F10
:1044000080832F5F3F4F2617370791F70DB407FEC4
:10441000FDCF08955D988AB184628AB95498089551
:1044200020E090E0990F87FF02C05A9A01C05A9885
:104430005D9A4C9991605D982F5F283011F0880F3C
:10444000F1CF892F90E0089520E030E013C0FC0107
:10445000E20FF31FE08140E0E7FF02C05A9A01C07B
:104460005A985D9A5D984F5F483011F0EE0FF4CF87
:104470002F5F3F4F2617370751F70895FC015A98D1
:1044800080E090E030E00BC020E0330F5D9A4C9963
:1044900031605D982F5F2830C1F731930196861700
:1044A000970791F708951F920F920FB60F9211245C
:1044B0002F933F934F935F936F937F938F939F932C
:1044C000AF93BF93EF93FF93E0919F05F091A00509
:1044D000309709F00995FF91EF91BF91AF919F91AE
:1044E0008F917F916F915F914F913F912F910F909D
:1044F0000FBE0F901F90189580919001882339F47A
:104500008FB78093A105F89481E0809390012B9858
:1045100008952B9A80919001813029F41092900196
:104520008091A1058FBF08956FEF80E090E00E9419
:104530007E1890E00895682F80E090E00C947E183B
:10454000DF92EF92FF920F931F93D82E7A018B0187
:10455000EBDF8D2D8064EFDF812F9927AA27BB2702
:10456000EADFC801AA27BB27E6DFBB27A12F902FD0
:104570008F2DE1DF8E2DDFDFDD2021F088E0D816E2
:1045800019F004C085E903C087E801C08FEFD3DFCD
:1045900010E0CADF8F3F19F41F5F1A30D1F790E0A7
:1045A0001F910F91FF90EF90DF900895A0E0B0E091
:1045B000ECEDF2E20C94E7753B014C012A01190184
:1045C00060C0E301D170CE01A0E0B0E074016301EE
:1045D000C81AD90AEA0AFB0AA12C32E0B32EAC1A97
:1045E000BD0A2A143B0408F4510180919103909173
:1045F0009203A0919303B0919403C816D906EA06DA
:10460000FB0669F179DFB701A60181E199DF882313
:1046100021F07FDF80E090E03AC086DF8E3FE9F74F
:1046200001E911E081DFF80181938F01F3E00139A5
:104630001F07C1F7C0929103D0929203E0929303B7
:10464000F0929403CF56DE4FA501BE01C2010E9435
:104650009D774A0C5B1C68DF67DF5BDF09C0CF56C4
:10466000DE4FA501BE01C2010E949D774A0C5B1C72
:104670002A183B08C501A0E0B0E0680E791E8A1E2A
:104680009B1E2114310409F09CCF81E090E0E2E10F
:10469000CDB7DEB70C940376A0E0B0E0E2E5F3E23C
:1046A0000C94E9755B016C012A0139016EC0E501CA
:1046B000D170CE01A0E0B0E086017501E81AF90AD8
:1046C0000A0B1B0B812C42E0942E8C1A9D0A681455
:1046D000790408F443018091910390919203A09191
:1046E0009303B0919403E816F9060A071B07C1F07B
:1046F000209729F480E0881682E0980648F420E0AC
:1047000032E041E951E0C801B70150DF8823E1F010
:10471000E0929103F0929203009393031093940319
:1047200081E9481681E0580639F0A401B201CE01B2
:104730008F569E4F0E949D77DFDEB801A70188E16A
:10474000FFDE882321F0E5DE80E090E024C08EEFDC
:10475000F2DEC1E9D1E08991EEDE83E0C139D8070C
:10476000D1F78FEFE8DE8FEFE6DEDEDE8F3FE9F791
:10477000DBDECFDE480C591CC401A0E0B0E0A80E7F
:10478000B91ECA1EDB1E681879086114710409F08D
:104790008ECF81E090E0E0E1CDB7DEB70C940576F6
:1047A000A0E0B0E0E6EDF3E20C94E9755B016C018A
:1047B0004A01E90138012701452B59F1012B49F143
:1047C000FF24232B09F5FF24F3941EC09201B601A8
:1047D000A501C401F30109958C010097E9F0FF20C0
:1047E00019F4C817D907A8F09801A401C601B501AA
:1047F00053DF882371F0C801A0E0B0E0A80EB91E15
:10480000CA1EDB1EC01BD10BFF2001F72097F1F65B
:1048100003C080E090E002C081E090E0E0E1CDB72D
:10482000DEB70C940576A0E0B0E0E9E1F4E20C9488
:10483000E9754B015C013A01E9012601452B71F153
:104840002115310559F10217130740F1E114F10464
:1048500029F1CC24DD24C21AD30A021B130B9E01BA
:10486000A301C501B401A2DE8823C1F09201B50104
:10487000A401C301F7010995882399F00C0D1D1DB2
:10488000C8018C0F9D1F8C179D0758F0CE01A0E02A
:10489000B0E0880E991EAA1EBB1EE1CF80E090E01A
:1048A00002C081E090E0E0E1CDB7DEB70C94057680
:1048B0001F93CF93DF93239A579A5F9A559A5D9AE5
:1048C00057981ADE26DE80E090E00E947118109260
:1048D000950310E029DE1F5F1436E1F70DDEC0E01E
:1048E000D0E040E050E060E070E080E029DE813020
:1048F00039F08FE0CF3FD80709F45BC02196F1CFA4
:1049000040E050E060E070E087E31ADE40E050E015
:1049100060E070E089E214DE82FD05C080919503BD
:10492000816080939503C0E0D0E08091950390E092
:1049300083709070892B61F040E050E060E070E09F
:1049400087E3FEDD40E050E060E070E089E205C012
:1049500040E050E060E070E081E0F2DD80FF06C002
:104960008FE7CF3FD80729F12196DFCF40E052E013
:1049700060E070E080E1E4DD8823D9F4CADD8FEFE8
:104980009FEFAFEFBFEF8093910390939203A093BB
:104990009303B093940320E032E041E951E060E0FA
:1049A00070E080E090E002DE882319F081E090E082
:1049B00003C0AFDD80E090E0DF91CF911F910895BB
:1049C0000F931F9360E080E2A1DA813009F58091B6
:1049D00096038F7B8093960380919603F2DA809101
:1049E000960380648093960380919603EADA00E947
:1049F00011E0C8010197F1F7809196038F7B8093B6
:104A0000960380919603DDDA75DAC8010197F1F714
:104A10001F910F91089590919603907F9093960324
:104A20009091960382958F70982B90939603C8CFA0
:104A30001F93182F80919603806180939603812F96
:104A4000EADF812F8295807FE6DF81E090E00E949F
:104A500069171F9108951F93182F809196038F7ED9
:104A600080939603812FD7DF812F8295807FD3DFBC
:104A700081E090E00E9469171F9108956093970369
:104A800080939803662319F0613019F008958068C7
:104A900001C0806CE0CF81E0DEDF82E0DCDF1092DD
:104AA00097031092980308951F93182F8A3048F1A6
:104AB0008D3019F46091970309C08A3051F46091E8
:104AC00097036F5F609397036230D0F480E0D6DF86
:104AD00018C080919803803158F0609197036F5F00
:104AE00060939703623060F41092980380E0C6DF11
:104AF000812F9EDF809198038F5F8093980301C080
:104B0000CADF1F9108951F93CF93DF9310929603EE
:104B100080E381DF85E090E00E94691751DF81E04A
:104B200090E00E9469174CDF81E090E00E946917D5
:104B300080E271DF85E090E00E9469178CE28BDFF4
:104B400081E089DF82E087DF8CE085DF10929703C8
:104B50001092980360E080E2D9D98130F9F410E036
:104B6000C0E0D0E012C0812F90E0C817D90724F030
:104B7000809196038F7703C080919603806880931D
:104B80009603809196031DDA1F5F17FFECCF2196E5
:104B9000C038D10514F410E0E6CFACD9809196036B
:104BA0008F7780939603DF91CF911F910895A2E1B3
:104BB000B0E0EDEDF5E20C94F475F0B080E8F82289
:104BC000809199038F1509F443C180919A03803134
:104BD00029F410929D0387EA93E008C0853159F4C7
:104BE00010929E0310929D0386EA93E090939C039B
:104BF00080939B0365C08D3189F400919B031091D4
:104C00009C03F80180810E94AC40F80180831092DF
:104C10009E0310929D0385EA93E0E8CF843289F4E5
:104C200000919B0310919C03F80180810E94AC408D
:104C3000F801808310929E0310929D0384EA93E012
:104C4000D5CF8A3279F400919B0310919C03F8012F
:104C500080810E94AC40F801808310929D0383EA1A
:104C600093E0C4CF8D3279F400919B0310919C03A3
:104C7000F80180810E94AC40F801808310929D036E
:104C800082EA93E0B3CF823379F400919B031091D1
:104C90009C03F80180810E94AC40F801808310924F
:104CA0009D0381EA93E0A2CF8A3351F400919B03E4
:104CB00010919C03F80180810E94AC40F801808330
:104CC00081E042DB20919F033091A003C901C3978B
:104CD0008336910530F540919A034C3121F04332EF
:104CE00011F04A3341F480919E0380FF49C081E076
:104CF00080932A0145C0E0919B03F0919C03309181
:104D00009D0381E090E0032E02C0880F991F0A9452
:104D1000E2F780952081282320833F5F30939D0315
:104D20002FC0C901875990408336910568F540919D
:104D30009A034C3121F0433211F04A3341F480910F
:104D40009E0380FD18C081E080932A0114C0E09189
:104D50009B03F0919C0330919D0381E090E0032E32
:104D600002C0880F991F0A94E2F72081282B208324
:104D70003F5F30939D0380919E038F5F80939E03DE
:104D80004F5F40939A0360C0C9018F5E9240873C99
:104D9000910508F459C0275D3640273C310508F0DD
:104DA00050C080912A018823D9F580919A038B33D2
:104DB000B9F58E010F5F1F4FC8010E94F8161982C6
:104DC0001A828091A6038B838091A5038C838091A6
:104DD000A4038E838091A30367E00E9477759D836F
:104DE0008091A2038F838091A10390E08053984F1C
:104DF00099878887C8010E9409168091A70381FFBF
:104E00000CC08F859889A989BA8980519E40A0409D
:104E1000B0408F87988BA98BBA8BC8010E94E71688
:104E200010922A0110929A031092A5031092A603E1
:104E30001092A4031092A3031092A2031092A10354
:104E400003C082E080932A011092A00310929F0376
:104E500080919F039091A0030A969093A003809362
:104E60009F03F0929903E5E062960C9410760F98F8
:104E700061E087ED95E20C948417A0E0B0E0E3E4F4
:104E8000F7E20C94F1756C017B01EB012E96FB01AE
:104E90008685682F70E06F707070660F771F660FE1
:104EA000771F8E01060F171FF80180818823F1F10B
:104EB000883009F048C08C859D85AE85BF85888B7C
:104EC000998BAA8BBB8B8091340190913501A09175
:104ED0003601B09137018C879D87AE87BF871B86CF
:104EE0001A86CE010E94C1400E94304E9B878A875D
:104EF000F801108211828281883F18F083818F5FD0
:104F00008383F8018281885F8283F701ADE2B1E09B
:104F1000868180838D918683319621E0A333B20709
:104F2000B9F7B701C6010E94C7350DC0F8018481E9
:104F300095818D519C4A39F480912B01813019F46F
:104F400082E080932B01E8E0CDB7DEB70C940D76BC
:104F50009C0106971CF0EFEFFFEF12C08FB7F8949B
:104F6000F901EE0FFF1FE20FF31F93E0EE0FFF1F9B
:104F70009A95E1F7EE55FA4F0190F081E02D8FBF41
:104F8000CF0108959C0106971CF02FEF3FEF11C051
:104F90008FB7F894F901EE0FFF1FE20FF31F53E0F4
:104FA000EE0FFF1F5A95E1F7EE55FA4F228933892C
:104FB0008FBFC90108959C0106971CF08FEF9FEFEA
:104FC00008958FB7F894F901EE0FFF1FE20FF31F5A
:104FD00093E0EE0FFF1F9A95E1F7EE55FA4F138A13
:104FE000128A20E130E0318320838FBF80E090E09F
:104FF0000895863091051CF08FEF9FEF08952FB72D
:10500000F894FC01EE0FFF1FE80FF91F73E0EE0F9D
:10501000FF1F7A95E1F7EE55FA4F80819181892B38
:1050200091F01182108212821382148215821186ED
:10503000108617821682138A128A118A108A158A9C
:10504000148A178A168A2FBF80E090E00895CF93C4
:10505000DF93C0E0D0E0CE01CCDF2196C630D10591
:10506000D1F7DF91CF9108954FB7F894E2EAF5E0D8
:1050700020E030E080819181892B11F4C90108C0C2
:105080002F5F3F4F789626303105A1F78FEF9FEFC6
:105090004FBF0895A0E0B0E0E0E5F8E20C94F275AF
:1050A000EC018B017A01DFB6F894DEDF9C018FEF13
:1050B0002F3F380701F1F901EE0FFF1FE20FF31F39
:1050C000B3E0EE0FFF1FBA95E1F7EE55FA4F80E11E
:1050D00090E09183808311861086D783C6831282E5
:1050E000138214821582138A128A118B008BF58A1F
:1050F000E48A178A168ADFBEC901E7E0CDB7DEB7BA
:105100000C940E76EF92FF920F931F93CF93DF9341
:105110009C01EB01FA0106971CF08FEF9FEF36C060
:10512000868590E08F709070880F991F880F991F67
:105130005EE0E52EF12CEE0EFF1EE80EF91E890151
:10514000000F111F020F131F93E0000F111F9A95FC
:10515000E1F70E551A4FF801808591850E94304E77
:10516000F70193838283F801868197810E94304EF4
:10517000F7019183808317821682CE0108960E94E0
:10518000304EF7019583848380E090E0E6E0CDB770
:10519000DEB70C940F76A0E0B0E0E1EDF8E20C94FD
:1051A000EC755C011EE0812E912C880E991EFC018D
:1051B0008685C82FD0E0CF70D070CC0FDD1FCC0F0C
:1051C000DD1FC80DD91D7FB6F894A2EAEA2EA5E02E
:1051D000FA2ECC24DD24F701068117818A819B8178
:1051E0000E94304E0817190709F046C0F7010085E4
:1051F0001185888199810E94304E08171907D1F1D5
:10520000F70180859185892BB9F582819381A481ED
:10521000B5810097A105B10579F58601000F111F31
:105220000C0D1D1DE3E0000F111FEA95E1F772EA76
:10523000E72E75E0F72EE00EF11EF40184859585CA
:10524000A685B785F70182839383A483B58388817C
:1052500099810E94304EF7019187808786E090E027
:10526000A80EB91E46E050E0B501C80184559A4F1A
:105270000E949D77C6010EC00894C11CD11CE8E1B4
:10528000F0E0EE0EFF1EF6E0CF16D10409F0A3CF3A
:105290008FEF9FEF7FBEEDE0CDB7DEB70C940876C1
:1052A000A0E0B0E0E6E5F9E20C94ED754B01EB010E
:1052B0002E96FB011685CB016EDF5C018F5F9F4F41
:1052C00009F47AC0012F10E00F701070000F111F49
:1052D000000F111F0C0F1D1FF801848195810E9482
:1052E000304E089709F468C0F4018685E82EFF2443
:1052F000FFE0EF22FF24EE0CFF1CEE0CFF1C86E10A
:1053000090E0E80EF91EE501CC0FDD1FCA0DDB1D94
:1053100093E0CC0FDD1F9A95E1F7CE55DA4FCE889A
:10532000DF88C114D104C1F0F801848195810E9405
:10533000304EBC01C4018E0D9F1DF601099580E120
:1053400090E099838883198618861A821B821C82B2
:105350001D821B8A1A8A30C088819981409761F525
:10536000F801848195810E94304E488959890897B7
:105370008417950740F4F801848195810E94304E8E
:10538000AC0148505040F501EE0FFF1FEA0DFB1D28
:1053900003E0EE0FFF1F0A95E1F7EE55FA4F538B2E
:1053A000428B80E290E091838083E80CF91CB70186
:1053B000848995890E949D77ECE0CDB7DEB70C9487
:1053C0000976A0E0B0E0E7EEF9E20C94E9753C0163
:1053D0004B018A014DB65EB686E0681671041CF07A
:1053E0008FEF9FEF48C00E94A0357AE2A72EB12C24
:1053F000A80CB91CEDB7FEB7EA19FB090FB6F89473
:10540000FEBF0FBEEDBFCDB6DEB60894C11CD11CE9
:1054100085E487878DB79EB78B96A401B8010E945B
:105420009D779401285F3F4F7301EE0CFF1CE60C43
:10543000F71C53E0EE0CFF1C5A95E1F7F701EE550F
:10544000FA4F6281738184819581860141E10E94D6
:105450002239A601B401C30155DEB601C701845546
:105460009A4F0E946035B601C5010E94C7350E945F
:105470007A3580E090E00FB6F8945EBE0FBE4DBE68
:10548000E0E10C9405766F927F929F92AF92BF926B
:10549000CF92DF92EF92FF920F931F93CF93DF9300
:1054A0006B017C01EA0139019FB6F894DDDD5C01F6
:1054B0008FEFA8168FEFB80609F48BC0F501EE0F39
:1054C000FF1FEA0DFB1DA3E0EE0FFF1FAA95E1F7FA
:1054D000EE55FA4F80E190E091838083D187C087B9
:1054E000C334D10529F484E490E09783868304C013
:1054F000C095D095D783C683E501CC0FDD1FCA0DBB
:10550000DB1DE3E0CC0FDD1FEA95E1F7FE01EE5570
:10551000FA4FC282D382E482F582138A128A718A98
:10552000608A158B048B178A168A8FEFC8168FEF47
:10553000D8068FEFE8068FEFF80641F100913801A9
:105540001091390120913A0130913B01009510955D
:1055500020953095B701A601402351236223732380
:105560008091340190913501A0913601B0913701BD
:1055700080239123A223B323481759076A077B0787
:10558000C1F4401751076207730741F48FEF828718
:10559000838784878587868787871BC09FBEAE01E8
:1055A00044555A4FC701B6010E948A379FB6F894F6
:1055B00010C09FBEAE0144555A4F60913C0170919E
:1055C0003D0180913E0190913F010E948A379FB634
:1055D000F8949FBEC501DF91CF911F910F91FF906D
:1055E000EF90DF90CF90BF90AF909F907F906F90A3
:1055F000089510922C01089581E080932C01089564
:1056000080913206882349F480914806909149069A
:10561000892B19F480E090E0089580918A06882310
:1056200049F48091A0069091A106892B19F481E09C
:1056300090E008958091E206882349F48091F8066D
:105640009091F906892B19F482E090E008958FEF8C
:105650009FEF0895AC0120E030E0F901EE0FFF1F4D
:10566000E65CF84F80819181892B29F45183408336
:1056700080E090E008952F5F3F4F2430310569F7B7
:105680008FEF9FEF0895AC0120E030E0F901EE0FBD
:10569000FF1FE65CF84F808191818417950719F40C
:1056A00080E090E008952F5F3F4F2430310571F77F
:1056B0008FEF9FEF0895AC016FEF7FEFAEE1B0E0A9
:1056C00020E030E088E590E0289FF001299FF00D70
:1056D000389FF00D1124EE5CF94F84819581841779
:1056E000950771F480818F3059F4868997898A17DC
:1056F0009B0730F486899789DC0180E18083B901BA
:105700002F5F3F4F23303105E9F6CB010895FC01AF
:10571000039718F08FEF90E0089588E590E09F01DF
:10572000289FF001299FF00D389FF00D1124EE5CA9
:10573000F94F808190E008959C01039790F488E5EB
:1057400090E0289FF001299FF00D389FF00D112463
:10575000EE5CF94F8081803121F486A197A10C94F1
:1057600038468FEF9FEF08959C01039790F488E5EA
:1057700090E0289FF001299FF00D389FF00D112433
:10578000EE5CF94F8081803121F486A197A10C94C1
:10579000AC458FEF9FEF0895A0E0B0E0E2EDFBE2B3
:1057A0000C94F1756C01FB01EA0130C080818130FD
:1057B00029F0813068F1883021F022C0319621979C
:1057C00025C0018110E022E0E22EF12CEE0EFF1E3A
:1057D00088E590E09C01C29EC001C39E900DD29EC0
:1057E000900D112444E050E0B701865B994F0E9470
:1057F0009D77F701E00FF11F3297C01BD10B06C058
:10580000818190E0E80FF91FC81BD90B209771F632
:10581000E8E0CDB7DEB70C940D76A0E0B0E0E3E1B0
:10582000FCE20C94F0756B017A018A01025F1F4F54
:10583000FA01B68428E530E0829FE001839FD00D15
:10584000929FD00D1124CE5CD94F8EA19FA10E94B2
:1058500055468C159D0524F4CC24CA94DC2C27C015
:105860008B2D90E08F709070880F991F880F991F73
:10587000080F191FF80124858EA19FA1F701468505
:1058800050E04F705070440F551F440F551F30E0CB
:10589000207F30703595279535952795420F531FFA
:1058A000425F5F4F4E0D5F1DB6010E946F46C601FD
:1058B000E9E0CDB7DEB70C940C76A0E0B0E0E3E60B
:1058C000FCE20C94EF75FC01AEE0AA2EB12CA80E00
:1058D000B91E8685C82FD0E0CF70D070CC0FDD1FE9
:1058E000CC0FDD1FCA0DDB1DCC24DD2488E590E044
:1058F000C89E7001C99EF00CD89EF00C112482E362
:1059000096E0E80EF91EF7018081882311F10281EB
:105910001381888199810E94304E08171907C9F4B4
:10592000F701048115818A819B810E94304E0817FE
:10593000190779F4F7012681378140855185F501F2
:1059400084859585A685B785281739074A075B079B
:1059500051F00894C11CD11CF3E0CF16D10431F6EC
:10596000CC24CA94DC2CC601EAE0CDB7DEB70C9497
:105970000B76A0E0B0E0EFEBFCE20C94ED75EC01EF
:105980001EE0812E912C880E991EEE8439DE5C017A
:105990008FEFA8168FEFB80609F477C0FF24EFE069
:1059A000EE22FF24EE0CFF1CEE0CFF1CE80CF91C91
:1059B000F701808191810E94304E28E530E0A29E5F
:1059C0006001A39ED00CB29ED00C112486010E5C07
:1059D000194FF80193838283F701828193810E949A
:1059E000304EF80195838483F40184859585A685DE
:1059F000B785F80186839783A087B187F701648113
:105A00007581868197810E94344E6095709580954E
:105A10009095F8016287738784879587F701648181
:105A20007581868197810E94344EF8016687778759
:105A3000808B918B11828AE090E0978B868B108E01
:105A4000118E128E138E6AE070E080E090E00E946A
:105A5000344EF801648F758F868F978F86A197A13A
:105A60000E943846F701868597850E94304EF801DE
:105A7000938B828B158A148A269646E050E0BE01ED
:105A8000C6018E5A994F0E949D77C501ECE0CDB7B3
:105A9000DEB70C9409762F923F924F925F926F92ED
:105AA0007F928F929F92AF92BF92DF92EF92FF927E
:105AB0000F931F93CF93DF93CDB7DEB724970FB625
:105AC000F894DEBF0FBECDBF9A838983D62E2A01FC
:105AD0007901580198012E5D3F4F3C832B8396E15D
:105AE000692E712C600E711E88E590E0E981FA81C3
:105AF000E89F4001E99F900CF89F900C11248401CD
:105B00000E5C194FF80186819781A085B185F5015A
:105B1000868B978BA08FB18F809134019091350146
:105B2000A0913601B0913701F30184839583A68358
:105B3000B783108686E0818784E2282E312C240EDC
:105B4000351EC1010E94304EF30193878287F80110
:105B5000848195810E94304EF50193A382A3F801C0
:105B6000828193810E94304EEB81FC8193838283FA
:105B7000F80162857385848595850E94344EEB819A
:105B8000FC816483758386839783F80166857785B6
:105B9000808991890E94344EEB81FC8160877187F6
:105BA0008287938780E98487D586C7010E94304E1B
:105BB000EB81FC8197878687118A108A138A128A63
:105BC000F801648D758D868D978D0E94344E6F5FC0
:105BD0007F4F8F4F9F4F0E94344EF801648F758F17
:105BE000868F978F40E150E060E070E0C501C69677
:105BF0000E94A677F8018081813051F582E0EB8127
:105C0000FC81848B84E0858B168A80E4878BF80185
:105C1000808D918DA28DB38D0097A105B105C9F13D
:105C200088E0EB81FC81808F8AE0818FB401625B28
:105C3000794F44E050E0C501CC960E949D77B401B5
:105C4000665B794F44E050E08B819C814E961FC08B
:105C5000F801808D918DA28DB38D0097A105B105BE
:105C6000C1F088E0EB81FC81848B8AE0858BB401F4
:105C7000625B794F44E050E0C501C8960E949D7771
:105C8000B401665B794F44E050E0C501CC960E94B8
:105C90009D7720E330E0420E531EB201C3010E9403
:105CA000C1400E94304EEB81FC81918B808B88E556
:105CB00090E029813A81289F7001299FF00C389F3C
:105CC000F00C1124F701EE5CF94F66817781808535
:105CD00091858501910146E00E942239B501C701F5
:105CE0008E5A994FEDD6B501C201469650D72496EB
:105CF0000FB6F894DEBF0FBECDBFDF91CF911F91DD
:105D00000F91FF90EF90DF90BF90AF909F908F909A
:105D10007F906F905F904F903F902F900895A6E4F2
:105D2000B0E0E5E9FEE20C94F2757C0183E0E81650
:105D3000F104C0F588E590E0E89E8001E99E100D31
:105D4000F89E100D11240E5C194FF80180818031EE
:105D500049F586A197A10E94AC45892B19F1F0D68F
:105D6000F80186A197A10E940046D82EF80186A1CD
:105D700097A10E94AC45892B89F4F80186A197A1CF
:105D80000E94AC4520E330E0281B390B8E010F5FE9
:105D90001F4F40E050E060E1C7017DDEABD68D2DA6
:105DA00090E002C080E090E0E7E0CA5BDF4F0C9437
:105DB0000E76A6E8B0E0EFEDFEE20C94E7753C014C
:105DC0002B011801039708F0FDC088E590E0689E5C
:105DD000F001699EF00D789EF00D1124EE5CF94FF4
:105DE0008081803109F0EEC0222349F0213009F092
:105DF000E9C0DE01A95BBF4FCC24DD241AC0DE015F
:105E0000A95BBF4FCC24DD2408C0FA01EC0DFD1DB9
:105E100080818D930894C11CD11CC414D504ACF3AB
:105E20000BC0F601E40FF51FE491ED930894C11C3B
:105E3000D11CC414D504ACF383D688E590E0689EE9
:105E40007001699EF00C789EF00C112482E396E0BC
:105E5000E80EF91EF70186A197A10E94AC4520E348
:105E600030E0281B390B8E010F5F1F4FA20168E144
:105E7000C30111DEF70182859385A485B58596015E
:105E80005901CC24B7FCC094DC2C8A0D9B1DAC1DA1
:105E9000BD1D82879387A487B587558A448A2AD6F1
:105EA0000E9447174C018F5F9F4F09F48BC012145B
:105EB000130424F041E06CE070E007C023E02216F8
:105EC000310434F441E068EC70E0C4010E9423170F
:105ED00037D688E590E0689E7001699EF00C789E48
:105EE000F00C112482E396E0E80EF91EF70182859A
:105EF0009385A485B5858A199B09AC09BD0982875C
:105F00009387A487B58786A197A10E94AC4520E31B
:105F100030E0281B390B8E010F5F1F4F40E050E02F
:105F200060E1C301B8DDF70182859385A485B5855D
:105F30008A0D9B1DAC1DBD1D82879387A487B587E5
:105F4000D9D5FED5C4010E940917892B39F5C401A2
:105F50000E94C71388E590E0689EF001699EF00DED
:105F6000789EF00D1124EE5CF94F82859385A4850F
:105F7000B5858A199B09AC09BD0982879387A487D7
:105F8000B5878091A8039091A90301969093A903E6
:105F90008093A80344244A94542C12C088E590E0CE
:105FA000689EF001699EF00D789EF00D1124EE5C64
:105FB000F94F84899589892B19F6C4010E94C7136A
:105FC00099D503C044244A94542CC201E2E1CA5733
:105FD000DF4F0C940376A6E4B0E0E1EFFFE20C940F
:105FE000F1756C0183E0C816D10408F0C0C088E5E3
:105FF00090E0C89EF001C99EF00DD89EF00D1124CE
:10600000EE5CF94F8081803109F0B1C00E944717E2
:106010008C019FEF0F3F190709F4A9C041E068EC1C
:1060200070E0C8010E94231788E590E0C89E7001C7
:10603000C99EF00CD89EF00C1124E2E3F6E0EE0EBF
:10604000FF1EF7018181882339F5C8010E940917D5
:10605000892B11F1C8010E94C71372D5F70186A1DF
:1060600097A10E94AC4520E330E0281B390B8E013C
:106070000F5F1F4F40E050E061E1C6010CDD81E79A
:10608000F701808337D50E9447177C01FFEF8F3FD0
:106090009F0709F46CC018C0C8010E940917892B1A
:1060A00009F0C2CF88E590E0C89EF001C99EF00DCE
:1060B000D89EF00D1124EE5CF94F178A168A1082D3
:1060C000C8010E94C71353C041E068EC70E00E9411
:1060D000231736D588E590E0C89EF001C99EF00DE3
:1060E000D89EF00D1124EE5CF94F86A197A10E9475
:1060F000AC4520E330E0281B390B8E010F5F1F4FAA
:1061000040E050E061E1C601C6DCF4D419D588E571
:1061100090E0C89EF001C99EF00DD89EF00D1124AC
:10612000EE5CF94F8081882329F4C7010E9409178A
:10613000892BC9F4C7010E940917892B31F788E51B
:1061400090E0C89E8001C99E100DD89E100D1124AC
:106150000E5C194F48E051E060E070E0C8010E9419
:10616000A677F8011082C7010E94C713C3D4E8E0E4
:10617000CA5BDF4F0C940D762F923F925F926F9225
:106180007F928F929F92AF92BF92CF92DF92EF92C7
:10619000FF920F931F93CF93DF935C016B011A0162
:1061A000522E039708F06CC088E590E0A89EF0019D
:1061B000A99EF00DB89EF00D1124EE5CF94F808180
:1061C000803109F05DC0CB0160E470E00E949775FA
:1061D0003B01E10188249924EE24FF2419C081E0C9
:1061E0008515E8F38701252DAE0160E470E0C50157
:1061F000E0DD8F5F9F4F39F40894E11CF11C83E0D0
:10620000E816F10461F70894811C911CC05CDF4F13
:10621000861497041CF4EE24FF24F1CF23E0E21649
:10622000F10461F1C6018F739070892B61F1E40173
:1062300026E0CC0FDD1F2A95E1F7C20DD31DC60164
:1062400060E470E00E9497754C01EE24FF2481E029
:10625000851560F08701252DAE01B401C501A9DDCA
:106260008F5F9F4F39F40894E11CF11C83E0E8161E
:10627000F1046CF323E0E216F10429F4C501ABDE6E
:10628000CC24CA94DC2CC601DF91CF911F910F91D1
:10629000FF90EF90DF90CF90BF90AF909F908F9046
:1062A0007F906F905F903F902F900895A6E4B0E0AC
:1062B000ECE5F1E30C94EF7580912C01813009F04D
:1062C0006AC032E3A32E36E0B32ECC24DD2488E569
:1062D00090E0C89E7001C99EF00CD89EF00C11246D
:1062E00082E396E0E80EF91EF70186899789892BEB
:1062F000C1F180818823A9F1868997890197978BBD
:10630000868B868997890A97A1F486A197A10E9416
:10631000AC4520E330E0281B390B8E010F5F1F4F87
:1063200040E050E061E1C601B6DB81E7F701808320
:1063300026C0F70186899789892B09F58E010F5FA1
:106340001F4F20E030E040E050E064E0C601A3DBF6
:1063500048E051E060E070E0C5010E94A677F701D7
:106360000BC088E590E0C89EF001C99EF00DD89E54
:10637000F00D1124EE5CF94F178A168A10820894EA
:10638000C11CD11C88E590E0A80EB91E93E0C91687
:10639000D10409F09CCFEAE0CA5BDF4F0C940B7686
:1063A000A0E0B0E0E6EDF1E30C94E7751B018B0192
:1063B000025F1F4FFB018685682E7724FFE06F2266
:1063C0007724660C771C660C771C600E711ECB015F
:1063D00074DA2C01F301858583718587FFEF4F16F1
:1063E000FFEF5F0651F4F301828193810E94304EEA
:1063F0004AD98F5F9F4F09F42AC3F3018485C82FC0
:10640000D0E0C07FD070D595C795D595C7956497D6
:106410008585823009F04CC0C101ABDA6C01FFEF19
:106420008F3F9F0709F413C3B3016C5E7F4FAE012A
:10643000B3D988E590E0C89E7001C99EF00CD89E43
:10644000F00C112482E396E0E80EF91E81E0F701DA
:106450008083F301868597850E94304EF701938BE8
:10646000828B86859785A089B1890196A11DB11D72
:1064700086879787A08BB18B810120E330E040E0D5
:1064800050E062E1C60107DBF70182859385A485B0
:10649000B5850196A11DB11D82879387A487B58715
:1064A00084E0808311828AE090E0978B868BCFC254
:1064B000FFEF4F16FFEF5F0609F4C9C288E590E0D1
:1064C000489E4001499E900C589E900C112482E3F6
:1064D00096E0880E991E8EE190E0F401978B868BF2
:1064E000B3016C5E7F4FAE01C20156D9F3018585C1
:1064F000823171F560857185828593850E94344E65
:10650000F4016287738784879587F30164817581BD
:10651000868197810E94344EF40166877787808B4D
:10652000918B86859785A089B1890196A11DB11DA2
:1065300086879787A08BB18BF301868597850E940C
:10654000304EF401938B828B80E1808311827FC275
:10655000F801828193810E94A440F301448550E0B8
:10656000407F50705595479555954795F101268583
:1065700030E02F703070220F331F220F331F420F75
:10658000531FEC01C41BD50B5E01CC24DD24F401A8
:1065900086A197A10E945546AA2797FDA095BA2FDC
:1065A0008A159B05AC05BD050CF451C2209709F472
:1065B0002DC1F401E684F78400891189F301648117
:1065C0007581868197810E94344EE616F70608078A
:1065D000190709F087C0A101BE01C2011ED98F5F52
:1065E0009F4F81F0F30164817581868197810E94BC
:1065F000344E6A0D7B1D8C1D9D1DF40166877787C7
:10660000808B918BF40186A197A10E94AC45C0E3D9
:10661000D0E09E01281B390B810140E050E060E191
:10662000C20139DA80914407909145078415950598
:1066300009F053C0609142077091430761157105DD
:1066400009F44BC0F40186859785A089B1899B0127
:1066500040E050E0820F931FA41FB51FE090460753
:10666000F090470700914807109149072E0D3F1DF4
:10667000401F511F82179307A407B50729F586A16C
:1066800097A14AE457E00E946F4680914607909197
:106690004707A0914807B0914907A80EB91ECA1E26
:1066A000DB1EF401A686B786C08AD18A86A197A18F
:1066B0000E94AC45C81BD90B81019E0140E050E00F
:1066C00060E1C201E8D909C08091AA039091AB03AF
:1066D00001969093AB038093AA0310924307109204
:1066E000420794C0F401E684F78400891189F3011C
:1066F00064817581868197810E94344EEA0CFB1C6F
:106700000C1D1D1DA60EB71EC81ED91EAE14BF043B
:10671000C006D10660F5F401C684D784E088F1880C
:10672000F30184819581A681B781F40186879787DB
:10673000A08BB18B86A197A10E94AC4520E330E0ED
:10674000281B390B810140E050E060E1C201A3D970
:10675000F401C686D786E08AF18A8091AC039091D5
:10676000AD0301969093AD038093AC034FC080912D
:10677000420790914307892B09F03FC0F3018485BC
:10678000F101068510E00F701070000F111F000F4F
:10679000111F90E0807F90709595879595958795CE
:1067A000080F191F025F1F4FF301648175818681F5
:1067B00097810E94344E60934607709347078093F9
:1067C0004807909349075092450740924407020DAD
:1067D000131DAE01B8018AE497E00E949D77D09323
:1067E0004307C09342078091AE039091AF03019697
:1067F0009093AF038093AE0309C08091AA03909158
:10680000AB0301969093AB038093AA03F3018585B4
:10681000813009F08AC088E590E0489EE001499EF9
:10682000D00D589ED00D1124CE5CD94F888182376F
:10683000F9F464817581868197810E94344E6F5F7F
:106840007F4F8F4F9F4F6E877F87888B998B8EA14D
:106850009FA10E94AC4520E330E0281B390B810149
:1068600040E050E060E1C20116D91F8A1E8A1882FA
:106870008881813709F5F30164817581868197816B
:106880000E94344E6F5F7F4F8F4F9F4F6E877F8781
:10689000888B998B8EA19FA10E94AC4520E330E0AC
:1068A000281B390B810140E050E060E1C201F3D8C0
:1068B0001F8A1E8A188222C088818031F9F4F30170
:1068C00060857185828593850E94344E6F5F7F4F0E
:1068D0008F4F9F4F6A877B878C879D878EA19FA153
:1068E0000E94AC4520E330E0281B390B810140E0D9
:1068F00050E061E1C201CFD882E7888388E590E06B
:10690000489EF001499EF00D589EF00D1124EE5C5A
:10691000F94F82859385A485B5850196A11DB11D8A
:1069200082879387A487B58792C0F30185858131DB
:1069300009F058C088E590E0489EE001499ED00DDE
:10694000589ED00D1124CE5CD94F8881813741F5F6
:1069500064817581868197810E94344E6F5F7F4F7D
:106960008F4F9F4F6E877F87888B998BF301608550
:106970007185828593850E94344E6A877B878C87D8
:106980009D878EA19FA10E94AC4520E330E0281B8B
:10699000390B810140E050E060E1C2017CD83DC08C
:1069A0008881803109F053C0F3016481758186814B
:1069B00097810E94344E6F5F7F4F8F4F9F4F6E873E
:1069C0007F87888B998B8EA19FA10E94AC4520E385
:1069D00030E0281B390B810140E050E061E1C20149
:1069E0005AD820C0F3018585803189F588E590E08B
:1069F000489EE001499ED00D589ED00D1124CE5CDA
:106A0000D94F8881843021F48FE0888319821FC098
:106A10008881823721F41F8A1E8A188218C08881D3
:106A2000813719F482E7888312C0EA84FB840C85DD
:106A30001D85F30160857185828593850E94344EA2
:106A4000E616F7060807190711F41D8A1C8AE2E109
:106A5000CDB7DEB70C9403760F931F93CF93DF93DC
:106A600062E086E591E30E9484171092430710923A
:106A700042070E94FC2AC0E0D0E088E590E0C89F71
:106A80008001C99F100DD89F100D112460E370E0A4
:106A9000C801865A994F0E9481450E5C194FF80132
:106AA00097A386A3178A168A1082CE0194DA2196BC
:106AB000C330D10511F7DF91CF911F910F91089548
:106AC000AC01FB0188E090E095878487DB0120E042
:106AD00030E0F901E35DFE4F8081FD018683FA011C
:106AE000E20FF31F80818D932F5F3F4F26303105DA
:106AF00081F708951F9380913301813061F41FB7AE
:106B0000F8941092330182E090E00E9403130E94F7
:106B1000FC2A1FBF13C08091B0039091B103A091D4
:106B2000B203B091B3030196A11DB11D8093B003D0
:106B30009093B103A093B203B093B3031F91089550
:106B40001F9380913301882369F41FB7F89481E083
:106B5000809333010E94F92A82E090E00E9443135F
:106B60001FBF13C08091B0039091B103A091B203F5
:106B7000B091B3030196A11DB11D8093B003909312
:106B8000B103A093B203B093B3031F910895EF92A2
:106B9000FF920F931F9320918A0730918B074091AA
:106BA0008C0750918D072F5F3F4F4F4F5F4F2093C2
:106BB0008A0730938B0740938C0750938D077C0195
:106BC0000027F7FC0095102F20918E0730918F073A
:106BD00040919007509191072E0D3F1D401F511F6E
:106BE00020938E0730938F0740939007509391071F
:106BF0000E949F1C1F910F91FF90EF9008950C949D
:106C0000B01D0895A8E5B2E0E8E0F6E30C94F7754E
:106C10000E94F61C8DE291E00E945B1CBE016F5F3A
:106C20007F4F88E592E0EBDF892BC1F744E256E322
:106C300060E070E082E090E00E9411135BDFE2E030
:106C4000C85ADD4F0C941376A8E5B2E0EAE2F6E309
:106C50000C94F3757E010894E11CF11CB70188E5E2
:106C600092E0CDDF8C01892B09F43EC080918A0728
:106C700090918B07A0918C07B0918D070196A11D73
:106C8000B11D80938A0790938B07A0938C07B093D4
:106C90008D079801442737FD4095542F80918E072A
:106CA00090918F07A0919007B0919107820F931F49
:106CB000A41FB51F80938E0790938F07A093900712
:106CC000B09391078D859E850E94304E28E08030DC
:106CD000920739F08650984039F4B701C8018CD03A
:106CE00003C0B701C801FED2E6E0C85ADD4F0C94DC
:106CF0000F7680919C07882319F0815080939C0720
:106D00008091A707882319F081508093A7070895E1
:106D10000F931F93CF93DF93EC01890102971CF02F
:106D200080E090E034C08BE090E0C89F9001C99F64
:106D3000300DD89F300D1124F901EE56F84F8081A7
:106D40009181A281B381FB0180839183A283B3836C
:106D5000D901AA56B84F20E030E0FA01E20FF31F44
:106D60008D9180832F5F3F4F26303105B1F78BE047
:106D700090E0C89FF001C99FF00DD89FF00D11243D
:106D8000EE56F84F8285F801808381E090E0DF9134
:106D9000CF911F910F9108950F931F93FC018B01C9
:106DA000858190E09F938F93848190E09F938F9350
:106DB000838190E09F938F93828190E09F938F9344
:106DC000818190E09F938F93808190E09F938F9338
:106DD00082EB90E09F938F937F936F930E946478F0
:106DE0008DB79EB740960FB6F8949EBF0FBE8DBF6D
:106DF000C8011F910F910895EF92FF920F931F9377
:106E0000CF93DF937C018B01EB012E968E819F81C6
:106E10000E94304E8130910521F0029709F44FC055
:106E200074C0288D398D4A8D5B8D8091340190918D
:106E30003501A0913601B0913701281739074A076B
:106E40005B0709F062C082E090E00E94304E9F83B1
:106E50008E83FE0190E08085828B9F5F31969A3011
:106E6000D1F780912D01888780912E0189878091AB
:106E70002F018A87809130018B87809131018C8727
:106E8000809132018D878091340190913501A091DC
:106E90003601B09137018E879F87A88BB98BF80197
:106EA000ADE2B1E0868180838D918683319681E069
:106EB000A333B807B9F7B801C70169DE26C02E852C
:106EC0003F8548895989E2E9F7E080819181A28173
:106ED000B38182179307A407B50791F42083318308
:106EE000428353838EE18287888584838985858365
:106EF0008A8586838B8587838C8580878D8581872E
:106F00003B9687E0E83AF80701F7E6E0CDB7DEB751
:106F10000C940F76A0E0B0E0E0E9F7E30C94E9759B
:106F20006B017C014A014DB65EB630919C0733235C
:106F300081F08091920790919307A0919407B0916E
:106F400095078C159D05AE05BF0519F420E030E0CE
:106F500013C02091A707222339F180919D079091BA
:106F60009E07A0919F07B091A0078C159D05AE05C7
:106F7000BF05D1F421E030E08BE090E0289FD00104
:106F8000299FB00D389FB00D1124AA56B84F20E0AC
:106F900030E0F401E20FF31F8D9180832F5F3F4FAC
:106FA00026303105B1F7C6C0332319F420E030E0B4
:106FB00007C0222319F06624772412C021E030E0B4
:106FC0008BE090E0289FF001299FF00D389FF00D95
:106FD0001124EE56F84FC082D182E282F382390149
:106FE0008DB79EB78A970FB6F8949EBF0FBE8DBF20
:106FF000ADB6BEB60894A11CB11C0DB71EB7015F9B
:107000001F4F81E090E00E94304EF8019183808311
:1070100080E098E00E94304EF8019383828386E0FE
:10702000848384E0858381E090E00E94304EF80103
:1070300097838683128A138A148A158A168A178A76
:10704000C08ED18EE28EF38E80912D01808780914B
:107050002E01818780912F01828780913001838763
:10706000809131018487809132018587809134013C
:1070700090913501A0913601B091370186879787AD
:10708000A08BB18BADE2B1E0F5018FEF80838D91E4
:107090008683319681E0A333B807B9F786E098E09C
:1070A0000E94304EF50195878487B5018AE290E011
:1070B0006EDD0E944717E82EFF2441E064E670E091
:1070C000C7010E9423178BE090E0689E9001699EA3
:1070D000300D789E300D1124F901EE56F84F82855F
:1070E000882399F0D901AA56B84F20E030E0F40186
:1070F000E20FF31F8D9180832F5F3F4F26303105C4
:10710000B1F7C7010E94C71315C0C7010E94091734
:10711000892B31F4C7010E94C71381E090E00CC0B5
:10712000C7010E940917C29771F6B5018AE290E083
:107130002EDDC9CF80E090E00FB6F8945EBE0FBEA2
:107140004DBEE0E10C94057610929C071092A707C3
:1071500062E089E796E30C9484170F931F938A01EA
:10716000292F30E03F932F93282F30E03F932F9328
:10717000272F30E03F932F9370E07F936F9380ED44
:1071800090E09F938F935F934F930E9464788DB7A5
:107190009EB70C960FB6F8949EBF0FBE8DBFC80168
:1071A0001F910F910895A0E0B0E0E9EDF8E30C9491
:1071B000EB753C010E94C1774C01C0E0D0E0AA24ED
:1071C000BB2460E070E080E090E023C0CC24D62EA9
:1071D000E72EF82E83010C0F1D1FC8010E941E7799
:1071E0009C01442737FD4095542FF80180818E3251
:1071F00021F40894A11CB11C05C021963196C81534
:10720000D905A1F7C701B601622B732B842B952BEF
:107210002196C815D90528F023E0A216B10431F053
:1072200008C024E0A216B10488F203C00E94344EC4
:1072300004C060E070E080E090E0EEE0CDB7DEB743
:107240000C9407769F92AF92BF92CF92DF92EF920B
:10725000FF920F931F935B016C01942EC90178017B
:10726000025F1F4F25E4F7012687F801118244963B
:107270000E94304EF801938382838CEA9DE19583CE
:10728000848380E4868317828087918613861286A2
:107290008091340190913501A0913601B091370170
:1072A00084879587A687B787A08AB18AC28AD38A3E
:1072B000F701668570E06F707070660F771F660F5C
:1072C000771FC8015ED70E94304EF80193878287EE
:1072D0001F910F91FF90EF90DF90CF90BF90AF90F4
:1072E0009F900895CF93DF93EC01FB013E9681853B
:1072F0008630C9F0813159F1813061F520893189B9
:10730000428953898091340190913501A0913601D1
:10731000B0913701281739074A075B07D9F4CE0126
:107320000E943D2717C02089318942895389809165
:10733000340190913501A0913601B09137012817A1
:1073400039074A075B0731F4CE012AD803C0CE01C2
:107350000E945029DF91CF9108951F93CF93DF931F
:10736000182FE901A0E0B0E0FE01EA0FFB1F8081C9
:107370008F3F69F0CD010196FE01E80FF91F2081D2
:10738000DC011196A20FB11DA036B1056CF31533C7
:1073900091F0163338F4123309F456C0133309F45C
:1073A00053C0B0C0173309F454C01733A8F01D33CD
:1073B00009F46BC0A7C0FE01EA0FFB1F1083CD01CB
:1073C0000196FE01E80FF91F21E020830196FE01DE
:1073D000E80FF91F408394C0FE01EA0FFB1F86E30C
:1073E00080839D012F5F3F4FFE01E20FF31F84E07A
:1073F00080832F5F3F4FFE01E20FF31F40832F5F1B
:107400003F4FFE01E20FF31FBB2777FDBA95A72F71
:10741000962F852F80832F5F3F4FFE01E20FF31FD2
:10742000CB01BB2797FDB095AB2F80832F5F3F4FDC
:10743000FE01E20FF31F872FBB2787FDB0959B2F1F
:10744000AB2F8083D9015DC0FE01EA0FFB1F1083C3
:10745000C8CFFE01EA0FFB1F1083CD010196FE018C
:10746000E80FF91F33E030830196FE01E80FF91FA2
:1074700021E020830196FE01E80FF91F3083019679
:10748000FE01E80FF91F26E03AC0FE01EA0FFB1FDC
:107490001083CD010196FE01E80FF91F27E020833C
:1074A0000196FE01E80FF91F21E020830196FE01FD
:1074B000E80FF91F20912D0120830196FE01E80FAE
:1074C000F91F20912E0120830196FE01E80FF91F7C
:1074D00020912F0120830196FE01E80FF91F2091D2
:1074E000300120830196FE01E80FF91F2091310140
:1074F00020830196FE01E80FF91F209132012083BD
:10750000DC011196CA0FDB1F8FEF8883CD01019636
:10751000DF91CF911F910895CF93DF93EC0181E02C
:107520008883898386E08A831B8244E050E06FE28F
:1075300071E0CE0104960E949D77198618861B86FD
:107540001A861C861D861E861F86188A198A1A8A24
:107550001B8A1C8A1D8A1E8A1F8A188E198E1A8EF3
:107560001B8E80912D018C8F80912E018D8F8091AB
:107570002F018E8F809130018F8F8091310188A3F0
:107580008091320189A3FE01BC9680E090E01192C7
:10759000019680349105D9F7FE01E459FF4F80E050
:1075A00090E01192019680389105D9F7C451DF4FD0
:1075B00083E692E8A3E5B3E688839983AA83BB8335
:1075C000CC5ED040FE01E051FF4F80E090E0119290
:1075D000019680369105D9F7C051DF4F8FEF888330
:1075E000DF91CF910895A0E0B0E0E9EFFAE30C94C9
:1075F000F2757C018B0120E030E0DD24F801E20F20
:10760000F31FE081EF3F09F45CC0E9012196E63009
:1076100011F1E73028F4E13051F0E33091F044C04B
:10762000E533C9F1E63359F1E333F9F03DC0B80170
:107630006F5F7F4F6C0F7D1F44E050E0C7010896DD
:1076400027C0B8016F5F7F4F6C0F7D1F44E050E093
:10765000C70104961DC0B8016F5F7F4F6C0F7D1F7F
:1076600044E050E0C7010C9613C0B8016F5F7F4F34
:107670006C0F7D1F44E050E0C701449609C0B8017B
:107680006F5F7F4F6C0F7D1F44E050E0C701409655
:107690000E949D7709C0FE01E00FF11FD1809E017D
:1076A0002F5F3F4F808107C0F801EC0FFD1F8081E5
:1076B0009E012F5F3F4F280F311D203631050CF4FE
:1076C0009DCF8D2D90E0E7E0CDB7DEB70C940E7620
:1076D000A0E0B0E0EEE6FBE30C94EF755C018B01FB
:1076E0006A01CB0119DFB0EFEB2EF12CE00EF11E99
:1076F000970143E050E060E070E085E32EDEF601A4
:107700004089518962897389970186E326DEF601F3
:107710004489558966897789970183E31EDEF601DE
:107720004081518162817381970182E316DE970166
:1077300040E050E060E070E08DE30FDE970140E054
:1077400050E060E070E087E308DEA80160E571E0EA
:10775000C5010E94E1290E944717EC01FFEF8F3F0E
:107760009F07F1F041E068EE73E00E942317C50126
:107770000E94A827809749F4CE010E94C713B70141
:10778000C60131DF853079F41EC0CE010E94091791
:10779000892B69F7CE010E94C713C5010E94F92702
:1077A0008FEF9FEF43C090E09F938F9388EF90E01F
:1077B0009F938F930E9441788FEF9FEF0F900F90D0
:1077C0000F900F9033C0F60180819181A281B38127
:1077D0008093340190933501A0933601B093370123
:1077E00080859185A285B385809338019093390176
:1077F000A0933A01B0933B0184819581A681B78122
:1078000080933C0190933D01A0933E01B0933F01D2
:1078100084859585A685B785809340019093410125
:10782000A0934201B093430180E090E0EAE0CDB73D
:10783000DEB70C940B76A0E0B0E0E1E2FCE30C9440
:10784000EF756C017B015A01CB0166DE87010051A7
:107850001F4F980141E050E060E070E085E37DDD7E
:1078600098014FEF5FEF6FE070E083E376DD980102
:1078700040E050E060E070E08DE36FDD980140E0B3
:1078800050E060E070E087E368DDA70160E571E04B
:10789000C6010E94E1290E944717EC018FEFCF3FFC
:1078A000D807F9F041E068EE73E0CE010E9423179B
:1078B000C6010E94A827809749F4CE010E94C713F1
:1078C000B801C50190DE823079F41EC0CE010E945D
:1078D0000917892B69F7CE010E94C713C6010E94C0
:1078E000F9278FEF9FEF1FC090E09F938F938CED50
:1078F00090E09F938F930E9441788FEF9FEF0F90BE
:107900000F900F900F900FC0F70180899189A28985
:10791000B389F50180839183A283B383C6010E945A
:10792000DB2780E090E0EAE0CDB7DEB70C940B7681
:107930004F925F926F927F928F929F92AF92BF927F
:10794000DF92EF92FF920F931F93CF93DF93CDB708
:10795000DEB74DB65EB68090340190903501A090B0
:107960003601B09037011092340110923501109217
:107970003601109237018DB79EB748970FB6F8942D
:107980009EBF0FBE8DBF6DB67EB60894611C711C84
:10799000805591400FB6F8949EBF0FBE8DBFEDB6D7
:1079A000FEB60894E11CF11C870120E531E043E4B8
:1079B00050E06FEF7FEF8FEF9FEF0E94432A8C0123
:1079C0009FEF0F3F1907C9F08AE0D82EA301B70136
:1079D000C80131DFDD2031F0DA9421F08F5F9F4F55
:1079E000A9F30EC08F5F9F4F59F48092340190929B
:1079F0003501A0923601B09237018FEF9FEF0CC096
:107A0000A301B701C80164DE8F5F9F4F71F3C80106
:107A10000E94F92780E090E00FB6F8945EBE0FBE9A
:107A20004DBEDF91CF911F910F91FF90EF90DF90AE
:107A3000BF90AF909F908F907F906F905F904F908E
:107A40000895AAE1B0E0E7E2FDE30C94F075B22EF0
:107A5000611571058105910579F44115510509F408
:107A600070C0CA01A9D06F3F2FEF72072FEF8207B6
:107A70002FEF920709F465C07E010894E11CF11C08
:107A8000870124E030E045E250E00E94432A6C0187
:107A90008FEFC8168FEFD80609F453C0A70160E036
:107AA00070E0C6010E94E1290E9447177C012FEF78
:107AB0008F3F920709F445C041E064EF71E00E94F6
:107AC0002317C6010E94A827809761F5C7010E946D
:107AD0000917892B39F1C6010E94C22704973CF18E
:107AE000FE013496DE01159680818D933197EC1757
:107AF000FD07D1F78E01075F1F4FC8010E94F816DE
:107B00008D819E81AF81B8858F8B988FA98FBA8F19
:107B1000BA8AC8010E94E313C8010E94E71600E078
:107B200010E007C0C7010E940917892B51F60FEF1B
:107B30001FEFC7010E94C713C6010E94F927C801A1
:107B400002C08FEF9FEFE9E06A960C940C76EF92FB
:107B5000FF920F931F93CF93DF938C017B010E94C1
:107B6000C1779C0121503040D701A80FB91FE8010F
:107B7000C20FD31F60E070E00EC048814E3221F486
:107B80006C9360E070E003C04C936F5F7F4F2150B7
:107B9000304011972197F901319637FFEECFEE0D66
:107BA000FF1D6083E80EF91EF70111820196E6E0E1
:107BB000CDB7DEB70C940F76A0E0B0E0E2EEFDE3C7
:107BC0000C94E9758C014DB65EB68DB79EB7825D9B
:107BD00090400FB6F8949EBF0FBE8DBFCDB6DEB6F7
:107BE0000894C11CD11C8DEC9AE1EDB7FEB79283CD
:107BF000818380E091E00E94304EF601938382837E
:107C000081E090E00E94304EF601958384831782D4
:107C1000168211861086138612869CE0692E712CBE
:107C20006C0C7D1CB301C80192DF7C01FC01EC0DE2
:107C3000FD1D158681E086871786808B6091400147
:107C4000709141018091420190914301860122EDA2
:107C500030E045E350E00E94432A5C018F5F9F4F74
:107C600009F456C085E0882E912C8E0C9F1C81E172
:107C700090E0E80EF91EA601B701C5010E94E129B6
:107C80000E9447178C019FEF0F3F190709F440C06E
:107C900041E068EC70E0C8010E942317C5010E9412
:107CA000A827809779F4C8010E94C713C5010E94D4
:107CB000F927F6018281938147D28F709070892BCA
:107CC00039F50CC0C8010E940917892B39F7C80182
:107CD0000E94C713C5010E94F9271AC08301080D2D
:107CE000191DF801828193812FD2019759F0F80173
:107CF0008285938529D29401245F3F4F280F391F35
:107D00004901ECCFF801648575858685978504C0A7
:107D10006FEF7FEF8FEF9FEF0FB6F8945EBE0FBE51
:107D20004DBEE0E10C940576A2E3B0E0EAE9FEE3A3
:107D30000C94EB7581E393E0C8D38F5F9F4F71F094
:107D40008E010D5E1F4FB8018DE293E078D54CE0B7
:107D500050E06DE271E0C8010E94BD480E94023609
:107D6000609032017724809031019924A0903001F5
:107D7000BB24C0902F01DD24E0902E01FF24009150
:107D80002D0110E00E94DC1C7F926F929F928F92D7
:107D9000BF92AF92DF92CF92FF92EF921F930F9319
:107DA0009F938F9381EE92E09F938F930E944178EF
:107DB0000E946D1D84ED92E09F938F930E94417805
:107DC0008DB79EB742960FB6F8949EBF0FBE8DBF7B
:107DD0000E948B1D8823E1F786EC92E09F938F939E
:107DE0000E944178B1D98DEA92E09F938F930E94CF
:107DF00041780E94272883E892E09F938F930E9406
:107E000041780E942C3588E592E09F938F930E94E1
:107E1000417883E592E059D32DB73EB7285F3F4FB5
:107E20000FB6F8943EBF0FBE2DBF8F5F9F4F71F40A
:107E300087E591E09F938F930E94417879DD0F90C1
:107E40000F90892BE9F08AE391E01CC08E010D5E52
:107E50001F4FB8018EE492E0F2D46BE472E0C801E7
:107E60000E947777892B09F053C087E591E09F93B3
:107E70008F930E9441785CDD0F900F90892B39F42D
:107E800085E291E09F938F930E9441783EC08AE300
:107E900091E09F938F930E944178B80184E191E033
:107EA000CED4C80180D9609334017093350180939A
:107EB000360190933701B80187E191E0C0D4C80141
:107EC00072D9609338017093390180933A0190938D
:107ED0003B01B80180E291E0B2D4C80164D960935B
:107EE0003C0170933D0180933E0190933F01B801A6
:107EF0008CE191E0A4D4C80156D9609340017093FD
:107F0000410180934201909343010F900F9044C030
:107F1000B80184E191E093D48F5F9F4F51F0C80185
:107F200042D9609334017093350180933601909368
:107F30003701B80187E191E082D48F5F9F4F51F004
:107F4000C80131D9609338017093390180933A01A7
:107F500090933B01B80180E291E071D48F5F9F4F15
:107F600051F0C80120D960933C0170933D0180938A
:107F70003E0190933F01B8018CE191E060D48F5FA6
:107F80009F4F51F0C8010FD9609340017093410198
:107F9000809342019093430183E1E82EF12CEC0E93
:107FA000FD1E6091340170913501809136019091F0
:107FB0003701A701D2D89F938F9388E392E09F93D4
:107FC0008F930E94417860913801709139018091BE
:107FD0003A0190913B01A701C0D89F938F9385E20E
:107FE00092E09F938F930E94417860913C01709141
:107FF0003D0180913E0190913F01A701AED89F9332
:108000008F9382E192E09F938F930E9441786091D9
:108010004001709141018091420190914301A7017B
:108020009CD89F938F938FEF91E09F938F930E94A3
:108030004178B7018BEF91E002D42DB73EB7205FB6
:108040003F4F0FB6F8943EBF0FBE2DBF8F5F9F4FBF
:1080500009F456C068EF71E0C7010E947777892B59
:1080600009F04EC084ED91E09F938F930E94417878
:10807000B7018CEC91E0E3D30F900F908F5F9F4F8F
:10808000B9F1C7010E941E778C01B70182EC91E023
:10809000D6D3202FA70160E070E080E090E0D1DC33
:1080A000892B19F5CE0101960E94F81689812A8143
:1080B0004B816C8190E09F938F9330E03F932F939F
:1080C00050E05F934F9370E07F936F9385EA91E068
:1080D0009F938F930E9441788DB79EB70A960FB6F3
:1080E000F8949EBF0FBE8DBF0BC083E991E002C024
:1080F00081E891E09F938F930E9441780F900F90B9
:1081000060E070E084E0BFD060913401709135018F
:108110008091360190913701AE014D5E5F4F1DD8C1
:108120009F938F938CE791E09F938F930E94417868
:1081300060E070E081E0A7D00F900F900F900F905B
:10814000EEE0E2960C9407769C01922F8827232F6D
:108150003327822B932B0895282F30E074E0369537
:1081600027957A95E1F7A90163E0440F551F6A95B9
:10817000E1F7220F331F240F351F8F70820F90E01D
:108180000895EF92FF920F931F93FC01EE24FF24BA
:10819000870112C080812181329690E0982F882734
:1081A000820F911D80959095A0E0B0E0E80EF91E39
:1081B0000A1F1B1F62507040623071055CF761300E
:1081C000710561F4808190E0982F882780959095C3
:1081D000A0E0B0E0E80EF91E0A1F1B1F980144271B
:1081E00055278FEF9FEFA0E0B0E0E822F9220A23A5
:1081F0001B232E0D3F1D401F511FCA01AA27BB275D
:1082000040705070820F931FA41FB51FA070B070F4
:108210001F910F91FF90EF90089584E491E0909367
:10822000B6088093B5089093B8088093B7088FEF8D
:108230008093A80784EB93E09093AC078093AB07FF
:108240001092AE071092AD0708958091A807823072
:10825000C9F48091AD079091AE07892B79F06091B8
:10826000AD077091AE078091A9079091AA07409140
:10827000AB075091AC0720E00E94BC301092AE07D3
:108280001092AD070895FF920F931F93F82E8B0164
:10829000DCDFF092A8071093AA070093A9071092B9
:1082A000AE071092AD071F910F91FF9008950F93A5
:1082B0001F938C01CADF47E050E0B80188EA97E0DD
:1082C0000E949D771F910F9108950F931F938C012A
:1082D000BCDF47E050E068EA77E0C8010E949D7784
:1082E0001F910F9108958091A807813019F0823075
:1082F00089F021C08091A9079091AA070E94D31804
:1083000018161906C4F48091A9079091AA070E9433
:10831000C1180FC08091A9079091AA070E94B42BA1
:108320001816190644F48091A9079091AA070E9493
:108330008F2E90E008958FEF9FEF08951F93182FD1
:108340008091A807823061F0843011F1813019F5F5
:108350008091A9079091AA07612F0E94AE181BC0B7
:108360008091AD079091AE07809709F46EDF809100
:10837000AD079091AE07E091AB07F091AC07E80F25
:10838000F91F108301969093AE078093AD0703C049
:10839000812F0E94542580E090E01F9108959093D2
:1083A000D5038093D40308950F931F93CF93DF9346
:1083B00080915401909155018F5F9F4F19F4CFEF39
:1083C000DFEF15C00091E0031091E103C0E0D0E0C1
:1083D0000BC080915201909153018C0F9D1F0E9400
:1083E000817A882321F02196C017D10794F3CE011A
:1083F000DF91CF911F910F910895AEE1B0E0E3E0DE
:10840000F2E40C94EF755C010E94C177CC24DD246A
:108410004CC08091520190915301800F911F0E9496
:10842000817A282FCE010196FC01EE0DFF1D2083DD
:108430002D3311F0222339F41082B5010E94B87750
:10844000892BD9F120C00894E11CF11C0F5F1F4F4C
:10845000ABDF08171907ECF216C08091520190911A
:108460005301800F911F0E94817A8D3081F080919D
:10847000520190915301800F911F0E94817A8823AD
:1084800031F00F5F1F4F90DF0817190734F3809109
:10849000520190915301800F911F0E94817A88238D
:1084A00071F068010894C11CD11C7EDFC816D90682
:1084B00034F48601EE24FF24CBCFC60102C08FEF37
:1084C0009FEFEAE06E960C940B76A0E0B0E0EBE64E
:1084D000F2E40C94F1757C01CDB6DEB60E9487778C
:1084E00001962DB73EB7281B390B0FB6F8943EBF47
:1084F0000FBE2DBF0DB71EB70F5F1F4FB701C801CD
:108500000E948077C80179DF0FB6F894DEBE0FBEF7
:10851000CDBEE8E00C940D76AF92BF92CF92DF9281
:10852000FF920F931F93CF93DF936C018091D4033D
:108530009091D503019709F458C036DF5C01C6015C
:108540005CDFEC018FEFCF3FD80719F48FEF9FEF7F
:108550004EC000E010E08DE0F82E11C08091520175
:10856000909153018C0F9D1F0E94817AF82E8DE00F
:10857000F81641F0FF2031F00F5F1F4F2196CA150A
:10858000DB0564F3C60139DFEC018DE0F81619F55F
:108590000F5F1F4F14C080915201909153018C0FB7
:1085A0009D1F800F911F0E94817A682F8091520138
:1085B000909153018C0F9D1F0E94897A2196F4DEC1
:1085C000C817D90744F3809152019091530160E09C
:1085D0008C0F9D1F08C080915201909153018C0F08
:1085E0009D1F60E001970E94897A81E090E0DF9111
:1085F000CF911F910F91FF90DF90CF90BF90AF90E0
:108600000895A0E0B0E0E7E0F3E40C94F1757C019C
:108610006B01F3DE8F5F9F4F19F08FEF9FEF5EC00E
:108620008091D4039091D503019709F455C0BCDE25
:10863000EC01892B19F400E010E01AC0809152017E
:10864000909153018C0F9D1F21966DE00E94897AB5
:10865000F2CFF701E00FF11F6081809152019091FC
:1086600053018C0F9D1FE9010E94897A0F5F1F4FF4
:10867000C7010E94C1779E012F5F3F4F081719075E
:1086800040F3809152019091530189016DE38C0F69
:108690009D1F0E94897AC0E0D0E00FC0F601EC0F68
:1086A000FD1F60818091520190915301800F911FB5
:1086B0000F5F1F4F0E94897A2196C6010E94C177E1
:1086C000C817D90758F3809152019091530160E087
:1086D000800F911F0E94897A81E090E0E8E0CDB799
:1086E000DEB70C940D760F931F93CF93DF93EC01BD
:1086F0008B0183DE8F5F9F4F11F0CE010DDFB8013C
:10870000CE017FDF81E090E0DF91CF911F910F914B
:108710000895A0E0B0E0EFE8F3E40C94EF757C017D
:108720006B01ADB6BEB60E94877701962DB73EB7F6
:10873000281B390B0FB6F8943EBF0FBE2DBF0DB7E7
:108740001EB70F5F1F4FB701C8010E948077B601A7
:10875000C801C9DF0FB6F894BEBE0FBEADBEEAE0D9
:108760000C940B76AEE1B0E0E8EBF3E40C94EF751B
:108770007C015B010E94C177C7013FDE8C018FEF56
:108780000F3F180709F455C0CC24DD2418C0809190
:10879000520190915301800F911F0E94817AFE0136
:1087A0003196EC0DFD1D80838D3311F0882311F47B
:1087B000108209C00894C11CD11C0F5F1F4FF4DD4B
:1087C0000817190724F38091520190915301800FEB
:1087D000911F0E94817A8D3361F5B701CE01019618
:1087E0000E94B877892B29F50F5F1F4FEE24FF24D5
:1087F00015C08091520190915301800F911F0E94EA
:10880000817AF501EE0DFF1D80838D3059F08823AC
:1088100049F00894E11CF11C0F5F1F4FC5DD0817DC
:1088200019073CF3EA0CFB1CF701108281E090E091
:1088300002C08FEF9FEFEAE06E960C940B76A0E0FB
:10884000B0E0E5E2F4E40C94EF757C016B01ADB6A9
:10885000BEB60E94877701962DB73EB7281B390B0D
:108860000FB6F8943EBF0FBE2DBF0DB71EB70F5FFA
:108870001F4FB701C8010E948077B601C80172DF9F
:108880000FB6F894BEBE0FBEADBEEAE00C940B76F8
:10889000CF93DF934AE050E065E373E086ED93E029
:1088A0000E946E7783EF97E09093E1038093E0035B
:1088B000C0E0D0E0FE01EA52FC4F6081CE010E9490
:1088C000897A2196CC30D105A9F78DE090E090937C
:1088D000530180935201809152019091530160E0C5
:1088E0000E94897ADF91CF9108950F931F93CF93C0
:1088F000DF93009152011091530156DD2091E00366
:108900003091E1031F930F939F938F933F932F9386
:1089100087E493E09F938F930E944178C0E0D0E07A
:108920008DB79EB708960FB6F8949EBF0FBE8DBF49
:1089300043C080915201909153018C0F9D1F0E9462
:10894000817A863261F010C080915201909153017A
:108950008C0F9D1F0E94817A8D3069F1219624DD54
:10896000C817D9078CF327C0809152019091530109
:108970008C0F9D1F0E94817A90E09F938F9384E4D7
:1089800093E09F938F930E94417880915201909140
:1089900053018C0F9D1F0E94817A0F900F900F90B2
:1089A0000F908D3041F482E493E09F938F930E9467
:1089B00041780F900F902196F7DCC817D9070CF477
:1089C000B8CF8FE393E09F938F930E9441780F90ED
:1089D0000F90DF91CF911F910F910895A0E2B0E029
:1089E000E4EFF4E40C94F57500E010E04AE050E0A8
:1089F000B80186ED93E00E94717A4AE050E060E0B1
:108A000071E086ED93E00E949077892BA9F44CE009
:108A100050E0B80186ED93E00E94717A1093550101
:108A20000093540180915401909155010D969093BB
:108A300053018093520106C00F5F1F4F27E0033F91
:108A40001207A1F680915401909155018F5F9F4FBD
:108A500019F48FEF9FEF1EC08E010F5F1F4FB801FB
:108A60008CE893E0ECDE8F5F9F4F91F068E873E055
:108A7000C8010E947777892B29F41092D5031092B0
:108A8000D40306C081E090E09093D5038093D40393
:108A900080E090E0E4E0A0960C9411769FDF8F5F79
:108AA0009F4F11F4F5DE9ACF089588E190E028E019
:108AB0000FB6F894A895809360000FBE20936000D5
:108AC000FFCF8091E2038823D9F481E08093E20311
:108AD0001092B0071092AF071092BB071092BA071E
:108AE0001092C6071092C5071092D1071092D007B6
:108AF0001092DC071092DB071092E7071092E6074E
:108B00000895AC01EFEAF7E020E030E08081918148
:108B1000892BC9F48BE090E0289FF001299FF00D8C
:108B2000389FF00D1124E155F84F51834083738332
:108B300062831782168215821482118610868FEF47
:108B40008287C90108952F5F3F4F3B96263031053C
:108B5000E9F68FEF9FEF08959C0106978CF48BE068
:108B600090E0289FF001299FF00D389FF00D11240F
:108B7000E155F84F82858F3F19F4808591850895DE
:108B80008FEF9FEF0895CF93DF93FC0106979CF53D
:108B90008BE090E0E89FD001E99FB00DF89FB00D09
:108BA0001124A155B84FED018A858F3F21F5288505
:108BB00039858A819B8128173907E8F4ED91FC916A
:108BC00011978C819D81E80FF91F60838C819D81B5
:108BD00001969D838C832A813B818217930711F430
:108BE0001D821C82FD018085918501969187808779
:108BF00080E090E002C08FEF9FEFDF91CF9108956A
:108C0000CF93DF93FC01069774F58BE090E0E89F2B
:108C1000D001E99FB00DF89FB00D1124A155B84FB8
:108C2000ED018A858F3FF9F488859985892BD9F0E4
:108C30008E819F81ED91FC911197E80FF91FE081E2
:108C400001969F838E832A813B818217930711F4BB
:108C50001F821E82ED0188859985019799878887F3
:108C60008E2F90E002C080E090E0DF91CF910895D8
:108C70009C010697BCF48BE090E0289FF001299FAF
:108C8000F00D389FF00D1124E155F84F82858F3F8C
:108C900049F417821682158214821186108680E0AC
:108CA00090E008958FEF9FEF0895FC0106971CF068
:108CB0002FEF3FEF12C08BE090E09F01289FF00163
:108CC000299FF00D389FF00D1124E155F84F2281B6
:108CD000338180859185281B390BC9010895EF9256
:108CE000FF920F931F93CF93DF937C018B01BA0107
:108CF00006970CF06CC08BE090E0E89EE001E99EE6
:108D0000D00DF89ED00D1124C155D84F8A858F3FC4
:108D100009F05DC04A815B81888599859A01281B8D
:108D2000390B2017310708F452C02C813D81C8014E
:108D3000820F931F8417950718F040E050E032C06F
:108D400088819981A801820F931F0E949D778C8151
:108D50009D81800F911F9D838C8327C08BE090E0C5
:108D6000E89EE001E99ED00DF89ED00D1124C1557A
:108D7000D84FA881B9818C819D81A80FB91FFB01B3
:108D8000E40FF51F80818C938C819D8101969D83DA
:108D90008C832A813B818217930711F41D821C82E8
:108DA0004F5F5F4F40175107C9F68BE090E0E89E98
:108DB000F001E99EF00DF89EF00D1124E155F84FF9
:108DC00080859185800F911F9187808702C00FEF6A
:108DD0001FEFC801E6E0CDB7DEB70C940F760F9316
:108DE0001F93CF93DF9378946CDE80E090E00E9435
:108DF0009D1813DA60E070E081E045DA8CE394E0DE
:108E00009F938F930E94417887E394E09F938F9381
:108E10000E944178CAE9D3E0DF93CF930E94417862
:108E200080E394E09F938F930E944178DF93CF93E8
:108E30000E9441780E94BD178AE294E09F938F932D
:108E40000E944178DF93CF930E9441780E94B8211D
:108E500081E294E09F938F930E944178DF93CF93B8
:108E60000E94417862E08AE498E40E94841716DE4A
:108E70008AE194E09F938F930E944178DF93CF9390
:108E80000E9441780E94001383E194E09F938F93A6
:108E90000E944178DF93CF930E9441780E94612025
:108EA0008DE094E09F938F930E944178DF93CF935E
:108EB0000E94417889E094E09F938F930E944178CB
:108EC0002DB73EB7205E3F4F0FB6F8943EBF0FBEA2
:108ED0002DBF60EA76E881E090E00E94471F813074
:108EE000B9F40E9422209F938F938BEF93E09F937E
:108EF0008F930E944178DF93CF930E9441788DB782
:108F00009EB706960FB6F8949EBF0FBE8DBF08C0E1
:108F10008BEA93E09F938F930E9441780F900F907C
:108F20000E94832587EF93E09F938F930E9441785F
:108F3000CAE9D3E0DF93CF930E94417860E070E00C
:108F400084E0A1D989EE93E09F938F930E944178AA
:108F500060E070E081E097D90E94BA1B0E94E91B93
:108F600084EE93E09F938F930E944178DF93CF9399
:108F70000E9441780E94FB1980EE93E09F938F93AB
:108F80000E944178DF93CF930E94417889ED93E06E
:108F90009F938F930E9441780E944F1E2DB73EB73A
:108FA000205F3F4F0FB6F8943EBF0FBE2DBF882302
:108FB00029F08BEA93E09F938F9302C0DF93CF93C6
:108FC0000E9441780F900F900E94372783ED93E025
:108FD0009F938F930E944178CAE9D3E0DF93CF93A8
:108FE0000E9441788CEC93E09F938F930E9441788C
:108FF0000E9458242DB73EB72A5F3F4F0FB6F89412
:109000003EBF0FBE2DBF882391F0DF93CF930E9408
:10901000417881EC93E09F938F930E9441780E9466
:109020007B5A0F900F900F900F90892B29F08BEAAD
:1090300093E09F938F9302C0DF93CF930E94417878
:109040000F900F900E94C65A8BEB93E09F938F93E3
:109050000E9441780AE913E01F930F930E94417820
:109060001CD084EB93E09F938F930E9441781F93D1
:109070000F930E9441780E94943E8DB79EB7089648
:109080000FB6F8949EBF0FBE8DBFDF91CF911F9199
:109090000F91089580E00C94A42180E090E0FC0101
:1090A000EE0FFF1FEE0FFF1FEF50F84F11821082DF
:1090B00001968A30910599F70895AC0120E030E0DF
:1090C000F901EE0FFF1FEE0FFF1FEF50F84F8081E9
:1090D00091818417950781F080819181892B39F4E2
:1090E000518340837383628380E090E008952F5F13
:1090F0003F4F2A30310521F78FEF9FEF0895E09120
:10910000E303F091E403EE0FFF1FEE0FFF1FEF509C
:10911000F84F80819181892B21F41092E403109201
:10912000E303E091E303F091E403EE0FFF1FEE0F82
:10913000FF1FEF50F84F0190F081E02D09958091CD
:10914000E3039091E40301969093E4038093E30397
:109150000895982F80538A3070F0892F8156863079
:1091600010F4865F08C0892F8154863010F08FEF8D
:1091700002C0892F875390E00895A0E0B0E0E3ECAF
:10918000F8E40C94EF756C015B017A01EE0CFF1CA6
:10919000C0E0D0E02CC0CE15DF059CF5C0FD0FC0AF
:1091A000CE0162E070E00E9497758B010A0D1B1DD5
:1091B000822FCFDF8295807FF80180830EC0CE01A1
:1091C00062E070E00E9497758B010A0D1B1D822FD3
:1091D000C0DFF8019081980F90830894C11CD11CC6
:1091E000F60180818A33C9F38D32B9F32196F601F5
:1091F0002081222381F6CE15DF0519F480E090E06E
:1092000002C08FEF90E0EAE0CDB7DEB70C940B76AA
:10921000CF93DF93FC01EB0160E880309607A9F162
:1092200097FD02C04BE204C0F095E195FF4F4DE27F
:109230009F01307084E690E0BC01269FC001279F0B
:10924000900D369F900D112460E071E00E9497759B
:109250007F936F938F2F992787FD9A959F938F9375
:10926000842F90E09F938F938DEF96E09F938F9341
:10927000DF93CF930E9464788DB79EB70A960FB69E
:10928000F8949EBF0FBE8DBF0EC089EF96E09F93EE
:109290008F93DF93CF930E946478C0E0D0E00F906B
:1092A0000F900F900F90CE01DF91CF910895CF9343
:1092B000DF93EB0190E09F938F938AE494E09F9378
:1092C0008F937F936F930E946478BE01CE014ADA38
:1092D0002DB73EB72A5F3F4F0FB6F8943EBF0FBE83
:1092E0002DBF8F5F9F4F11F4C0E0D0E0CE01DF9122
:1092F000CF910895A8E0B0E0E0E8F9E40C94ED75B2
:109300004C01FC010AC0CF0101962B3329F41082D5
:109310007C015F01FC0111C0FC012081222399F72F
:10932000EE24FF24AA24BB2408C0CF0101962B33CE
:1093300019F410825C0104C0FC0120812223A9F7EA
:1093400063E177E0C4010E947777892B21F0C12C7B
:1093500020E8D22E0CC042E050E08E010F5F1F4F7C
:10936000B801C7010ADFC8010E943E206C016BE012
:1093700077E0C4010E947777892BD9F440E150E06F
:109380008E010F5F1F4FB801C701F7DEC8010E94B1
:10939000141F6C01805F9F4F61F4C8010E94141F6D
:1093A000EFEF803F9E0721F4C12C90E8D92E01C039
:1093B0006C0167E077E0C4010E947777892B19F48C
:1093C000C7016CD06C01E114F10431F00894E1089C
:1093D000F1088BE3F7018083A114B10431F0089404
:1093E000A108B1088BE3F5018083C601ECE0289663
:1093F0000C940976A0E4B0E0E0E0FAE40C94F57592
:109400008E010F5F1F4FB80152DF892B19F480E0E6
:1094100090E802C0C8016EDFE4E0C05CDF4F0C944E
:10942000117680915601909157012FEF8F3F92074F
:1094300069F445EE53E063E070E08FE790E10E944D
:109440004A28909357018093560108950E94A827B7
:10945000809719F58091E503CDDF9093E703809322
:10946000E60345EE53E063E070E080915601909191
:1094700057010E94E12980915601909157010E9465
:10948000F92745EE53E063E070E08FE790E10E943A
:109490004A2890935701809356010895A3E0B0E0C5
:1094A000E4E5FAE40C94EF757C01FC0101C031960F
:1094B00080818A3311F08823D1F7309709F48CC06A
:1094C00011928F01CF010E941E77898380E090E87E
:1094D0009B838A83C7010E94D3386115710581057A
:1094E000910521F0C7010E94D33803C0C7010E9433
:1094F000DC3D6B017C018FEFC8168FEFD8068FEF34
:10950000E8068FEFF80609F467C0015010408AE3BF
:10951000F80180835E010894A11CB11C850123E041
:1095200030E04FE750E1C701B6010E94432A7C01B9
:10953000FFEF8F3F9F0719F48FEF9FEF0DC0A5013D
:1095400063E070E00E94E1290E9447178C018FEFD1
:109550000F3F180721F4C7010E94F9273DC041E0E1
:1095600064EF71E0C8010E942317C7010E94A82779
:10957000809769F4C8010E940917892B41F0C7013F
:109580000E94C2270397F1F4CA80DB801EC0C80185
:109590000E940917892BB1F0C8010E940917C297D0
:1095A00031F4A50163E070E0C7010E94E129C80120
:1095B0000E94091764E670E00E948375892BA9F266
:1095C00030DFD3CFC12C40E8D42EC8010E94C7138E
:1095D000C7010E94F92703C0C12C30E8D32EC60171
:1095E000EAE023960C940B760F931F938B0102DF16
:1095F000B8010EDE1F910F910895AAE4B0E0E3E0F8
:10960000FBE40C94EC755C0180910A0190910B01D4
:109610009A83898328E0FE01339611922A95E9F70F
:109620009C878B878EE3FE013D9611928A95E9F720
:109630000E94895E8FE796E09F938F930E94417806
:109640006BE776E0C5010E94E65C0F900F90892BD6
:1096500049F167E776E0C5010E940E5DFC01EE0F5F
:10966000FF1FEA0DFB1DE654FF4F808191810E9490
:109670001E779F938F938AE494E09F938F938E013C
:10968000055F1F4F1F930F930E946478C8010E94CB
:109690008C422DB73EB72A5F3F4F0FB6F8943EBFBE
:1096A0000FBE2DBF882499249F928F928AE494E064
:1096B0009F938F93EBE0CE2ED12CCC0EDD1EDF924C
:1096C000CF920E946478B601C5010E94355D2DB726
:1096D0003EB72A5F3F4F0FB6F8943EBF0FBE2DBF77
:1096E000892B09F451C062E776E0C5010E940E5D46
:1096F000FC01EE0FFF1FEA0DFB1DE654FF4FE0805B
:10970000F1806AE676E0C5010E940E5DFC01EE0F75
:10971000FF1FEA0DFB1DE654FF4F0081118166E635
:1097200076E0C5010E940E5DFF92EF921F930F93AA
:10973000FC01EE0FFF1FEA0DFB1DE654FF4F808179
:1097400091819F938F938DE596E09F938F938E01E8
:10975000045F1F4FC6010E94C177800F911F9F9326
:109760008F930E946478C6010E94C177080F191F69
:10977000B801C6010E9473438DB79EB70A960FB613
:10978000F8949EBF0FBE8DBF782CB601882D8FDD5B
:10979000892B99F0D60101C0DF01FD0181918B3346
:1097A000D9F71C927F01DF0101C0DF01FD0181912A
:1097B0008B33D9F71C926F0102C01B8676018E0194
:1097C0000F5F1F4FB801872D0FDF9F928F929F92DF
:1097D0008F92DF92CF92FF92EF92CE010B969F93E2
:1097E0008F931F930F939F928F9283E694E09F93A2
:1097F0008F930E9441780894811C911C2DB73EB72D
:10980000205F3F4F0FB6F8943EBF0FBE2DBF38E02C
:109810008316910409F048CF8AE594E09F938F93D3
:109820000E9441780E94805E0F900F90EDE0C65B31
:10983000DF4F0C94087666E277E081E19AE43DDC44
:1098400067E177E08DEF9AE40C945E5ECF93DF934F
:10985000EC010E94C177FE01E80FF91F06C080816C
:109860008F3211F4119204C03197EC17FD07B9F74C
:10987000CF01DF91CF910895A6E5B0E0E2E4FCE4EA
:109880000C94EF758C015B01E1DF6C01081719077F
:1098900019F468E571E001C0B8018E010F5F1F4F38
:1098A000A8018091190890911A080E942659B801C0
:1098B0008091190890911A080E946A577C01892B9F
:1098C000C9F420C0B601C8010E94B877892B91F471
:1098D0009501442737FD4095542FFE01E15BFF4F72
:1098E00060817181828193810E94AA758901C7017B
:1098F0009AD40AC08E01045D1F4FB801C7016ED50E
:10990000882301F70FEF1FEFC7010E946057C801BE
:10991000EAE0CA5ADF4F0C940B76ACE5B0E0E3E91D
:10992000FCE40C94E7757C011A012B016D963FAFA6
:109930002EAF6D973801B8019FDFAA2797FDA0953C
:10994000BA2F281639064A065B061CF00FEF1FEFE8
:1099500088C0C7017BDF6C01E816F90619F468E5D9
:1099600071E001C0B7018E010B5F1F4FA80180910C
:10997000190890911A080E942659B8018091190877
:1099800090911A080E946A574C01892B89F464C08F
:10999000B601C8010E94B877892B51F4FE01ED5A37
:1099A000FF4FE080F18002811381C4013CD40CC0E0
:1099B0008E01005D1F4FB801C40110D5882341F707
:1099C000EE24EA94FE2C87015301CC24B7FCC0940A
:1099D000DC2CC801B701A60195010E94CC75611568
:1099E000710581059105C1F5BE01605D7F4F8091D4
:1099F000190890911A080E949A577C01892B61F1ED
:109A0000C601B501A20191010E94587569837A834C
:109A10008B839C8340E0BE016F5F7F4FC7010E9434
:109A2000E455882399F0A3016D966EAD7FAD6D97D7
:109A3000C70117D320E030E0892B11F421E030E09A
:109A40002615370519F000E010E002C00FEF1FEFF8
:109A5000C7010E94655702C00FEF1FEFC4010E94AB
:109A60006057C801E2E1C45ADF4F0C940376AEE5BB
:109A7000B0E0EDE3FDE40C94E7757C016F964CAF2C
:109A80005DAF6EAF7FAF6F9719012801B801F4DEAB
:109A9000AA2797FDA095BA2F6F962CAD3DAD4EAD80
:109AA0005FAD6F9782179307A407B5071CF40FEFFC
:109AB0001FEF96C0C701CADE6C01E816F90619F45B
:109AC00068E571E001C0B7018E010B5F1F4FA8016F
:109AD0008091190890911A080E942659B801809126
:109AE000190890911A080E946A573C01892B89F441
:109AF00072C0B601C8010E94B877892B51F4FE01EB
:109B0000ED5AFF4FE080F18002811381C3018BD3B6
:109B10000CC08E01005D1F4FB801C3015FD48823C4
:109B200041F7EE24EA94FE2C87015201CC24B7FCC5
:109B3000C094DC2CC801B701A60195010E94CC7528
:109B4000611571058105910509F045C0BE01605D93
:109B50007F4F8091190890911A080E949A574C01E2
:109B6000892BC9F1C601B5016F962CAD3DAD4EAD47
:109B70005FAD6F970E94587569837A838B839C834E
:109B8000E616F7060807190714F040E005C0198229
:109B90001A821B821C8242E0BE016F5F7F4FC401AC
:109BA0000E94E455882389F0A201B101C4010E94FA
:109BB0003B5620E030E0892B11F421E030E0241501
:109BC000350519F000E010E002C00FEF1FEFC401EF
:109BD0000E94655702C00FEF1FEFC3010E9460573C
:109BE000C801E2E1C25ADF4F0C940376A6E5B0E06B
:109BF000ECEFFDE40C94F3758C0128DE7C01081772
:109C0000190719F468E571E001C0B8018E010F5F12
:109C10001F4FA8018091190890911A080E94265997
:109C2000B8018091190890911A080E946A578C0116
:109C3000009751F0AE01445D5F4FB70190D6882385
:109C400019F0EE24FF2403C0EE24EA94FE2CC80190
:109C50000E946057C701E6E0CA5ADF4F0C940F76A6
:109C600089279827892708956927962769277827BC
:109C7000872778270895EF92FF920F931F93CF9332
:109C8000DF93EC017B016A897B896C5E7F4FC701A2
:109C9000F3DD2FEF8F3F920761F4C701A7DF0A8939
:109CA0001B890C5E1F4F9E0140E050E060E070E0B9
:109CB0000AC00A891B890C5E1F4FAC01662757FD3D
:109CC0006095762F9E01C701D2DE20E030E08F5FE5
:109CD0009F4F11F021E030E0C901E6E0CDB7DEB7DB
:109CE0000C940F76EF92FF920F931F93CF93DF9315
:109CF000EC017B016A897B896C5E7F4FC701BCDD0B
:109D00002FEF8F3F920719F480E090E015C0019784
:109D1000AC01662757FD6095762F0A891B890C5E7A
:109D20001F4F9E01C701A3DE20E030E08F5F9F4FF1
:109D300011F021E030E0C901E6E0CDB7DEB70C94C8
:109D40000F76EF92FF920F931F93CF93DF93EC0167
:109D50007B016A897B896C5E7F4FC7018DDD2FEFA8
:109D60008F3F920719F480E090E00FC00A891B89A9
:109D70000C5E1F4F0197AC01662757FD6095762F4B
:109D80009E01C701CADD81E090E0E6E0CDB7DEB715
:109D90000C940F7688E397E008958BEC9AE0089591
:109DA000A2E0B0E0E6EDFEE40C94F575DC01892B51
:109DB00079F16230710560F10D911C911197660F78
:109DC000771F80E090E0FD01268137814085518535
:109DD000620F731F841F951FD801ED91FC9122E043
:109DE00030E0AE014F5F5F4F0995882389F02981EC
:109DF0003A812115310571F0BFEF273F3B0741F054
:109E0000C9014096079720F0EFEF283F3E0710F07A
:109E100020E030E0C901E4E022960C941176A2E043
:109E2000B0E0E5E1FFE40C94E9755C01009709F40A
:109E300046C06230710508F442C0FC01668077803C
:109E4000808491842E010894411C511C660F771F59
:109E50007B0100E010E0E60CF71C081D191DD50180
:109E6000ED91FC910190F081E02D22E030E0A20123
:109E7000C801B7010995882311F1C980DA80C1149E
:109E8000D10401F1C60140960897C8F0B8EFCB168F
:109E9000BFEFDB0610F0CC24DD241A821982D50135
:109EA000ED91FC910480F581E02D22E030E0A201EB
:109EB000C801B7010995B601CD2821F603C080E09D
:109EC00090E002C081E090E0E0E122960C940576FB
:109ED000AAE0B0E0EEE6FFE40C94E7753C012B014C
:109EE000009709F48EC0DC01ED91FC912081318155
:109EF0003A8729870480F581E02DF887EF83FC01FC
:109F000086819781A085B1858B839C83AD83BE8339
:109F100082859385A485B585B695A79597958795F0
:109F20001C015A01CC24DD2442E0842E912C42C035
:109F3000C401880F991F7C0100E010E02B813C8157
:109F40004D815E81E20EF31E041F151F22E030E0FA
:109F5000AE014F5F5F4FC801B701A985BA85FD010A
:109F60000995882309F44DC089819A81892BF9F4D8
:109F7000C114D10429F48FEF9FEF9A83898302C023
:109F8000DA82C98222E030E0AE014F5F5F4FC80144
:109F9000B701EF81F8850995882381F00894A1081D
:109FA000B108A114B10411F464010AC06401089459
:109FB000811C911C8214930408F4BACFAB28F1F4ED
:109FC000F2E04F165104F8F0DA82C982440C551CB5
:109FD000B20180E090E02B813C814D815E81620F77
:109FE000731F841F951F22E030E0AE014F5F5F4F6B
:109FF000AF81B885FD010995882329F4B601C30115
:10A000000EDFCC24DD24C601E2E12A960C9403760F
:10A0100080E190E00895CF93DF93EC01892BC1F0AC
:10A0200062307105A8F06250704080E090E02889AD
:10A03000398940E050E00E9458759B01AC018A8943
:10A040009B89AC89BD89280F391F4A1F5B1F04C03B
:10A0500020E030E040E050E0CA01B901DF91CF914B
:10A060000895A6E0B0E0E7E3F0E50C94E7752C0175
:10A070007A8369835C834B83009709F4CAC0672B9A
:10A0800009F4C7C0452B09F4C4C0FC01A5A4B6A4BB
:10A09000C7A4D0A825A136A147A150A56B817C817A
:10A0A000CB01A0E0B0E08A0D9B1DAC1DBD1D2817A3
:10A0B00039074A075B0738F42A193B093C832B838D
:10A0C000232B09F4A9C0D201ED91FC91208831889D
:10A0D000F20101A8F2A9E02DFE83ED83EF2B71F5CB
:10A0E000F20103A0F4A1E02DFE83ED83EF2B39F400
:10A0F000A114B104C104D10409F48EC08AC0A11412
:10A10000B104C104D104D1F0860175010FC06D8185
:10A110007E81D2018D919C9143DE9E838D83892B1C
:10A1200009F477C0E618F7080809190931018824ED
:10A130009924E614F7040805190548F7089421083E
:10A14000310831016A207B200894211C311C8B804E
:10A150009C80D201ED91FC915101A618B7088A1498
:10A160009B0408F45401C080D180730100E010E02A
:10A170006D817E81CF014FDFE60EF71E081F191F8C
:10A18000F601C080D180950149815A81C801B7018B
:10A19000F6010995882321F18A189B08C501A0E0E2
:10A1A000B0E0F20125A536A547A550A9280F391F13
:10A1B0004A1F5B1F25A736A747A750ABC501860DD1
:10A1C000971D8215930598F06D817E818081918124
:10A1D000E7DD9E838D83892B41F4F20112AA11AA37
:10A1E0004B815C814819590919C0662477246D8117
:10A1F0007E81F20172AB61AB8114910439F08981E7
:10A200009A818A0D9B1D9A838983A3CF4B815C81A0
:10A2100005C04FEF5FEF02C040E050E0CA01E2E14D
:10A2200026960C940376FC01892B19F480E090E0CB
:10A23000089583A194A196A785A710AA17A681E0E7
:10A2400090E00895A0E0B0E0E8E2F1E50C94F1754B
:10A250008C017901F901C081D1818281938180963D
:10A2600093838283F8018081853E09F4B0C08823FE
:10A2700009F4ADC08FA198A5A9A5BAA50097A1051D
:10A28000B10521F44FA358A769A77AA7209709F42D
:10A290009BC00115110509F497C0F801908199231D
:10A2A00009F492C0B801655F7F4F83858F3041F517
:10A2B000892F90E08F7390702DE030E0829FA00195
:10A2C000839F500D929F500D11249A012D503040C4
:10A2D00060E871E0DE01A20FB31F0EC0FB018191A7
:10A2E000BF01F801E80FF11D80818D932F5F3F4F73
:10A2F0002417350709F46BC02F31310578F367C097
:10A300008881882309F04DC0A801DE01680130E092
:10A31000F60190819032A1F09C93F801848583FF2F
:10A3200008C0F6018081813420F08B3510F4905EF6
:10A330009C933F5F0894C11CD11C1196383041F7A3
:10A340008881853011F485EE8883F801808580321C
:10A3500011F4232F22C0FE01E30FF11D8EE2808352
:10A36000232F2F5FFA0190859032B9F0DE01A20F02
:10A37000B11D9C93F801848584FF08C0FA01808593
:10A38000813420F08B3510F4905E9C932F5F4F5FEB
:10A390005F4F832F8C5F281729F7FE01E20FF11D15
:10A3A0001082FB01808188A3F801828D938D9AA38E
:10A3B00089A3848D958DA68DB78D8BA39CA3ADA30A
:10A3C000BEA381E0F701848380E090E002C081E0D9
:10A3D00090E0E8E0CDB7DEB70C940D76A7E2B0E0F0
:10A3E000E4EFF1E50C94E7752C017FA36EA30097D1
:10A3F00009F484C0672B09F481C0DC016D907C9066
:10A40000F30120883188FC0185A496A4A7A4B0A8F4
:10A410004BE250E060E070E08EA19FA10E94A67721
:10A4200045E050E060E070E0CE0101960E94A67722
:10A430008EA19FA19A8389838114910409F04BC056
:10A44000F3012288338886899789281A390A43C0FC
:10A45000750100E010E08114910431F4F301668984
:10A460007789808D918D03C0B401C301D4DD6E0D59
:10A470007F1D801F911F1C821B82D301ED91FC91D7
:10A4800081010A191B090280F381E02D6E010894F5
:10A49000C11CD11C22E2E22E21E5F22E20E230E0A6
:10A4A000AE014A5F5F4F0995882341F18B819C8102
:10A4B000A80EB91EA214B30470F0B401C30170DC7D
:10A4C0004C01892B31F4F20183A094A0AA24BB246F
:10A4D00006C0AA24BB248D81882309F4B9CFF201D8
:10A4E00096A685A6B0AAA7A620E030E0AEA1BFA19F
:10A4F0008C91882329F021E030E002C020E030E098
:10A50000C901E2E1A7960C940376A0E1B0E0EBE884
:10A51000F2E50C94ED758C016230710518F480E061
:10A5200090E021C078DD4B015C0140E150E060E04B
:10A5300070E06E010894C11CD11CC6010E94A67770
:10A54000D8014D915C91F80120893189FA01A681E9
:10A55000B781EE24FF2408E010E5A601C501B4018F
:10A56000FD01099590E0ECE060960C940976A3E07B
:10A57000B0E0EDEBF2E50C94E7754C018B01892B13
:10A5800009F4A7C04115510509F4A3C0CA010E94EE
:10A59000C1770C966DE070E00E9483756F5F6B83EE
:10A5A000F80123A034A02114310451F0AA24BB24C3
:10A5B0006501EE24FF2487014424552432010BC099
:10A5C000F401E688F788008D118D428853886488ED
:10A5D0007588570168011A82E414F5040605170509
:10A5E00009F047C02114310409F473C0E114F104E7
:10A5F0000105110561F1B101C401D2DB009731F50C
:10A6000041E050E0B101C40163DC8C01892B09F405
:10A6100060C002501040B80180E090E00E5F1F4F14
:10A62000F4012089318940E050E00E9458755B01B7
:10A630006C01F40182899389A489B589A80EB91E99
:10A64000CA1EDB1EB801C40160DF46C01C01B10197
:10A65000C401E1DC7B018C01F401808991892C012A
:10A66000662477244E0C5F1C601E711E5701680122
:10A670001A82D401ED91FC910190F081E02D21E04E
:10A6800030E0AE014F5F5F4FC801B70109958823E5
:10A6900001F18981853E11F0882379F4BA81BF5F89
:10A6A000BA83EB81BE17C0F480E290E0A0E0B0E096
:10A6B000E80EF91E0A1F1B1F8FCF30E2A32EB12C0C
:10A6C000C12CD12CAE0CBF1CC01ED11E8601750141
:10A6D00082CFAA24BB246501C601B501E2E123961D
:10A6E0000C9403764F925F927F928F929F92AF92DB
:10A6F000BF92CF92DF92EF92FF920F931F93CF936F
:10A70000DF93CDB7DEB7A0970FB6F894DEBF0FBECC
:10A71000CDBFFC018B01892B09F409C161157105BD
:10A7200009F405C10190F081E02D44805580FB01C2
:10A7300087A090A4A1A4B2A4CB010E94C177F82E57
:10A7400090E00C966DE070E00E949775762E4BE0DD
:10A7500050E060E270E0CE0101960E94A6776EE2C2
:10A7600070E0C8010E94E777FC010097B1F06C012E
:10A770000894C11CD11C8181882379F0C6010E94F4
:10A78000C177F81AFA94482F843008F043E050E07B
:10A79000B601CE0109960E949D77CE010196F8E0A0
:10A7A000FF1588F04F2D50E0B8010E949D77D80129
:10A7B0008C918E3209F5F80181818E3209F4828103
:10A7C0008823C9F019C048E050E0B8010E949D7785
:10A7D000F80181A1982F92959F70803A10F4905DB6
:10A7E00001C09F598F708A3010F4805D01C08F596D
:10A7F0009F83888701C077248981853E11F485E095
:10A80000898345E150E060E070E0CE010C960E9443
:10A81000A677F80180A18C8781A192A19C8F8B8F54
:10A8200083A194A1A5A1B6A18D8F9E8FAF8FB8A350
:10A83000672D70E045E0660F771F4A95E1F780E0ED
:10A8400090E0680D791D8A1D9B1D20E230E0AE016D
:10A850004F5F5F4FF2010995882309F468C0E980D2
:10A86000FE0132968E2D8695E794EE24E794E82A31
:10A870008191E80ECE010C96E817F90799F7F72CAD
:10A8800050C040E250E06FEF70E0CE0101960E94B0
:10A89000A6770D5010408DE0F89E90011124200FF6
:10A8A000311F035F1F4F91E0FE013196AF01490F49
:10A8B000511DD9018C91DA018C93892F8F5FE80F9C
:10A8C000F11D10829E5F9B3021F09A3119F49CE1BA
:10A8D00001C09EE0F9018081882329F09F3118F49E
:10A8E0002F5F3F4FE1CFF982F71419F48F2D806469
:10A8F00089838FE08C87EE861D861B8E1C8E20E25E
:10A9000030E0AE014F5F5F4FC501B401F201099520
:10A9100080E290E0A0E0B0E0880E991EAA1EBB1E67
:10A92000FA94FF2009F0ADCF81E090E002C080E012
:10A9300090E0A0960FB6F894DEBF0FBECDBFDF91BA
:10A94000CF911F910F91FF90EF90DF90CF90BF902C
:10A95000AF909F908F907F905F904F900895A0E070
:10A96000B0E0E5EBF4E50C94F1757C018B01EA01B4
:10A97000892B09F441C06115710509F43DC0FB0143
:10A9800080818823C9F1452BB9F1BE01C70126DDBD
:10A99000882349F0BE01C8010E94B877892BA9F726
:10A9A000C70141DC29C0F701C080D1804BE250E0F3
:10A9B00060E070E0CE010E94A6774FE150E0B80160
:10A9C000CE010E94D877AE01B701C601D0DD6FA3DA
:10A9D00078A789A79AA7611571058105910561F08E
:10A9E000BE01C6017FDE90E0882309F491E081E09A
:10A9F0009827892F90E002C080E090E0E8E0CDB792
:10AA0000DEB70C940D76A6E0B0E0E9E0F5E50C9435
:10AA1000E9757C012A013B01009709F4C8C0FC01DB
:10AA200003A114A10190F081E02DC088D188011507
:10AA3000110531F4411551056105710509F4A3C0F3
:10AA40004B825C826D827E8214C0B801D7018D91E9
:10AA50009C91A6D90097D1F02B813C814D815E81DC
:10AA6000281939094A095B092B833C834D835E838E
:10AA70008C014601AA24BB248B819C81AD81BE81BF
:10AA800088169906AA06BB0600F394C068016B817C
:10AA90007C818D819E81680D791D8A1D9B1D615071
:10AAA000704080409040A50194010E94AA75A901C0
:10AAB000B801D7018D919C910BDA009709F477C00A
:10AAC000012B21F4F70194A383A36C01F70145A2A4
:10AAD00056A267A270A6411451046104710411F4D6
:10AAE00014A213A2B7016E5F7F4FD7018D919C9185
:10AAF000F9DD882309F45BC0411451046104710439
:10AB000029F4B601F701808191813CC02B813C8101
:10AB10004D815E8182169306A406B506A0F1D70189
:10AB20000D911C910115110571F1B2E0CB16D10404
:10AB300050F1B601C80134D95C018FEF9FEF9A83C1
:10AB40008983F80180809180CC0CDD1CB60180E007
:10AB500090E02681378140855185620F731F841FE5
:10AB6000951FF401A481B58122E030E0AE014F5F72
:10AB70005F4FFD010995882331F0A114B10419F04C
:10AB8000B501C8014CD9F70185A596A5A7A5B0A91F
:10AB9000481659066A067B0638F4F70145A656A6FC
:10ABA00067A670AA12AA11AA81E090E009C080E00D
:10ABB00090E006C068010115110509F468CF86CF41
:10ABC000E0E126960C940576A0E0B0E0EAEEF5E52B
:10ABD0000C94F175EC016B01892B09F445C06115EA
:10ABE000710509F441C08DA59EA5AFA5B8A9413056
:10ABF00059F0413018F0423069F036C0FB01E08076
:10AC0000F1800281138113C0FB01E080F180028199
:10AC1000138109C0FB01E080F180028113818DA1C5
:10AC20009EA1AFA1B8A5E80EF91E0A1F1B1F8DA19A
:10AC30009EA1AFA1B8A58E159F05A007B10730F45E
:10AC4000B801A701CE01DFDE882371F0EDA6FEA6D4
:10AC50000FA718AB1AAA19AAF601E082F1820283A3
:10AC6000138381E090E002C080E090E0E8E0CDB79F
:10AC7000DEB70C940D76A6E0B0E0E1E4F6E50C94C6
:10AC8000E7755C017A8369835C834B83009709F4E1
:10AC900011C1672B09F40EC1452B09F40BC1FC014E
:10ACA00065A476A487A490A885A196A1A7A1B0A524
:10ACB00086159705A805B90508F4FCC08081918127
:10ACC000FC0120883188F50101A8F2A9E02DFE835E
:10ACD000ED83EF2B09F050C0F50103A0F4A1E02DA6
:10ACE000FE83ED83EF2B99F46114710481049104C8
:10ACF00009F0E0C041E050E060E070E0E9D89E83F8
:10AD00008D83F50194A383A3892B09F4D3C0F501A6
:10AD1000E5A4F6A407A510A9E114F10401051105A5
:10AD200019F52AC0E81AF90A0A0B1B0B6D817E81FE
:10AD3000D5018D919C9134D8009719F09E838D8315
:10AD400013C0E114F1040105110509F0B3C041E09D
:10AD500050E06D817E81F50180819181B9D80097A5
:10AD600009F4A8C09E838D83C101A0E0B0E0E8167D
:10AD7000F9060A071B07B0F60894210831082101DB
:10AD8000462057200894211C311C6B807C80D50103
:10AD9000ED91FC914101841895086814790408F438
:10ADA0004301C080D180720100E010E06D817E819E
:10ADB000CF0131D9E60EF71E081F191FF601A48135
:10ADC000B581940149815A81C801B701FD010995F6
:10ADD000882309F447C068187908C401A0E0B0E0EE
:10ADE000F50125A536A547A550A9280F391F4A1FEB
:10ADF0005B1F25A736A747A750ABC401840D951D3F
:10AE00008215930500F16D817E81808191810E9480
:10AE1000D04E009719F09E838D8313C06114710486
:10AE200051F041E050E06D817E81D5018D919C9182
:10AE30004FD8009721F4F50112AA11AA13C09E83DE
:10AE40008D83442455242D813E81F50132AB21AB05
:10AE50006114710439F089819A81880D991D9A8352
:10AE6000898395CFF50185A596A5A7A5B0A9E5A0ED
:10AE7000F6A007A110A5E816F9060A071B07A8F413
:10AE800085A396A3A7A3B0A7B5016E5F7F4F80816E
:10AE9000918128DC882349F4F50165A476A46E1815
:10AEA0007F08E5A6F6A607A710AB8B819C818619C3
:10AEB000970902C08FEF9FEFE2E126960C9403768C
:10AEC000009711F00C94C8760895009711F00C9437
:10AED000C8760895EF92FF920F931F93CF93DF935D
:10AEE0007C018B01892BF1F061157105D9F0FB0113
:10AEF00080A184FF17C081E390E00E941E76009736
:10AF000089F0EC014BE250E0B80102960E949D7777
:10AF1000F982E882F80181A192A19EA78DA718AAC3
:10AF20001FA602C0C0E0D0E0CE01E6E0CDB7DEB79C
:10AF30000C940F76EF92FF920F931F93CF93DF93B2
:10AF40007C018B01892B01F161157105E9F0FB0191
:10AF500080A184FD19C083E390E00E941E760097D3
:10AF600099F0EC014BE250E0B80102960E949D7707
:10AF7000F982E8821DA61EA61FA618AAF80181A1C3
:10AF800092A19AAB89AB02C0C0E0D0E0CE01E6E06E
:10AF9000CDB7DEB70C940F76ACE2B0E0E2EDF7E5AA
:10AFA0000C94E7759AA789A7009709F447C1FC019B
:10AFB00084819581892B09F441C186819781892BF0
:10AFC00009F43CC18AE190E00E941E769CA78BA701
:10AFD000009709F433C198A78FA34AE150E060E0DD
:10AFE00070E00E94A677E9A5FAA5AFA1B8A5ED93F8
:10AFF000FC93218432844384548419E0220C331C52
:10B00000441C551C1A95D1F7C201B101655F7F4FF1
:10B010008F4F9F4F0190F081E02D29E130E0AE018C
:10B020004F5F5F4F0995882309F404C1E981FA81D4
:10B03000FBA3EAA32C813D81FB81FCA34E818F8180
:10B0400098859EA38DA3E985FA856C857D856E889C
:10B050007F88888C998C611471048104910431F487
:10B06000309709F4E7C03F018824992461157105E0
:10B0700009F4E0C0C901A0E0B0E08A8F9B8FAC8FDB
:10B08000BD8F80E090E0242F30E040E050E00E944F
:10B0900058756E8F7F8F88A399A3840173012A8DC1
:10B0A0003B8D4C8D5D8DE21AF30A040B150BE61AED
:10B0B000F70A080B190B8AA19BA101972DA13EA1AC
:10B0C000B5E0220F331FBA95E1F7820F931F6AA1F3
:10B0D0007BA10E94837580E090E0E61AF70A080BD6
:10B0E000190B8CA1282F30E040E050E0C801B701D7
:10B0F0000E94AA7579018A01253F9FE0390790E0F7
:10B10000490790E0590708F495C0255F3F4F40403C
:10B11000504010F486E001C08BE0E9A5FAA58087D5
:10B1200048E150E060E070E08BA59CA502960E948B
:10B13000A6772AA13BA15901CC24DD24C401B30187
:10B14000A60195010E945875EBA5FCA56283738347
:10B1500084839583C601B5012A8D3B8D4C8D5D8D11
:10B160000E945875260E371E481E591EEBA5FCA5D9
:10B170002682378240865186E9A5FAA580858630E9
:10B1800029F462E070E080E090E004C064E070E0E8
:10B1900080E090E022E030E040E050E0E20EF31E7C
:10B1A000041F151FA80197010E945875EBA5FCA567
:10B1B00062877387848795872AA13BA13787268773
:10B1C0003CA1832F90E0AC01AAA1BBA14A9FC00182
:10B1D0004B9F900D5A9F900D1124918B808B6E8DFB
:10B1E0007F8D88A199A1A60195010E945875EBA5B4
:10B1F000FCA52681378140855185620F731F841F0E
:10B20000951F668B778B808F918FADA1BEA19D011D
:10B2100040E050E0A5E0220F331F441F551FAA95C0
:10B22000D1F7620F731F841F951F628B738B848B02
:10B23000958B06C08BA59CA50E94C87618A61FA258
:10B240008FA198A5E2E1AC960C9403766F927F9261
:10B250008F929F92BF92CF92DF92EF92FF920F93C5
:10B260001F93CF93DF933C01EB017A01892B09F403
:10B270005FC0672B09F45CC08881882309F458C03B
:10B28000452B09F455C08F3209F421964BE250E06A
:10B2900060E070E0C7010E94A67780E1F70180A31B
:10B2A0008881882309F447C0B701C30113DE6C010C
:10B2B000892B09F43DC06FE270E0CE010E94AD77AA
:10B2C000009739F0B82EBC1A4C010894811C911CCF
:10B2D00027C0CE010E94C177B82E4E01880E911C66
:10B2E0001FC0C7010E94C1778C018B2D90E0081709
:10B2F0001907B1F4A801B701CE010E94CA77892BC2
:10B3000079F4C601DDDDC00FD11F8881882399F053
:10B31000F70180A184FF0CC0E401CC24DD2405C02A
:10B32000B701C6015BD88823E1F6C601C9DDB8CFF5
:10B3300080E090E002C081E090E0DF91CF911F912A
:10B340000F91FF90EF90DF90CF90BF909F908F90E4
:10B350007F906F9008956F927F928F929F92AF929D
:10B36000BF92DF92EF92FF920F931F93CF93DF93E1
:10B37000CDB7DEB760970FB6F894DEBF0FBECDBF76
:10B380007C015B014A013901D02E892B09F49CC054
:10B39000672B09F499C083E080170CF495C007FD72
:10B3A0001DC0602F772767FD7095B4E0660F771F8B
:10B3B000BA95E1F762547E4F882777FD8095982FE4
:10B3C00020E130E0AE014F5F5F4FF7010995882320
:10B3D00009F47AC08D81882309F476C081E190E078
:10B3E0000E941E76009709F46FC08C0141E150E085
:10B3F00060E070E00E94A677F801F182E082B382FB
:10B40000A2829582848277826682D7FC59C08D8120
:10B4100080872A8530E040E050E0542F432F322FC0
:10B4200022278B8590E0A0E0B0E0DC0199278827F7
:10B43000282B392B4A2B5B2B898590E0A0E0B0E0CC
:10B44000282B392B4A2B5B2B8C8590E0A0E0B0E0B9
:10B45000B82FAA2799278827282B392B4A2B5B2B13
:10B4600021873287438754872E8530E040E050E0C3
:10B47000542F432F322F22278F8590E0A0E0B0E099
:10B48000DC0199278827282B392B4A2B5B2B8D85AC
:10B4900090E0A0E0B0E0282B392B4A2B5B2B888969
:10B4A00090E0A0E0B0E0B82FAA2799278827282BA2
:10B4B000392B4A2B5B2B258736874787508B06C055
:10B4C0008FEFF801808702C000E010E0C8016096AD
:10B4D0000FB6F894DEBF0FBECDBFDF91CF911F91A5
:10B4E0000F91FF90EF90DF90BF90AF909F908F9063
:10B4F0007F906F9008950F93CF93DF93CDB7DEB712
:10B50000AB970FB6F894DEBF0FBECDBF00E020EDC5
:10B5100033E24CE453E263E174E286ED92E21BDF36
:10B5200090931C0880931B08892B81F40FEF20ED6A
:10B5300033E24CE453E263E174E286ED92E20BDF26
:10B5400090931C0880931B08892BA1F080911B0805
:10B5500090911C0821DD90931A0880931908009798
:10B5600049F0AE014F5F5F4F64E171E06FDE80E054
:10B5700090E002C08FEF9FEFAB960FB6F894DEBF5E
:10B580000FBECDBFDF91CF910F91089580E090E085
:10B59000FC01EE0FFF1FEE0FFF1FE35EF74F11825E
:10B5A000108201968C30910599F70895AC0120E046
:10B5B00030E0F901EE0FFF1FEE0FFF1FE35EF74FC4
:10B5C000808191818417950781F080819181892BF9
:10B5D00039F4518340837383628380E090E008955F
:10B5E0002F5F3F4F2C30310521F78FEF9FEF0895EC
:10B5F000A0E0B0E0EEEFFAE50C94EF755C016B01B2
:10B60000FB01E080F1806EE57BE0C7010E94777767
:10B61000892B11F589E39BE09F938F930E944178DA
:10B62000CFE1D8E00F900F9088819981009771F059
:10B630009F938F930E94417886E39BE09F938F9323
:10B640000E9441780F900F900F900F902496F8E091
:10B65000CF34DF0749F723C00FE118E0C0E0D0E0A6
:10B66000F8016081718161157105C9F0C7010E94FF
:10B670007777892B71F4CC0FDD1FCC0FDD1FC35EF4
:10B68000D74FE881F981B601C501099580E090E0C6
:10B6900008C021960C5F1F4FCC30D10509F78FEF02
:10B6A0009FEFEAE0CDB7DEB70C940B76EF92FF92F6
:10B6B0000F931F93CF93DF93EC018B017A010E94CC
:10B6C000C177AC01F801D183C08320E030E060E0B5
:10B6D00070E0A0E038C0FE01E20FF31F80818D30E2
:10B6E00051F08E3018F4882339F02BC08032C9F025
:10B6F000823221F026C010829A0123C0AA2371F45D
:10B700001082FB01EE0FFF1FE00FF11FCE0101962B
:10B71000820F931F91838083A1E013C01082A0E069
:10B7200010C0AA2371F410826F5F7F4FFB01EE0FF0
:10B73000FF1FE00FF11FCE010196820F931F91832F
:10B7400080832F5F3F4F241735071CF46E157F054C
:10B7500014F2CB010196E6E0CDB7DEB70C940F767C
:10B76000A8E4B0E0E6EBFBE50C94F37529E0E22EEB
:10B77000F12CEC0EFD1EBC01C7010E94807744E055
:10B7800050E08E010F5F1F4FB801C7018FDFB80176
:10B790002FDFE6E0C85BDF4F0C940F76A8E0B0E047
:10B7A000E4EDFBE50C94F57544E050E08E010F5F8D
:10B7B0001F4FB8017BDFB8011BDFE4E028960C9433
:10B7C0001176A7E0B0E0E7EEFBE50C94F775809109
:10B7D000B8049091B9042FEF8F3F9207F1F480E500
:10B7E00090E00E945B2B9093B9048093B8048F5F24
:10B7F0009F4F09F4BFC081E080938C041092B30482
:10B800001092B2041092EA031092E9031092E80336
:10B81000109291041092900412C00E94872B8823EA
:10B8200089F48091B8049091B9040E94EB2F8FEFB6
:10B830009FEF9093B9048093B80410928C041092F7
:10B840008D0498C080918C04813009F457C061C088
:10B850008091B8049091B9040E948F2E8A3009F427
:10B860004DC090918D042091B2043091B30499237E
:10B8700071F4F901E851FC4F8283F9013196F0939C
:10B88000B304E093B204E851FC4F128206C02F5F6C
:10B890003F4F3093B3042093B2048D3079F5992350
:10B8A000E1F443E050E066ED7BE08AEE93E00E9435
:10B8B0006177892B11F481E00BC044E050E061ED29
:10B8C0007BE08AEE93E00E946177892B31F482E07D
:10B8D00080938D0488EE93E026D180918D04882397
:10B8E00049F08091B2049091B304019719F483E078
:10B8F00080938C041092B3041092B2048091B80427
:10B900009091B9040E94B42B181619060CF4A0CF1C
:10B9100031C0833079F5CE0101960E946541609176
:10B92000B8047091B90482E00E94434188EE93E02C
:10B93000F9D1019769F088EE93E02ED2019741F09A
:10B9400083E69BE09F938F930E9441780F900F9026
:10B950000E942541CE0101960E9457418091B80472
:10B960009091B9040E94EB2F8FEF9FEF9093B90451
:10B970008093B804E2E027960C9413760F931F93FC
:10B980008DD180E590E00E942A2B0FEF1FEF1093DE
:10B99000B9040093B80480E590E09F938F9380EE04
:10B9A0009BE09F938F930E9441786AED7BE081EE4C
:10B9B0009BE50E945D481093B9040093B8040F9072
:10B9C0000F900F900F901F910F910895A0E0B0E09D
:10B9D000ECEEFCE50C94EF75FC016B01E855FF4FB4
:10B9E000E190F190EF01AA24BB2400E010E00DC02B
:10B9F000B601888199810E947777892B19F4AA244E
:10BA0000AA94BA2C0F5F1F4F22960E151F0584F3C0
:10BA1000C501EAE0CDB7DEB70C940B76A0E0B0E04C
:10BA2000E4E1FDE50C94EF75FC016B01E855FF4F77
:10BA3000E190F190EF01AA24AA94BA2C00E010E062
:10BA40000BC0B601888199810E947777892B09F410
:10BA500058010F5F1F4F22960E151F0594F3C50165
:10BA6000EAE0CDB7DEB70C940B76A0E0B0E0EBE3F4
:10BA7000FDE50C94EF75FC016B01E855FF4FE1907B
:10BA8000F190EF01AA24BB2400E010E00DC0B60144
:10BA9000888199810E94B877892B19F4AA24AA94E5
:10BAA000BA2C0F5F1F4F22960E151F0584F3C50198
:10BAB000EAE0CDB7DEB70C940B76CF92DF92FF921F
:10BAC0000F931F93CF93DF93EC016C011FC088830A
:10BAD000F60180818532B1F486010F5F1F4F680146
:10BAE0000894C11CD11CF80180810E94A948F82E3D
:10BAF000F29480EFF822F882F80181810E94A9482F
:10BB0000F82AF88221960894C11CD11CF601808184
:10BB10008823E9F61882DF91CF911F910F91FF9052
:10BB2000DF90CF900895A0E0B0E0E9E9FDE50C9446
:10BB3000F175EC01FC0180E090E022812F3241F0B0
:10BB4000222331F001963196823A9105B1F7A1C0D6
:10BB50009C012F5F3F4FAE014E5F5F4FCA01820FC6
:10BB6000931F99838883EE24FF2415C0F901EC0FFD
:10BB7000FD1F82818F3339F412822F5F3F4F7A018C
:10BB8000E20EF31E06C0803211F0882311F41282F7
:10BB900005C02F5F3F4F223A310544F328EAC22EF9
:10BBA000D12CCC0EDD1ED6011D921C92088119816C
:10BBB000C8010E94C177892B29F467EF7BE0C80197
:10BBC0000E948077E114F10409F463C081E090E001
:10BBD000F60191838083C654DF4FF982E882609733
:10BBE000F982E882CA5AD04019C08632A1F4D7013E
:10BBF0001D927D01DE01A855BF4FED91FC9111977B
:10BC00003196ED93FC93EE0FFF1FEC0FFD1FE855EF
:10BC1000FF4FF182E0820894E11CF11CF701808162
:10BC2000882319F78E0106551F4FEE24FF2428C0E4
:10BC3000D8012D913C91F801318B208B10C08D33B0
:10BC400031F4D9011D929D01F801B18BA08BD9016E
:10BC50008C918B3211F480E28C932F5F3F4FF9016E
:10BC60008081882361F7D8018D919C9126DFF801AE
:10BC70008089918922DF0894E11CF11C0E5F1F4F1F
:10BC8000C855DF4F88819981C85AD0408E159F05CD
:10BC90007CF6E8E0CDB7DEB70C940D7680E090E05E
:10BCA000FC01EE0FFF1FEE0FFF1FE35BF74F11824A
:10BCB000108201968431910599F70895AC0120E036
:10BCC00030E0F901EE0FFF1FEE0FFF1FE35BF74FB0
:10BCD000808191818417950781F080819181892BE2
:10BCE00039F4518340837383628380E090E0089548
:10BCF0002F5F3F4F2431310521F78FEF9FEF0895DC
:10BD000082E09CE09F938F930E9441780F900F9068
:10BD1000089585E19CE09F938F930E9441780F9056
:10BD20000F900895EF92FF920F931F93CF93DF939D
:10BD30007C010FE418E0C0E0D0E0F801608171817F
:10BD40006115710511F1F701808191810E9477776A
:10BD5000892BA9F48FE29CE09F938F930E944178F6
:10BD6000CC0FDD1FCC0FDD1FC35BD74FE881F981FE
:10BD7000C701099581E090E00F900F9008C02196CF
:10BD80000C5F1F4FC431D105C1F68FEF9FEFE6E086
:10BD9000CDB7DEB70C940F76ACE9B0E0E2EDFEE58E
:10BDA0000C94E7753C01FC0100811181C8010E94DF
:10BDB000C177080F191F2224332416C0F8012081EF
:10BDC0002F3249F411928F01F30160817181AE012C
:10BDD000495F5F4F0CC02E3221F418010894211CDA
:10BDE000311C015010400197009741F7AAC0809183
:10BDF000190890911A082ADABE01695F7F4F809175
:10BE0000190890911A0866D82C01892BB9F496C0AC
:10BE1000B801C7010E94B877892B81F4FE01EB5A63
:10BE2000FF4FA080B180C280D380C2010E94135115
:10BE3000A114B104C104D10469F480C022E3E22E4C
:10BE4000F12CEC0EFD1EB701C2010E94EE518823B9
:10BE5000F9F674C0B7018091190890911A086AD850
:10BE60004C01892B09F464C0198262E07DE0C101B4
:10BE70000E947777892B39F06EEF7CE0C1010E9438
:10BE80007777892B31F468EF7CE0CE0101960E9430
:10BE900080773F922F92CE0101969F938F93DF92EE
:10BEA000CF92BF92AF928DE79CE09F938F930E94B9
:10BEB00041780E9425418DB79EB70A960FB6F89437
:10BEC0009EBF0FBE8DBF90EDE92EF12CE60CF71C46
:10BED000F701808191810E94872B882361F48FEF85
:10BEE0009FEFF7019183808384EA90E0680E791ECA
:10BEF000F30110821DC08DE5C82ED12CCC0EDD1EA5
:10BF000040E450E0B601C4010E9431508C0101961A
:10BF1000029770F020E0A601B801F70180819181BD
:10BF20000E94BC300034110574F601E010E002C03C
:10BF30000FEF1FEFC4010E94655709C00FEF1FEFFD
:10BF400006C0AE01495F5F4F66E171E050CFC201AC
:10BF50000E946057C801E2E1C456DF4F0C9403769B
:10BF6000A7E0B0E0E6EBFFE50C94F3758091BA042E
:10BF70009091BB042FEF8F3F920799F587E190E0F6
:10BF80000E945B2B9093BB048093BA048F5F9F4FFA
:10BF900009F4CDC08E010F5F1F4FC8010E9465419B
:10BFA0006091BA047091BB0482E00E94434189E130
:10BFB0009DE09F938F930E944178C8010E94574152
:10BFC0001092ED041092EC041092BC041092EF0455
:10BFD0001092EE048091BA049091BB040E949C2BB5
:10BFE000A4C00E94872B882369F48091BA049091A1
:10BFF000BB040E94EB2F8FEF9FEF9093BB048093C5
:10C00000BA0495C08091EE049091EF04892B41F120
:10C0100030C08091BA049091BB040E948F2E8A3068
:10C02000F9F087FD1DC02091EC043091ED04203320
:10C0300031056CF4F901E654FB4F8283F901319626
:10C04000F093ED04E093EC04E654FB4F12828D3044
:10C0500039F481E090E09093EF048093EE0409C0FE
:10C060008091BA049091BB040E94B42B1816190653
:10C0700084F28091EE049091EF04019709F057C08B
:10C080007E010894E11CF11CC7010E94654160918A
:10C09000BA047091BB0482E00E94434144E050E046
:10C0A00062EF74E08CEB94E001DB8C019093F1047F
:10C0B0008093F00464E17DE08091F2049091F304B8
:10C0C0000E947777892BD1F48AE09DE09F938F932C
:10C0D0000E9441780E94254160E070E081E00E946A
:10C0E00043418091BA049091BB040E94EB2F8FEFE3
:10C0F0009FEF9093BB048093BA0417C062EF74E083
:10C10000C80176DA87E09DE09F938F930E94417883
:10C11000C7010E9457411092ED041092EC04109256
:10C12000BC041092EF041092EE040F900F90E6E022
:10C1300027960C940F7687E190E00E942A2B87E1E6
:10C1400090E09F938F938DE49DE09F938F930E9447
:10C15000417866E47DE080EB9FE50E945D480F90AA
:10C160000F900F900F9008959C01FC01EE0FFF1FA0
:10C17000E80FF91FEE0FFF1FE256F74F84819581FC
:10C180008F5F9F4FC1F16281738180919D0877FF1E
:10C1900007C040E090E00E949775892B39F405C0F4
:10C1A00040E090E06817790709F441E0F901EE0FEB
:10C1B000FF1FE20FF31FEE0FFF1FE256F74F6081E4
:10C1C00071818091B00877FF07C020E090E00E9465
:10C1D0009775892B39F405C020E090E0681779073E
:10C1E00009F421E0413039F480E0213009F081E0A8
:10C1F000842790E0089580E090E00895A0E2B0E008
:10C20000E4E0F1E60C94F3757C017F936F9386E68E
:10C210009DE09F938F938E010F5F1F4F1F930F938E
:10C220000E946478B701C8010E94B2432DB73EB79F
:10C230002A5F3F4F0FB6F8943EBF0FBE2DBFE6E01A
:10C24000A0960C940F7643E050E030CAA0E2B0E034
:10C25000ECE2F1E60C94F5759F938F9386E69DE0F2
:10C260009F938F938E010F5F1F4F1F930F930E9419
:10C270006478C8010E948C428DB79EB706960FB6AF
:10C28000F8949EBF0FBE8DBF80E090E0E4E0A096E2
:10C290000C941176A0E2B0E0E0E5F1E60C94F375C1
:10C2A000EE24FF24FF92EF9286E69DE09F938F930A
:10C2B0008E010F5F1F4F1F930F930E946478C80178
:10C2C0000E94FD412DB73EB72A5F3F4F0FB6F8944D
:10C2D0003EBF0FBE2DBF8F5F9F4F51F00894E11CF2
:10C2E000F11C83E0E816F104E9F6EE24EA94FE2C52
:10C2F000C701E6E0A0960C940F76A0E2B0E0E3E878
:10C30000F1E60C94F3757C01C5DF2FEF8F3F9207A8
:10C31000C9F09F938F9386E69DE09F938F938E0144
:10C320000F5F1F4F1F930F930E946478B701C801DE
:10C330000E9401438DB79EB706960FB6F8949EBF34
:10C340000FBE8DBF80E090E0E6E0A0960C940F76E3
:10C35000ADE2B0E0EEEAF1E60C94F5758E01025F15
:10C360001F4FBC01C8014ADFBE016F5F7F4FC8018C
:10C370006ADF8E01095F1F4FC8010E94654160E0BE
:10C3800070E080E00E9443418D819E8107DAC80100
:10C390000E945741E4E0AD960C941176A2E1B0E022
:10C3A000E4EDF1E60C94F575CE0101960E94F816C5
:10C3B0009C8180919D08891729F49B818091B00808
:10C3C000891799F08C8180939D088B818093B008A8
:10C3D00000E010E0C801C8DE892B11F0C801B8DF09
:10C3E0000F5F1F4F03301105A9F7E4E062960C942C
:10C3F0001176A2E1B0E0EFEFF1E60C94F7758FEF64
:10C400009FEF9093A3088093A2089093A90880932C
:10C41000A8089093AF088093AE08CE0101960E94C1
:10C42000F8168C8180939D088B818093B00868E911
:10C430007DE08EEC91E60E945D48E2E062960C940D
:10C440001376A6E2B0E0E7E2F2E60C94F175D1DFF4
:10C45000EE24FF24CC24DD24FF92EF9286E69DE0BB
:10C460009F938F938E01095F1F4F1F930F930E941D
:10C470006478B801C8010E94B2432DB73EB72A5F65
:10C480003F4F0FB6F8943EBF0FBE2DBF8F5F9F4F3B
:10C4900021F1BE016F5F7F4FC801D5DE0397E9F43C
:10C4A0008601000F111F0C0D1D1D000F111F0256DC
:10C4B000174FF801F582E48289819A810E941E77E4
:10C4C000F801938382838B819C810E941E77F801FF
:10C4D000918380830894C11CD11C0894E11CF11C39
:10C4E000F3E0EF16F10409F0B7CFE8E0A6960C945C
:10C4F0000D767FDFA6DF42DA1EDE6CD10C941B4C7A
:10C50000DDD132D40E94A66B0E94D36E89D40E94E2
:10C51000166E78D10E940E6DC6D458D5E8D60E940A
:10C520005B6F0E94E06F0E9420730E9443750C9421
:10C530003F6DA3E4B0E0EFE9F2E60C94E975CE01BB
:10C5400042960E94F8169B898091FD04891709F490
:10C550003CC18B898093FD04CE0101960E94654108
:10C5600060E070E084E00E94434160E080E00E946F
:10C570003E259C898091FE048917D1F08C892D89F4
:10C5800090E09F938F9330E03F932F9388E09EE05D
:10C590009F938F930E9441788C898093FE042DB7DE
:10C5A0003EB72A5F3F4F0FB6F8943EBF0FBE2DBF78
:10C5B00061E080E00E943E258B8965E00E947775EE
:10C5C000992309F0FCC08091FA049091FB04019634
:10C5D0009093FB048093FA0486EF9DE09F938F93E2
:10C5E0000E9441780F900F908091FA049091FB0483
:10C5F0008330910509F450C08430910534F48130C2
:10C60000910579F00297B1F1CEC08530910509F41A
:10C6100060C0853091050CF459C0069709F4A4C098
:10C62000C2C08E01085F1F4FB8018091FC040E94B8
:10C63000F44A1F930F938091FC0490E09F938F9393
:10C6400089EE9DE09F938F930E9441788091FC0436
:10C650008F5F8093FC042DB73EB72A5F3F4F0FB624
:10C66000F8943EBF0FBE2DBF883008F4A8C01092CA
:10C67000FC04A5C08C8D9D8DAE8DBF8DBF93AF93F7
:10C680009F938F938CED9DE09F938F930E944178B1
:10C690008DB79EB7069681C06091340170913501C7
:10C6A0008091360190913701AE014C5D5F4F0E9441
:10C6B000AD389F938F9389ED9DE09F938F930E9458
:10C6C00041780F900F900F900F9079C08AEC9DE009
:10C6D00070C00E9442703B014C0184E2482E512CF4
:10C6E0004C0E5D1EC2010E943170892B09F41CA200
:10C6F0000E94E66F7B018C010E94E66F5B016C017A
:10C700005F924F92C801B701A40193010E94CC75BA
:10C710007B018C0168EE73E080E090E0A40193015E
:10C720000E94CC75C801B7010E9458759F938F93E2
:10C730007F936F93C601B501A40193010E94CC754C
:10C740005F934F933F932F938DEB9DE09F938F9338
:10C750000E9441782DB73EB7245F3F4F0FB6F89443
:10C760003EBF0FBE2DBF2BC0898D9A8D288DEF89BE
:10C7700064E670E00E9483759F938F9330E03F934F
:10C780002F93F0E0FF93EF938AEA9DE09F938F93BE
:10C790000E9441788DB79EB708960FB6F8949EBF59
:10C7A0000FBE8DBF0CC01092FB041092FA048DE9ED
:10C7B0009DE09F938F930E9441780F900F900E946D
:10C7C0002541CE0101960E945741E0E1CD5BDF4F4C
:10C7D0000C940576A2E1B0E0E0EFF3E60C94F77577
:10C7E000CE0101960E94F8168A818093FD046EE1C5
:10C7F0007EE089E992E60E945D48E2E062960C9450
:10C800001376089567E27EE081E094E657CAAFE1CF
:10C81000B0E0EDE0F4E60C94F07587E39EE09F93C2
:10C820008F930E944178CC24DD240F900F9086E0F6
:10C83000E82EF12CEC0EFD1E9E012F5F3F4FA7014D
:10C84000BE016E5F7F4FC6010E948836813041F580
:10C85000B980BB2029F18E01045F1F4FB801C701C9
:10C860000E94CC367C016A817B818C819D81A801EC
:10C870000E94AD382B2D30E03F932F93FF92EF9223
:10C880009F938F938FE29EE09F938F930E944178B6
:10C890008DB79EB708960FB6F8949EBF0FBE8DBF9A
:10C8A0000894C11CD11C92E0C916D10409F0BFCF75
:10C8B00080E090E0E9E06F960C940C7664E47EE012
:10C8C00087E094E60C94D65AA2E1B0E0EAE6F4E6FA
:10C8D0000C94F3757C01CE0101960E94F8168091AC
:10C8E000FF04909100050196909300058093FF044A
:10C8F000088519858F812E8149816A81EB81AC8100
:10C900001F930F9390E09F938F9330E03F932F936B
:10C9100050E05F934F9370E07F936F93F0E0FF934D
:10C92000EF93B0E0BF93AF938CE09FE09F938F9322
:10C930000E9441786B857C858D859E8520E831E558
:10C9400041E050E00E94AA758DB79EB740960FB6A1
:10C95000F8949EBF0FBE8DBF2115310541055105CD
:10C9600051F1213031054105510599F45F934F9301
:10C970003F932F9383E09FE09F938F930E94417892
:10C98000EDB7FEB736960FB6F894FEBF0FBEEDBFFB
:10C9900012C05F934F933F932F9389EF9EE09F9335
:10C9A0008F930E9441788DB79EB706960FB6F89484
:10C9B0009EBF0FBE8DBF6B857C858D859E8520E8D3
:10C9C00031E541E050E00E94AA7520E13EE040E000
:10C9D00050E00E94AA75211531054105510591F0DD
:10C9E0005F934F933F932F9380EF9EE09F938F939E
:10C9F0000E944178EDB7FEB736960FB6F894FEBFA9
:10CA00000FBEEDBF6B857C858D859E8520E13EE068
:10CA100040E050E00E94AA752CE330E040E050E096
:10CA20000E94AA75211531054105510591F05F93CA
:10CA30004F933F932F9387EE9EE09F938F930E9497
:10CA400041788DB79EB706960FB6F8949EBF0FBE7D
:10CA50008DBF6B857C858D859E852CE330E040E025
:10CA600050E00E94AA75611571058105910591F04C
:10CA70009F938F937F936F938FED9EE09F938F9300
:10CA80000E944178EDB7FEB736960FB6F894FEBF18
:10CA90000FBEEDBF83ED9EE09F938F930E94417880
:10CAA00020918E0730918F07409190075091910708
:10CAB0000F900F902030F4E03F07F0E04F07F0E0D8
:10CAC0005F0770F45F934F933F932F9387EC9EE043
:10CAD0009F938F930E9441788DB79EB7069648C06A
:10CAE000203090E0390790E1490790E05907A8F419
:10CAF000FAE05695479537952795FA95D1F75F93C4
:10CB00004F933F932F938AEB9EE09F938F930E94C6
:10CB10004178EDB7FEB7369653C02030F0E03F07BE
:10CB2000F0E04F07F0E45F0748F5DA01C901AF70A4
:10CB3000B070EAE0B695A79597958795EA95D1F7F5
:10CB4000BF93AF939F938F9374E156954795379515
:10CB500027957A95D1F75F934F933F932F9387EA69
:10CB60009EE09F938F930E9441788DB79EB70A965F
:10CB70000FB6F8949EBF0FBE8DBF27C0DA01C90162
:10CB8000BF7364E1B695A795979587956A95D1F798
:10CB9000BF93AF939F938F938EE1569547953795AB
:10CBA00027958A95D1F75F934F933F932F9384E90D
:10CBB0009EE09F938F930E944178EDB7FEB73A961F
:10CBC0000FB6F894FEBF0FBEEDBF80ED90E0E80E0B
:10CBD000F91EF701808191819F938F938091FF04CB
:10CBE000909100059F938F9380918A0790918B0776
:10CBF000A0918C07B0918D07BF93AF939F938F93B4
:10CC000088E49EE09F938F930E9441788DB79EB7F2
:10CC10000A960FB6F8949EBF0FBE8DBFE6E06296EF
:10CC20000C940F76CF92DF92EF92FF920F931F93A7
:10CC30008091B0039091B103A091B203B091B3037E
:10CC4000BF93AF939F938F9380918A0790918B07A7
:10CC5000A0918C07B0918D07BF93AF939F938F9353
:10CC600080918E0790918F07A0919007B0919107C6
:10CC7000BF93AF939F938F9389E690E19F938F9398
:10CC80000E9441788091AC039091AD039F938F9364
:10CC90008091AE039091AF039F938F938091AA03ED
:10CCA0009091AB039F938F938091A8039091A903D8
:10CCB0009F938F9388E290E19F938F930E94417896
:10CCC0000E94A03582E70E94961C082F81E00E94F6
:10CCD000501D7C0181E10E94501D6C010E947A353B
:10CCE0008CE190E19F938F930E9441788BE090E1DB
:10CCF0009F938F930E94417887EF9FE09F938F933C
:10CD00000E94417810E01F930F9382EE9FE09F9363
:10CD10008F930E9441788DB79EB782960FB6F89494
:10CD20009EBF0FBE8DBFFF92EF928FEC9FE09F934F
:10CD30008F930E944178DF92CF928CEB9FE09F937C
:10CD40008F930E9441788DB79EB708960FB6F894DE
:10CD50009EBF0FBE8DBF80E090E01F910F91FF90AE
:10CD6000EF90DF90CF90089568EA70E182E196E657
:10CD70000E94D65A6EE970E184E694E60C945E5EF9
:10CD8000CF93DF93EC010E94895EC855DF4F888105
:10CD90009981C85AD040892B59F486EC90E19F9331
:10CDA0008F930E9441780E94805E0F900F9030C058
:10CDB00060EC70E1CE010E94E65C892B49F164EBE6
:10CDC00070E1CE010E940E5DFC01EE0FFF1FEC0F23
:10CDD000FD1FE654FF4F6AEB70E1808191810E9454
:10CDE0007777892BA9F48EEA90E19F938F930E9425
:10CDF00041780E94805E0E942541C053DF4F8881A8
:10CE000099810E94EB2F0E9455450F900F90FFCF04
:10CE1000DF91CF9108950E94554580E090E00895FC
:10CE200061E571E18BE097E60E94D65A67E471E113
:10CE300080EC96E60C945E5EA4E1B0E0E2E2F7E6F8
:10CE40000C94F5758B01029701F5FB0182819381AA
:10CE50000E94DC3DAE014F5F5F4F0E94AD389F9353
:10CE60008F93F801828193819F938F9388E691E15C
:10CE70009F938F930E9441788DB79EB706960FB609
:10CE8000F8949EBF0FBE8DBF08C087E591E19F93C8
:10CE90008F930E9441780F900F9080E090E0E4E043
:10CEA00064960C94117668E771E18CE197E60C9436
:10CEB000D65ACF93DF9382E092E19F938F930E94A3
:10CEC00041788FEC91E19F938F930E944178C0E06D
:10CED000D0E00F900F900F900F908C2F0E940B1AA4
:10CEE00068E873E101960E94241A9C0168EE73E0E1
:10CEF0000E9497759F938F93C90168EE73E00E941B
:10CF000097757F936F93DF93CF9385E891E19F931C
:10CF10008F930E94417821968DB79EB708960FB6E1
:10CF2000F8949EBF0FBE8DBFC830D105B1F68CE717
:10CF300091E19F938F930E9441780E94805E0F90B1
:10CF40000F90DF91CF910895CF93DF93EB0164EAC7
:10CF500072E18A819B810E947777892B51F58C81C0
:10CF60009D810E941E77EC0188309105A8F40E94F3
:10CF70000B1A9F938F93DF93CF9384E992E19F9352
:10CF80008F930E9441788DB79EB706960FB6F8949E
:10CF90009EBF0FBE8DBF15C09F938F938BE692E10E
:10CFA0009F938F930E9441780F900F900F900F9056
:10CFB00008C088E592E19F938F930E9441780F907B
:10CFC0000F9080E090E0DF91CF91089560EB72E1E7
:10CFD00084EA97E60E94D65A68EA72E189E597E604
:10CFE0000C945E5EAAE0B0E0E8EFF7E60C94F17511
:10CFF0007C0128EA30E0E20EF31EF7018081918186
:10D0000028E53FEFE20EF31E892B79F1CC24DD24D5
:10D0100027C0802F90E09F938F9381EB93E19F93A4
:10D020008F938E010F5F1F4F1F930F930E946478A1
:10D03000B801C7010E94355DEDB7FEB736960FB651
:10D04000F894FEBF0FBEEDBF892B21F08C2D0E94FE
:10D05000B01B03C08C2D0E94A61B0894C11CD11CC0
:10D060000C2D0E94831BC816A0F20E94895E83E6E5
:10D0700093E19F938F930E944178CC24DD2447C095
:10D080008C2D0E94861B082F8C2D0E94861B10E081
:10D09000077010701F930F9386958695869590E084
:10D0A0008F5B9F4F9F938F938DE393E19F938F931C
:10D0B0000E944178EF2CFF24FF92EF9283E193E1ED
:10D0C0009F938F930E9441788C2D0E94931B2DB7C4
:10D0D0003EB7265F3F4F0FB6F8943EBF0FBE2DBF41
:10D0E000882361F0FF92EF928BE093E19F938F93FF
:10D0F0000E9441780F900F900F900F908FEF92E168
:10D100009F938F930E9441780894C11CD11C0F906B
:10D110000F90FC2C0E94831BC81608F4B1CF84EB3F
:10D1200092E19F938F930E9441780E94805E0F90BE
:10D130000F90E8E02A960C940D76FF920F931F93C0
:10D14000CF93DF930E94895E82E194E19F938F9356
:10D150000E944178C0E0D0E03BC08C2F0E94CE1BE3
:10D16000082F8C2F0E94CE1B10E0077010701F93A9
:10D170000F9386958695869590E08F5B9F4F9F9342
:10D180008F938CEE93E19F938F930E9441788F2D24
:10D1900090E00E94DB1B2DB73EB72A5F3F4F0FB6D2
:10D1A000F8943EBF0FBE2DBF882319F080EE93E1A7
:10D1B00002C083ED93E19F938F930E9441780F907B
:10D1C0000F9088EC93E19F938F930E944178219672
:10D1D0000F900F90FC2E0E94CB1BC81708F4BDCFF8
:10D1E00088EB93E19F938F930E9441780E94805E29
:10D1F0000F900F90E5E0CDB7DEB70C9410760F934B
:10D200001F93CF93DF938B01FB01848195810E9453
:10D210001E77EC010E94831B90E0C817D90714F415
:10D22000D7FF0DC0DF93CF9380EB94E19F938F9353
:10D230000E9441780F900F900F900F9051C0F8010D
:10D24000028113816CEA74E1C8010E947777892B0F
:10D2500089F168EA74E1C8010E947777892B61F04F
:10D2600061EA74E1C8010E947777892B49F48C2F19
:10D270000E94931B882359F48C2F0E94B01B1AC064
:10D280006BE974E1C8010E947777892B21F48C2F18
:10D290000E94A61B0FC00E94831B90E09F938F9358
:10D2A00081E794E19F938F930E9441780F900F90B4
:10D2B0000F900F908C2F0E94931B90E09F938F9361
:10D2C000DF93CF9380E694E19F938F930E94417800
:10D2D0008DB79EB706960FB6F8949EBF0FBE8DBF52
:10D2E00080E090E0DF91CF911F910F9108956EED56
:10D2F00074E18FEF98E60E94D65A63ED74E18DE9F0
:10D3000098E60E945E5E67EC74E182EF97E60C940B
:10D310005E5EA0E1B0E0EFE8F9E60C94F57560918F
:10D3200034017091350180913601909137018E0161
:10D330000F5F1F4FA8010E94AD389F938F9386E225
:10D3400099E19F938F930E94417860913801709189
:10D35000390180913A0190913B01A8010E94AD38BA
:10D360009F938F9389E199E19F938F930E944178D6
:10D3700060913C0170913D0180913E0190913F018F
:10D38000A8010E94AD389F938F938CE099E19F9301
:10D390008F930E944178609140017091410180918A
:10D3A000420190914301A8010E94AD389F938F9351
:10D3B00083E099E19F938F930E944178809132019D
:10D3C00090E09F938F938091310190E09F938F9392
:10D3D0008091300190E09F938F9380912F0190E096
:10D3E0009F938F9380912E0190E09F938F938091D4
:10D3F0002D0190E09F938F9387ED98E19F938F93FA
:10D400000E9441788DB79EB74E960FB6F8949EBF96
:10D410000FBE8DBF80E090E0E4E060960C94117642
:10D42000A0E2B0E0E6E1FAE60C94F5758C010E940A
:10D43000895E08551F4FF80180819181085A10407C
:10D44000892BA9F48FEC98E19F938F930E944178E8
:10D4500086EC98E10E94B05B80EC98E10E94B05BA2
:10D4600087EB98E19F938F930E944178C3C060EB54
:10D4700078E1C8010E94E65C892B09F4C0C082E60D
:10D4800098E19F938F930E9441788E010F5F1F4F09
:10D49000B8018DE598E10E941F4480E098E19F93D8
:10D4A0008F930E9441786DEF77E1C8010E947777F2
:10D4B0000F900F900F900F90892B41F485EF97E11B
:10D4C0009F938F930E9441780F900F9089EE97E180
:10D4D0009F938F930E944178B80186EE97E10E9456
:10D4E0001F440F900F90019759F060913401709193
:10D4F00035018091360190913701A8010E94AD3825
:10D500001F930F9381E797E19F938F930E94417838
:10D51000B8018CE697E10E941F440F900F900F9086
:10D520000F90019759F06091380170913901809105
:10D530003A0190913B01A8010E94AD381F930F93CF
:10D5400082EF96E19F938F930E944178B8018DEE10
:10D5500096E10E941F440F900F900F900F9001973B
:10D5600059F060913C0170913D0180913E01909194
:10D570003F01A8010E94AD381F930F9389E796E100
:10D580009F938F930E944178B80185E796E10E94AE
:10D590001F440F900F900F900F90019759F06091DA
:10D5A0004001709141018091420190914301A80195
:10D5B0000E94AD381F930F938FEF95E19F938F9348
:10D5C0000E944178B8018BEF95E10E941F440F90B3
:10D5D0000F900F900F90019729F0B8018DE291E024
:10D5E0000E94CC361F930F938EE195E19F938F930A
:10D5F0000E9441780F900F900F900F90A1C067EE9E
:10D6000074E1C8010E94E65C892B79F067EE74E151
:10D61000C8010E940E5DFC01EE0FFF1FE00FF11F1D
:10D62000E654FF4F6081718102C068E171E087EECE
:10D6300094E10E9489436CEE74E1C8010E94E65CAB
:10D64000892B91F06CEE74E1C8010E940E5DFC0123
:10D65000EE0FFF1FE00FF11FE654FF4F6081718155
:10D660008CEE94E10E9489436FEE74E1C8010E9440
:10D67000E65C892B91F06FEE74E1C8010E940E5DAB
:10D68000FC01EE0FFF1FE00FF11FE654FF4F60811A
:10D6900071818FEE94E10E94894364EF74E1C801C7
:10D6A0000E94E65C892B91F064EF74E1C8010E944E
:10D6B0000E5DFC01EE0FFF1FE00FF11FE654FF4F60
:10D6C0006081718184EF94E10E94894369EF74E184
:10D6D000C8010E94E65C892B91F069EF74E1C801F2
:10D6E0000E940E5DFC01EE0FFF1FE00FF11FE654DC
:10D6F000FF4F6081718189EF94E10E9489436DEF52
:10D7000074E1C8010E94E65C892B91F06DEF74E131
:10D71000C8010E940E5DFC01EE0FFF1FE00FF11F1C
:10D72000E654FF4F608171818DEF94E10E9489433F
:10D7300081E095E19F938F930E9441780F900F9025
:10D740000E94805EE4E0A0960C9411766AE379E191
:10D7500089E899E60E94D65A6EE279E180E19AE67C
:10D760000C945E5EA4E2B0E0E8EBFBE60C94F57589
:10D770008C010E94895E08551F4FF80180819181BC
:10D78000085A1040892B09F065C08E010B5F1F4FAE
:10D79000B80183E499E10E941F4488EF9AE19F93C6
:10D7A0008F930E94417865EF7AE1C8010E947777F4
:10D7B0000F900F90892B41F48DEE9AE19F938F93F8
:10D7C0000E9441780F900F9081EE9AE19F938F9382
:10D7D0000E94417883E499E10E9465420F900F9086
:10D7E0008F5F9F4F31F0B80187E499E10E941F4499
:10D7F00005C06FEC7AE1C8010E94807781E599E16C
:10D800000E9465429E012F5F3F4F8F5F9F4F31F017
:10D81000B90181E599E10E941F4405C06DEC7AE1F0
:10D82000C9010E948077CE0101969F938F93CE010C
:10D8300005969F938F9386E799E19F938F930E941C
:10D8400041788DB79EB706960FB6F8949EBF0FBE6F
:10D850008DBF56C063E479E1C8010E94E65C892B64
:10D8600079F063E479E1C8010E940E5DFC01EE0FDE
:10D87000FF1FE00FF11FE654FF4F6081718102C06E
:10D880006CE171E083E499E10E94894367E479E106
:10D89000C8010E94E65C892B91F067E479E1C80138
:10D8A0000E940E5DFC01EE0FFF1FE00FF11FE6541A
:10D8B000FF4F6081718187E499E10E94894361E5AE
:10D8C00079E1C8010E94E65C892B91F061E579E17C
:10D8D000C8010E940E5DFC01EE0FFF1FE00FF11F5B
:10D8E000E654FF4F6081718181E599E10E9489438F
:10D8F00089E599E19F938F930E9441780F900F9053
:10D900000E94805EE4E0A4960C941176A6E2B0E05A
:10D91000ECE8FCE60C94F1758B01029709F070C0FD
:10D9200032E0C32ED12CC60ED71EFB01828193811B
:10D930000E94D338611571058105910579F4F801CC
:10D94000828193810E94DC3D7B018C016F5F7F4F60
:10D950008F4F9F4F29F488EE9BE154C07B018C01CF
:10D96000F601808191819F938F9385ED9BE19F9339
:10D970008F930E94417881E599E10E9465420F9062
:10D980000F900F900F908F5F9F4F41F0BE016D5E23
:10D990007F4F81E599E10E941F4401C01B8ACE019F
:10D9A00043960E943B779B01AC0140E050E0C801E8
:10D9B000B7010E94213D8F5F9F4FF9F0CE01019684
:10D9C0000E94F8168A812B814C8190E09F938F935F
:10D9D00030E03F932F9350E05F934F9389EB9BE1AF
:10D9E0009F938F930E9441788DB79EB708960FB68C
:10D9F000F8949EBF0FBE8DBF0BC080EB9BE102C0B1
:10DA00008EE99BE19F938F930E9441780F900F9036
:10DA100080E090E0E8E0A6960C940D7669EF7BE15B
:10DA200086E89CE60E94D65A61EF7BE182EB9BE69A
:10DA30000C945E5EAAE0B0E0E0E2FDE60C94F575C1
:10DA4000FB010297B1F4828193810E947A498E0191
:10DA50000F5F1F4FB8010E9408491F930F938DEF6E
:10DA60009BE19F938F930E9441780F900F900F90AE
:10DA70000F9080E090E0E4E02A960C94117660E04C
:10DA80007CE18AE19DE60C94D65AA0E2B0E0EBE49A
:10DA9000FDE60C94F1756C010E94895E28EA30E085
:10DAA000C20ED31EF6018081918128E53FEFC20EA0
:10DAB000D31E892B71F58DE89FE19F938F930E9470
:10DAC000417800E010E00F900F90B8016E010894CB
:10DAD000C11CD11CC6010E94FE60019791F41F93E6
:10DAE0000F93DF92CF928BED9EE19F938F930E94D5
:10DAF00041788DB79EB706960FB6F8949EBF0FBEBD
:10DB00008DBF0F5F1F4F03301105F9F68FE29EE1C5
:10DB100009C068E27EE1C6010E94E65C892B49F0FB
:10DB200083E49CE19F938F930E9441780F900F9024
:10DB300078C06FE37CE1C6010E94E65C892B09F4A2
:10DB400055C06CE37CE1C6010E940E5DFC01EE0F46
:10DB5000FF1FEC0DFD1DE654FF4F808191810E9457
:10DB60001E777C0169E37CE1C6010E940E5DFC0129
:10DB7000EE0FFF1FEC0DFD1DE654FF4F80819181DC
:10DB80000E941E778C0165E37CE1C6010E940E5D58
:10DB9000FC01EE0FFF1FEC0DFD1DE654FF4F8081D1
:10DBA00091819F938F931F930F93FF92EF928AE23D
:10DBB0009CE19F938F938E010F5F1F4F1F930F93D5
:10DBC0000E946478C8010E947D610E9421628DE0FC
:10DBD0009CE19F938F930E944178EDB7FEB73C96EE
:10DBE0000FB6F894FEBF0FBEEDBF1BC069E07CE12D
:10DBF000C6010E94E65C892BA1F065E07CE1C601CC
:10DC00000E940E5DFC01EE0FFF1FEC0DFD1DE654A2
:10DC1000FF4F808191810E941E770E9426610E94A1
:10DC200021620E94805EE8E0A096F7C760EC7FE189
:10DC300085E49DE60C945E5E0E94895E80ED9FE126
:10DC40009F938F930E9441780E94754489EC9FE1D5
:10DC50009F938F930E9441780E94805E0F900F9057
:10DC60000F900F900895A0E2B0E0E8E3FEE6B9C798
:10DC70007B0102970CF48AC082E0C82ED12CC60E1C
:10DC8000D71E61E770E2F701828193810E94777766
:10DC9000892B19F00FEF1FEF13C06EE670E28E01B3
:10DCA0000F5F1F4FC8010E948077B80180E690E2A5
:10DCB0000E94894381E090E00E94CF4100E010E0A3
:10DCC00066E570E2F601808191810E947777892B69
:10DCD000D9F480E090E00E94CF4162E570E28E01CD
:10DCE0000F5F1F4FC8010E948077B80184E490E263
:10DCF0000E94894386E390E29F938F930E9441782C
:10DD000000E010E00F900F9062E370E2F601808176
:10DD100091810E947777892B59F4F7016681778189
:10DD2000848195810E947343019711F400E010E013
:10DD30006EE270E2F601808191810E947777892BF3
:10DD400049F4F701848195810E948C42019711F476
:10DD500000E010E068E270E2F601808191810E94AB
:10DD60007777892B21F40E94754400E010E062E28D
:10DD700070E2F601808191810E947777892B19F4F6
:10DD80000E9448440BC00F5F1F4F41F486ED9FE196
:10DD90009F938F930E9441780F900F9080E090E0C6
:10DDA000E8E0A0963AC763E870E283E39EE60E944B
:10DDB000D65A69E770E28CE19EE60C945E5EABE0B9
:10DDC000B0E0E4EEFEE611C70E94895E8FEF90E2BC
:10DDD0009F938F930E944178198210E00F900F90CB
:10DDE00023C060E00E94861F8130D9F4112341F0E6
:10DDF0008DEF90E29F938F930E9441780F900F9048
:10DE00001F5F898190E09F938F9385EF90E29F93AE
:10DE10008F930E9441780E947A1F0F900F900F906D
:10DE20000F9089818F5F8983898187FFDACF8CEC9E
:10DE300090E29F938F930E94417888E489830F90AA
:10DE40000F9029C08E010F5F1F4FC8010E943E2016
:10DE500080509048E9F0C8010E943E208E010E5F7C
:10DE60001F4FB8010E9408491F930F93898190E0CA
:10DE70009F938F9380E990E29F938F930E944178C4
:10DE80008DB79EB706960FB6F8949EBF0FBE8DBF96
:10DE900089818F5F898389818035A0F289E890E24A
:10DEA0009F938F930E9441780E94805E0F900F9005
:10DEB000E4E02B96B6C669E371E28FED9EE60C9422
:10DEC0005E5EA2E1B0E0E6E6FFE68EC60E94895EF5
:10DED0008BE791E29F938F930E944178FF24FA94FD
:10DEE0000F900F90F894BE016F5F7F4F8F2D0E94AF
:10DEF000991EF82E78948FEFF81619F489E691E2BE
:10DF000005C09EEFF91649F48DE591E29F938F933A
:10DF10000E9441780F900F904EC088E591E29F9348
:10DF20008F930E9441788E010F5F1F4F0F900F90CB
:10DF3000F80181918F0190E09F938F9382E591E2A8
:10DF40009F938F930E9441780F900F900F900F90A6
:10DF5000CE0108960817190759F7888590E09F9316
:10DF60008F938BE491E29F938F930E9441788981F4
:10DF70000E94FD1E9F938F930E944178CE010196CF
:10DF80000E94141F8E01075F1F4FB8010E940849AD
:10DF90001F930F9381E491E29F938F930E944178A6
:10DFA0008DB79EB70A960FB6F8949EBF0FBE8DBF71
:10DFB000FF2009F097CF0E94805EE5E0629630C6B0
:10DFC00064EA71E281E69FE60C945E5E8FB7F89496
:10DFD0008FBF6091040570910505809106059091B1
:10DFE000070508952FB7F89460930405709305050D
:10DFF00080930605909307052FBF08958091010532
:10E000008823B9F48091040590910505A091060537
:10E01000B09107050196A11DB11D80930405909351
:10E020000505A0930605B093070581E080930105DF
:10E0300008951092010508950F931F938C010E947B
:10E04000F816F80120E030E080E090E8958B848BB2
:10E050002F5F3F4F329620393105B1F71F910F9155
:10E060000895CF93DF93EC01BC0180EE91E20E9412
:10E070001F448F5F9F4F11F4C0E0D0E0CE01DF91CD
:10E08000CF910895A0E1B0E0E7E4F0E7AEC58E01DE
:10E090000F5F1F4FB80180EB91E20E941F448F5F1A
:10E0A0009F4F29F461E070E080E090E002C0C80179
:10E0B000E2D6E4E06096B5C5A4E5B1E0E1E6F0E7BC
:10E0C00086C580E291E09CAB8BABDCDF3B014C0171
:10E0D00084E092E29F938F937E010894E11CF11CEF
:10E0E000FF92EF92F1D78E010F5D1F4FC801A4DFA1
:10E0F000B701C8010E94A14E8DE392E29F938F93D6
:10E10000C0D785E3282E312C2C0E3D1E44245524E7
:10E110008DB79EB706960FB6F8949EBF0FBE8DBF03
:10E120004114510439F08BE392E29F938F93A9D766
:10E130000F900F90F10180819181F0E880309F076E
:10E1400041F485E392E29F938F939BD70F900F90BA
:10E1500030C05C01CC24B7FCC094DC2CC601B501F6
:10E16000A401930119D57B018C0168EE73E080E076
:10E1700090E0A401930110D5C801B70199D49F93F1
:10E180008F937F936F93C601B501A401930104D5CA
:10E190005F934F933F932F938AE292E29F938F93E3
:10E1A00070D78DB79EB70A960FB6F8949EBF0FBE74
:10E1B0008DBF0894411C511CE2E0F0E02E0E3F1E82
:10E1C000F0E94F16510409F0ABCF86E292E29F933B
:10E1D0008F9357D70F900F9060E070E080E090E051
:10E1E000E2E1CC5ADE4F0FC5A2E7B0E0E9EFF0E77D
:10E1F000F2C433E5C32ED12CCC0EDD1EC60131DFB7
:10E20000DF92CF9287E192E29F938F9323E1822E58
:10E21000912C8C0E9D1E9F928F9256D78FE092E28A
:10E220009F938F9393E3692E712C6C0E7D1E7F92CA
:10E230006F924AD7CE0101960E94F816EE800F81A8
:10E24000A884B9840E94CA4EDF92CF929F928F9287
:10E25000FF24FF92EF9210E0015010401F930F93A4
:10E26000BF92AF927F926F929F938F930AD724DFD2
:10E270000E94CD4E9F938F9304D78DB79EB74A9639
:10E280000FB6F8949EBF0FBE8DBFEEE0CE58DF4FA5
:10E29000BEC4A0E2B0E0EEE4F1E799C48C01F2DE86
:10E2A0001B012C01CE010196DCDE892B09F41982B9
:10E2B0000E94895E08551F4FF80180819181085A9C
:10E2C0001040892B09F03FC081DE7B018C017EDE8E
:10E2D0005B016C017BDE3B014C011F930F93FF92AE
:10E2E000EF9281E090E08C0F9D1F9F938F93C6016A
:10E2F000B501A201910150D47B018C0168EE73E05D
:10E3000080E090E0A201910147D4C801B701D0D3C9
:10E310009F938F937F936F93C401B301A2019101E7
:10E320003BD45F934F933F932F938DE894E29F9359
:10E330008F93A7D6EDB7FEB770960FB6F894FEBFD1
:10E340000FBEEDBF94C066E874E2C8010E94E65CAF
:10E35000892BC1F18E010F5E1F4FB80180ED91E254
:10E360000E941F448F5F9F4F91F063E874E2C801E1
:10E37000BED5892B69F48BE794E29F938F931F930B
:10E380000F93A2D60F900F900F900F9001C0198A93
:10E39000CE0101969F938F935F924F923F922F925F
:10E3A000CE0141969F938F9380E792E29F938F9344
:10E3B00068D68DB79EB70A960FB6F8949EBF0FBE6B
:10E3C0008DBF55C06AEF71E2C8010E94E65C892BDF
:10E3D00091F06AEF71E2C8010E940E5DFC01EE0F40
:10E3E000FF1FE00FF11FE654FF4F6081718180EB4A
:10E3F00091E20E94894365EF71E2C8010E94E65CE8
:10E40000892B91F065EF71E2C8010E940E5DFC015D
:10E41000EE0FFF1FE00FF11FE654FF4F6081718187
:10E4200080EE91E20E9489436CEE71E2C8010E9485
:10E43000E65C892B79F06CEE71E2C8010E940E5DFA
:10E44000FC01EE0FFF1FE00FF11FE654FF4F60814C
:10E45000718102C060E271E080ED91E20E94894327
:10E4600085E592E29F938F930CD60F900F900E94B8
:10E47000805EE2E1A096C7C3EF92FF921F93CF9315
:10E48000DF93CDB7DEB760970FB6F894DEBF0FBE4F
:10E49000CDBF1FB7F8946091040570910505809178
:10E4A0000605909107052AE030E07E010894E11C02
:10E4B000F11CA70197D51FBFB70181EC91E20E9423
:10E4C000894360960FB6F894DEBF0FBECDBFDF91D3
:10E4D000CF911F91FF90EF900895A6E7B1E0E2E79A
:10E4E000F2E77FC380E291E0FE01ED5BFF4F938B8B
:10E4F000828BCE0141960E94F8168B896AE0F7D292
:10E50000992351F49B8980910305891729F0109272
:10E5100002058B898093030580910205882309F009
:10E520008BC08E010F5F1F4FB80180ED91E20E94FA
:10E530001F448F5F9F4F61F068EE74E2C801D7D42B
:10E54000892B31F48B896EE1D2D2992309F494DFBF
:10E5500003E4E02EF12CEC0EFD1EC7016DDD84E01E
:10E5600092E29F938F938E010D5D1F4F1F930F9328
:10E57000ABD5B801C7010E94A14E0F900F900F902C
:10E580000F90009721F4B801C7010E943B4E0197FC
:10E5900009F04FC0F70127813085888D998D2817A4
:10E5A000390741F496818F89981721F495818E89D6
:10E5B000981769F08E010D5B1F4FC8013DDDBE014C
:10E5C0006D5D7F4FC8010E943B4E019791F50C890C
:10E5D000FB88FCDC9B01AC0113E4C12ED12CCC0EDA
:10E5E000DD1E8F2D6AE083D210E0F801EE0FFF1FD1
:10E5F000E00FF11FEE0FFF1FE80FF11DEE0FFF1FE1
:10E60000EC0DFD1D8091080590910905281B390B23
:10E61000358B248BDBDC60930805709309058093B0
:10E620000A0590930B05BE016D5D7F4FC6010E94E8
:10E63000724E81E080930205E8E0CA58DE4FEDC2D9
:10E64000A0E1B0E0E5E2F3E7D0C21092030560E09C
:10E6500070E080E090E0C6DC8E010F5F1F4FB801D4
:10E6600081EC91E20E941F448F5F9F4F19F0C80117
:10E6700002D4B8DCABDC6093080570930905809385
:10E680000A0590930B051FB7F8946EEF7FE680E0C4
:10E690000E94752060E086E00E94922080E00E9447
:10E6A00083201FBF6BE075E289E491E70E945E5E04
:10E6B0006AEF74E284EF90E70E945E5E6BEE74E2B4
:10E6C0008DE692E70E945D4808DFE4E06096A9C20B
:10E6D0000F931F938C010E94F816F80120E030E0A0
:10E6E00080E090E8958B848B2F5F3F4F32962039E6
:10E6F0003105B1F71F910F910895A4E9B1E0E2E867
:10E70000F3E76FC2182F91E2C92ED12CCC0EDD1E7B
:10E71000B6010E945749892B09F47DC0812F90E0F2
:10E720009F938F938DE195E29F938F937E01089441
:10E73000E11CF11CFF92EF92C7D48E010F591F4FBD
:10E7400080E291E0F801938B828BC801C1DFB701B1
:10E75000C8010E94A14EC60114D4F601E80FF91FAA
:10E7600031978DB79EB706960FB6F8949EBF0FBE31
:10E770008DBF01C0319780818B33E1F73196FF93D4
:10E78000EF9387E695E29F938F937BD485E7C82E1E
:10E79000D12CCC0EDD1EEE24FF240F900F900F9095
:10E7A0000F90E114F10439F085E695E29F938F9381
:10E7B00068D40F900F908E010F5D1F4FB801F601C6
:10E7C000808191810E940849892B41F48FE595E26F
:10E7D0009F938F9356D40F900F900BC01F930F935E
:10E7E0008BE595E29F938F934CD40F900F900F90F1
:10E7F0000F900894E11CF11C82E090E0C80ED91E35
:10E8000090E9E916F10469F687E595E29F938F9305
:10E8100038D40F900F90E8E0CC56DE4FFEC1A2E74F
:10E82000B0E0E4E1F4E7D5C12C0180E595E29F93E7
:10E830008F9353E5C52ED12CCC0EDD1EDF92CF92E7
:10E8400043D4DF92CF9280E495E29F938F9343E18C
:10E85000842E912C8C0E9D1E9F928F9235D48EE229
:10E8600095E29F938F9333E3632E712C6C0E7D1E84
:10E870007F926F9229D4CE0101960E94F816EE8005
:10E880000F81A884B9840E94CA4EDF92CF929F92D2
:10E890008F92FF24FF92EF9210E0015010401F93DF
:10E8A0000F93BF92AF927F926F929F938F93E9D312
:10E8B00066E175E2C2010E94E65C2DB73EB7245EB8
:10E8C0003F4F0FB6F8943EBF0FBE2DBF892B89F086
:10E8D00066E175E2C2010E940E5DFC01EE0FFF1FB2
:10E8E000E40DF51DE654FF4F80819181A7D205DF2D
:10E8F00009C000E010E0802F00DF0F5F1F4F0830DD
:10E900001105C9F70E94CD4E9F938F93BAD30F90F4
:10E910000F90E0E1CE58DF4F78C1CF93DF93EC0149
:10E9200066E175E20E94E65C892B11F480E00FC07D
:10E9300066E175E2CE010E940E5DFC01EE0FFF1F45
:10E94000EC0FFD1FE654FF4F8081918177D2D5DE19
:10E95000DF91CF910895A6E6B1E0E0EBF4E741C185
:10E9600080E291E0FE01EB5BFF4F91838083CE015B
:10E9700001960E94F8168B816AE0B9D0992351F470
:10E980009B8180910D05891729F010920C058B81D0
:10E9900080930D0580910C05883008F070C00E94AE
:10E9A000FA496C018050904809F464C013E3E12EE9
:10E9B000F12CEC0EFD1EC7018BDE80910C0590E062
:10E9C0009F938F938DE195E29F938F938E010D5EC0
:10E9D0001F4F1F930F9378D3B801C7010E94A14E18
:10E9E0002DB73EB72A5F3F4F0FB6F8943EBF0FBE1C
:10E9F0002DBF009721F4B801C7010E943B4E01973B
:10EA0000C9F52AAD3BAD888599852817390741F4AA
:10EA100099AD8F81981721F498AD8E81981769F080
:10EA20008E010D5C1F4FC80153DEBE016D5E7F4F2E
:10EA3000C8010E943B4E0197E9F42C818B816AE06A
:10EA400056D030E0F901EE0FFF1FE20FF31FEE0F7B
:10EA5000FF1FE80FF11DEE0FFF1FEC0FFD1FE95B1D
:10EA6000FF4FD182C082BE016D5E7F4FCE01C39643
:10EA70000E94724E80910C058F5F80930C05E8E038
:10EA8000CA59DE4FCAC010920D0563E975E28BEAE0
:10EA900094E70E945D4869E875E28DE894E70E947A
:10EAA0005E5E6AE775E28FE094E70E945E5E53CF98
:10EAB000629FD001739FF001829FE00DF11D649F62
:10EAC000E00DF11D929FF00D839FF00D749FF00DEE
:10EAD000659FF00D9927729FB00DE11DF91F639F8F
:10EAE000B00DE11DF91FBD01CF0111240895991B3F
:10EAF00079E004C0991F961708F0961B881F7A9535
:10EB0000C9F780950895AA1BBB1B51E107C0AA1F36
:10EB1000BB1FA617B70710F0A61BB70B881F991FBE
:10EB20005A95A9F780959095BC01CD01089597FB62
:10EB3000092E07260AD077FD04D0E5DF06D0002095
:10EB40001AF4709561957F4F0895F6F79095819529
:10EB50009F4F0895A1E21A2EAA1BBB1BFD010DC0F9
:10EB6000AA1FBB1FEE1FFF1FA217B307E407F5077D
:10EB700020F0A21BB30BE40BF50B661F771F881F59
:10EB8000991F1A9469F760957095809590959B01EF
:10EB9000AC01BD01CF01089597FB092E05260ED0CB
:10EBA00057FD04D0D7DF0AD0001C38F450954095AB
:10EBB000309521953F4F4F4F5F4F0895F6F7909551
:10EBC0008095709561957F4F8F4F9F4F08952F923D
:10EBD0003F924F925F926F927F928F929F92AF92ED
:10EBE000BF92CF92DF92EF92FF920F931F93CF933A
:10EBF000DF93CDB7DEB7CA1BDB0B0FB6F894DEBFD1
:10EC00000FBECDBF09942A88398848885F846E84F6
:10EC10007D848C849B84AA84B984C884DF80EE8040
:10EC2000FD800C811B81AA81B981CE0FD11D0FB649
:10EC3000F894DEBF0FBECDBFED010895CF93DF93F3
:10EC4000AC01029710F442E050E0A091B308B091FB
:10EC5000B408FD01C0E0D0E020E030E020C08081B9
:10EC600091818417950769F482819381209719F027
:10EC70009B838A8304C09093B4088093B3089F0158
:10EC800032C04817590738F42115310519F0821799
:10EC9000930708F49C01EF010280F381E02D309787
:10ECA000F1F62115310599F1C901841B950B0497E3
:10ECB00008F4A901E0E0F0E028C08D919C91119743
:10ECC00082179307F9F44817590781F4ED018A81F7
:10ECD0009B81309719F09383828304C09093B4088A
:10ECE0008093B3089D012E5F3F4F4EC0841B950B50
:10ECF000FD01E80FF91F4193519302978D939C9367
:10ED00009F0142C0FD01A281B3811097B1F68091AD
:10ED1000B1089091B208892B41F48091260190911D
:10ED200027019093B2088093B10820912801309177
:10ED300029012115310541F42DB73EB780912401F9
:10ED400090912501281B390BA091B108B091B20810
:10ED5000A217B307B8F42A1B3B0B2417350790F012
:10ED6000CA0102962817390768F09D012E5F3F4FB0
:10ED7000C901840F951F9093B2088093B1084D93F9
:10ED80005C9302C020E030E0C901DF91CF9108958B
:10ED9000CF93DF93009709F44EC0EC0122971B82BA
:10EDA0001A82A091B308B091B408109711F140E015
:10EDB00050E001C0DC01AC17BD0700F1BB83AA83A2
:10EDC000FE0121913191E20FF31FEA17FB0771F465
:10EDD0008D919C911197280F391F2E5F3F4F3983DA
:10EDE0002883FD01828193819B838A83411551058C
:10EDF00059F4D093B408C093B3081DC0FD018281BB
:10EE00009381AD010097B1F6FA01D383C2832191BA
:10EE10003191E20FF31FEC17FD0769F488819981A6
:10EE2000280F391F2E5F3F4FFA01318320838A81DB
:10EE30009B8193838283DF91CF910895FC01882782
:10EE40009927E89421912032E9F3293010F02E30EF
:10EE5000C8F32B3239F02D3231F4689403C009D154
:10EE6000820F911D219120532A30C8F31EF49095F2
:10EE700081959F4F08951F93FC0199278827BC0116
:10EE8000E89411911032E9F3193010F01E30C8F3F4
:10EE90001B3249F01D3241F4689405C0D5D0610F92
:10EEA000711D811D911D119110531A30B8F33EF45C
:10EEB00090958095709561957F4F8F4F9F4F1F91D3
:10EEC0000895FB01DC0104C08D910590801921F4A7
:10EED00041505040C8F7881B990B0895FB01DC0195
:10EEE00002C005900D9241505040D8F70895FB01A3
:10EEF000DC018D91059080190110D9F3990B0895CB
:10EF0000FB01DC0105900D920020E1F70895FC0162
:10EF100005900020E9F7809590958E0F9F1F08952A
:10EF2000FB01DC0104C08D910190801921F4415056
:10EF30005040C8F7881B990B0895FB01DC0102C003
:10EF400001900D9241505040D8F70895DC0101C066
:10EF50006D9341505040E0F70895FC018191861770
:10EF600021F08823D9F7992708953197CF01089583
:10EF7000FB01DC018D91019080190110D9F3990BEF
:10EF80000895FC0101900020E9F7809590958E0F7F
:10EF90009F1F0895FB01DC014150504030F08D91DE
:10EFA0000190801919F40020B9F7881B990B089576
:10EFB000FB01DC014150504048F001900D920020CF
:10EFC000C9F701C01D9241505040E0F70895FC017F
:10EFD00081E090E00190061609F4CF010020D1F7FE
:10EFE00001970895FA01CF93FF93EF9322303CF1FC
:10EFF00025322CF5C22FE894CA3049F497FB3EF431
:10F0000090958095709561957F4F8F4F9F4F2C2FD6
:10F01000332744275527FF93EF939CDDEF91FF9112
:10F02000605D6A330CF0695D6193B901CA0160509B
:10F0300070408040904059F716F4CDE2C1931082A1
:10F040008F919F91CF9189C2592F482F372F262F0B
:10F05000660F771F881F991F660F771F881F991FDC
:10F06000620F731F841F951F660F771F881F991FDC
:10F0700008957AE0979F902D879F802D910D112400
:10F080000895A2E0B0E0E6E4F8E7B1CDFE013796DE
:10F0900061917191FA83E983E091B708F091B80822
:10F0A00083818860838349815A818091B7089091D8
:10F0B000B8082CD0E091B708F091B8082381277FD9
:10F0C0002383E2E02296AFCDA0E1B0E0E9E6F8E7E5
:10F0D0008CCD0F89188D8EE08E831C830B838FEF70
:10F0E0009FE798878F83AE01455E5F4F5A834983C0
:10F0F000698D7A8DCE01039609D029853A85020F54
:10F10000131FF8011082E4E060968BCD2F923F929E
:10F110005F926F927F928F929F92AF92BF92CF92A7
:10F12000DF92EF92FF920F931F93CF93DF93CDB7B0
:10F13000DEB72B970FB6F894DEBF0FBECDBF3C01F4
:10F140004B016A01FC0117821682838181FD03C095
:10F150008FEF9FEFAEC11E010894211C311CF301FB
:10F160003381F40133FD859133FF81914F01882371
:10F1700009F49CC1853239F433FD859133FF8191C7
:10F180004F01853221F4B30190E0F7D1E8CF982FF9
:10F1900010E05524AA241032B0F49B3269F09C325E
:10F1A00028F4903251F0933271F40BC09D3239F053
:10F1B000903349F411602AC01260146027C01860AF
:10F1C00025C0106123C017FD2AC0292F20532A30E3
:10F1D00088F416FF07C08AE0A89EC0011124A22E61
:10F1E000A80E14C08AE0589EC0011124522E580E59
:10F1F00010620CC09E3221F416FD58C1106406C086
:10F200009C3611F4106802C0983649F4F40133FDBD
:10F21000959133FF91914F01992309F0BCCF892F2C
:10F220008554833018F08052833038F424E030E085
:10F23000C20ED31E8FE389830FC0933631F093370C
:10F2400081F0933509F052C01FC0F6018081898397
:10F2500022E030E0C20ED31E710181E0A82EB12C55
:10F2600011C0F601E080F18016FD03C06FEF7FEF63
:10F2700002C06A2D70E022E030E0C20ED31EC7014A
:10F2800061D15C011F7712C0F601E080F18016FDAC
:10F2900003C06FEF7FEF02C06A2D70E022E030E024
:10F2A000C20ED31EC70143D15C01106813FF06C014
:10F2B00019C0B30180E290E060D15A94852D90E0AE
:10F2C000A816B906B0F30EC0F70117FD859117FF18
:10F2D00081917F01B30190E050D151105A9408946C
:10F2E000A108B108A114B10479F7DDC0943611F07A
:10F2F000993661F517FF0AC0F6016081718182813C
:10F30000938124E030E0C20ED31E0DC0F60180814F
:10F3100091819C01B901882777FD8095982F42E063
:10F3200050E0C40ED51E012F0F7697FF08C09095B0
:10F330008095709561957F4F8F4F9F4F00682AE0B1
:10F3400030E0A10146D1B82EB2183CC0953721F467
:10F350001F7E2AE030E01CC0197F9F3661F0903795
:10F3600020F4983509F0A2C00FC0903739F09837D3
:10F3700009F09CC004C028E030E00AC0106114FD10
:10F38000146020E130E004C014FD166020E132E09A
:10F3900017FF08C0F601608171818281938144E08A
:10F3A00050E008C0F60180819181BC0180E090E0CE
:10F3B00042E050E0C40ED51EA1010BD1B82EB21808
:10F3C000012F0F7706FF09C00E7FBA1430F404FF37
:10F3D00006C002FD04C00F7E02C01B2D01C01A2D05
:10F3E00004FF0CC0FE01EB0DF11D8081803311F490
:10F3F000097E08C01F5F02FF05C003C0802F86780A
:10F4000009F01F5FE02E03FD13C000FF0EC01515AD
:10F4100010F0AB2C0AC0AB2CA50CA11A152D05C001
:10F42000B30180E290E0A9D01F5F1515C8F304C0B6
:10F43000151510F4511A01C05524E4FE0FC0B30194
:10F4400080E390E09AD0E2FE1CC0E1FE03C088E5B4
:10F4500090E002C088E790E0B3010CC08E2D867862
:10F4600081F0E1FE02C08BE201C080E207FD8DE287
:10F47000B30190E082D005C0B30180E390E07DD07D
:10F48000AA94BA14C8F3BA94F101EB0DF11D80816E
:10F49000B30190E072D0BB2031F0F5CFB30180E230
:10F4A00090E06BD05A945520C9F759CEF30186816C
:10F4B00097812B960FB6F894DEBF0FBECDBFDF91BC
:10F4C000CF911F910F91FF90EF90DF90CF90BF9061
:10F4D000AF909F908F907F906F905F903F902F9014
:10F4E0000895DC01CB01FC01F999FECF06C0F2BD05
:10F4F000E1BDF89A319600B40D9241505040B8F7F2
:10F500000895F999FECF92BD81BDF89A992780B5EB
:10F510000895262FF999FECF1FBA92BD81BD20BD57
:10F520000FB6F894FA9AF99A0FBE01960895FC0165
:10F530000590615070400110D8F7809590958E0F1E
:10F540009F1F0895FC016150704001900110D8F791
:10F55000809590958E0F9F1F0895DC01FC01672F09
:10F5600071917723E1F7329704C07C916D9370839A
:10F570006291AE17BF07C8F308950F931F93CF93FF
:10F58000DF938C01EB018B8181FF1BC082FF0DC0DB
:10F590002E813F818C819D812817390764F4E88191
:10F5A000F9810193F983E88306C0E885F985802F06
:10F5B0000995892B31F48E819F8101969F838E83DB
:10F5C00002C00FEF1FEFC801DF91CF911F910F9184
:10F5D0000895FA01AA27283051F1203181F1E894E9
:10F5E0006F936E7F6E5F7F4F8F4F9F4FAF4FB1E036
:10F5F0003ED0B4E03CD0670F781F891F9A1FA11D31
:10F60000680F791F8A1F911DA11D6A0F711D811D31
:10F61000911DA11D20D009F468943F912AE0269FF6
:10F6200011243019305D3193DEF6CF010895462F55
:10F630004770405D4193B3E00FD0C9F7F6CF462F36
:10F640004F70405D4A3318F0495D31FD405241939F
:10F6500002D0A9F7EACFB4E0A6959795879577955C
:10F660006795BA95C9F700976105710508959B01E3
:10F67000AC010A2E06945795479537952795BA956C
:10F68000C9F7620F731F841F951FA01D0895FFCF38
:10F690004D4350636F6E6669670000000000000014
:10F6A000000000002F002F006F6666006F66660086
:10F6B0006F6666002000BB08000003FF0102036FB5
:10F6C000551CC801C0A8B26FFFFFFF00C0A8B2015F
:10F6D000C0A8B20100000003000000009E41734179
:10F6E0000000FFFFFFFFFFFF2F00CC21D621DD210F
:10F6F000F3210A22102224223E22D9195B1907196C
:10F70000FB18FB18108500228D00289400009C0037
:0EF7100001030507090E10121416181C1E0026
:00000001FF
